:020000021000EC
:10FC00000C9446FE0C9463FE0C9463FE0C9463FE0D
:10FC10000C9463FE0C9463FE0C9463FE0C9463FEE0
:10FC20000C9463FE0C9463FE0C9463FE0C9463FED0
:10FC30000C9463FE0C9463FE0C9463FE0C9463FEC0
:10FC40000C9463FE0C9463FE0C9463FE0C9463FEB0
:10FC50000C9463FE0C9463FE0C9463FE0C9463FEA0
:10FC60000C9463FE0C9463FE0C9463FE0C9463FE90
:10FC70000C9463FE0C9463FE0C9463FE0C9463FE80
:10FC80000C9463FE0C9463FE0C9463FE11241FBE5F
:10FC9000CFEFD0E1DEBFCDBF11E0A0E0B1E0E0E505
:10FCA000FFEF01E00BBF02C007900D92A030B1073B
:10FCB000D9F712E0A0E0B1E001C01D92A330B10776
:10FCC000E1F70C9452FF0C9400FE5F9BFECF8CB1C9
:10FCD0009927382F22272115310521F081E08093C3
:10FCE000000202C0109200025F9BFECF8CB1280F71
:10FCF000311DC90130930202209301022FEF8F3F83
:10FD0000920731F0982F8827909302028093010286
:10FD100008951BBE81E085BF15BE1F921F920895F6
:10FD2000089540E0E0E0F1E02FEF30E05F9BFECF90
:10FD30008CB199278193480F2150304037FFF6CF7F
:10FD40005F9BFECF8CB120E030E0481711F421E03A
:10FD500030E0C90108958BB1992787FD90958827D8
:10FD6000990F881F992708958CB1992708955D9B55
:10FD7000FECF8CB908950F931F93CF93DF9300E0CC
:10FD800010E0C0E0D1E080910002882311F081E012
:10FD90008BBF809101029091020260E0800F911F61
:10FDA000BBD01BBE488129813327322F2227240F45
:10FDB000311D8217930719F080E090E009C00E5FB3
:10FDC0001F4F229681E000301807E9F681E090E0AD
:10FDD000DF91CF911F910F9108950F931F93CF93B0
:10FDE000DF9300E010E0C0E0D1E02881898199270D
:10FDF000982F8827B801820F911D83D00E5F1F4F67
:10FE0000229681E00030180781F780910002882354
:10FE100011F081E08BBF63E08091010290910202BA
:10FE200069D065E0809101029091020263D07FD099
:10FE3000DF91CF911F910F9108955D9BFECF84E4D8
:10FE40008CB95D9BFECF80E78CB95D9BFECF83E6CE
:10FE50008CB95D9BFECF84E58CB98CB15D9BFECFE8
:10FE600081E28CB932DF80910102909102028F5FB2
:10FE70009F4F39F41BBE81E085BF15BE1F921F92B4
:10FE800008954FDF882351F0A8DF75DF882319F02C
:10FE90005D9BFECFE5CF5D9BFECF02C05D9BFECF9D
:10FEA00080E4DFCFF894189A1AB81BB886E88093DC
:10FEB00095001092900088E18AB98CE089B98E9AF9
:10FEC000139A1B9A3FD03ED03DD08CB15D9BFECFA4
:10FED0008EE38CB937D036D035D034D08CB18C335A
:10FEE00009F4ABDF1BBE81E085BF15BE1F921F92D8
:10FEF0000895089522D0F92FE82F60936800E895BF
:10FF000008951BD0F72FE62F192E082E31E03093DD
:10FF10006800E89511240895F92FE82F60FD60939B
:10FF20006800C895802DE395C895902D089505D05B
:10FF3000B1E1B0936800E8950895B0916800B0FD14
:10FF4000FCCF0895AFEFBCE71197B7FFFDCF089541
:040000031000FC00ED
:100000000C948D0D0C949F560C94AA0D0C94AA0D73
:100010000C94AA0D0C94AA0D0C94AA0D0C94AA0D84
:100020000C94AA0D0C94AA0D0C94AA0D0C94AA0D74
:100030000C94AA0D0C94AA0D0C94AA0D0C942512E4
:100040000C94AA0D0C9488560C94F6540C94AA0D9A
:100050000C94AC540C9402570C94AA0D0C94AA0D59
:100060000C94AA0D0C94AA0D0C94AA0D0C94AA0D34
:100070000C94AA0D0C94AA0D0C941B550C94AA0D6B
:100080000C94D1540C94AA0D0C94AA0D412000009C
:1000900042C80000461C40004CBEBC205A0E1BCA81
:1000A000749DC5AE3DCCCCCD3C23D70A38D1B71713
:1000B000322BCC7724E695950A4FB11F0639652C73
:1000C000033AA23B593C1EBAE03D633BF43E75FF48
:1000D0004E3F3172113F800000000540B504F441ED
:1000E000A0000141E2463241A0000040E246303F1C
:1000F0008000000541778C4F40C32CE24117BF249C
:10010000C1A48DD9C0E1D8A1C05B67820000000006
:10011000002070707070707070707070707070709F
:1001200070707070707070707070707070707070CF
:1001300070707070707070707070707070707070BF
:1001400070707070707070707070707070707070AF
:10015000707070707070707070707070707070709F
:10016000707070707070707070707070707070708F
:10017000707070707070707070707070707070707F
:10018000707070707070702000000000000000003F
:10019000000000000000000000000000000000005F
:1001A0000000000000000000E0F0F838383838386F
:1001B000383838383838383838380000F8F8F80027
:1001C00000008080C0E0E0F070783838181808002F
:1001D000F8F8F80000000000000000000000000037
:1001E000F8F8F80000000000000000000000000027
:1001F00000000000000000000000000000000000FF
:1002000000000000000000000000000000000000EE
:1002100000000000000000000000000000000000DE
:1002200000000000000000000103070707070707A0
:10023000070707070707078FFEFEFC00FFFFFF0EFB
:100240001F1F3B7B71F1E0E0C0C080000000000098
:100250000F1F1F3C3838383838383838383838B8F5
:10026000FFFFFF0000000000000000000000000091
:10027000000000000000000000000000000000007E
:10028000000000000000000000000000000000006E
:10029000000000000000000000000000000000005E
:1002A0000000000000000000070707070707070716
:1002B00007070707070707070303010007070700EA
:1002C0000000000000000001010303070706060408
:1002D00004000007070707070707070707070707BF
:1002E0000303010000000000000000000000000007
:1002F00000000000000000000000000000000000FE
:1003000000000000000000000000000000000000ED
:1003100000000707070707070707FFFFFF07070793
:10032000070707070700FFFFFF070707070707077C
:10033000070707070707FFFEFC0000F8FCFE1E0F7B
:100340000707070707070707070F0EFEFCF800005F
:1003500000010307070F1E3C3878F0E0C0C0E0E062
:10036000F0783C1C1E0F0703030100010307070F71
:100370001E3C3878F0E0C0C0E0E0F0783C1C1E0F76
:10038000070303010000000000000000000000005F
:1003900000000000000000000000FFFFFF00000060
:1003A000000000000000FFFFFF0707070F0F1F1FDF
:1003B0003F3F7777E7E7C7C3818000FFFFFF07076D
:1003C0000707070707070707070707FFFFFF0000E3
:1003D0000080C0C0E0F078383C1E0F070703070F0D
:1003E0000E1E3C7870F0E0C080800080C0C0E0F05D
:1003F00078383C1E0F070703070F0E1E3C7870F07D
:10040000E0C080800000000000000000000000004C
:100410000080C0C0C0C0C0C0C0C0C0C0C0C0C0C0DC
:10042000C0C0C0C0C0C0C0C0C0C0C0C0C0C0C0C0CC
:10043000C0C0C0C0C0C0C0C0C0C0C0C0C0C0C0C0BC
:10044000C0C0C0C0C0C0C0C0C0C0C0C0C0C0C0C0AC
:10045000C0C0C0C0C0C0C0C0C0C0C0C0C0C0C0C09C
:10046000C0C0C0C0C0C0C0C0C0C0C0C0C0C0C0C08C
:10047000C0C0C0C0C0C0C0C0C0C0C0C0C0C0C0C07C
:10048000C0C0C0C0C0C0C0800000000000000000AC
:10049000000001010101010101010101010101014E
:1004A000010101010101010101010101010101013C
:1004B000010101010101010101010101010101012C
:1004C000010101010101010101010101010101011C
:1004D000010101010101010101010101010101010C
:1004E00001010101010101010101010101010101FC
:1004F00001010101010101010101010101010101EC
:100500000101010101010100000000000B500A146B
:100510004E0A0D0F0C0F0E0C0D0C0F17FFFFFFFFF7
:100520003FFEF8C000FFFFFFFFFFFFFFFF000007D7
:100530001F7FFFFFFFFF0000000000000000000021
:10054000000000E0F8FCFE1F0F0707070F1FFEFC6E
:10055000F8E0071F3F7F78F0E0E0E0F0F87F3F1F12
:100560000700000000000000000000000000000084
:10057000FFFFFFFF0707078FFFFEFEF8FFFFFFFFEC
:100580000707070707030100000000000000000044
:1005900000000000E0F8FCFE1F0F0707070F1FFE1A
:1005A000FCF8E0071F3F7FF8F0E0E0E0F0F87F3F65
:1005B0001F07000000000000003070F0F0E0E0E0F5
:1005C000E0FFFFFFFF878787C7FFFFFE7C0000FF7C
:1005D000FFFFFF03070F3F7FFDF8E0C08000000032
:1005E000000000000000000000000078FCFEFFE7B3
:1005F000C7C7C7878E1E007870F1E1E3E3E3F7FF1A
:100600007F3F1E0000000000000000000000000707
:1006100007070707FFFFFFFF0707070700000000A6
:1006200000FFFFFFFF0000000000000000000000CE
:10063000000000000000FFFFFFFF00000000FFFFC0
:10064000FFFF1F3F7FFFF0E0E0F0FF7F3F1F000054
:1006500000000000000000000000010F7FFFFEF01E
:10066000800080F0FEFF7F0F01000000031FFFFFEE
:10067000FCFFFF1F0300000000000000000000005E
:1006800000000000000000033FFFFFFCC00000F07E
:10069000FFFF3FFFFFF88000C0FCFFFF3F030000AB
:1006A000011FFFFFF8FFFF1F0100031FFFFFFCFFFB
:1006B000FF1F01000000000000000000000000001B
:1006C00000000000000000000000000000330A01EC
:1006D00030050406080A0C8080808080808080803D
:1006E000808080808080808080808080808080800A
:1006F0008080808080808080808080808080802159
:10070000D00A0E206000020506070809020303054F
:100710000802040204070407070707070707070280
:1007200002070707080E0908080807070908020753
:1007300008070B0809070909070808090D07080831
:100740000404040608030707060707050707020352
:1007500006020A0707070705060507070B06070530
:100760000501050708FEFE18181E1E001E1E0000CB
:1007700000000090F89E90F89E1C00001C000018DD
:100780003C26FF66CC88040C183C180C041C221C68
:10079000C0308E408000001804000C100C80CC7E0D
:1007A00072F2DE0C80000C1C1010101C0C1C101EB1
:1007B0001E0000F0FC061C7CC006FCF0C07C1C1473
:1007C000140E14140000000000606060FCFC606007
:1007D000600000000C0C00000000005838C0C0C0D1
:1007E000C0000000000000181800C03806180400FF
:1007F00000F8FC0E060EFCF8040C1C181C0C041867
:100800000CFEFE00001C1C181C86C6663E1C181C34
:100810001C18181818888C062626FEDC040C1C18D8
:10082000180C04C0E0B88CFEFE80040404041C1CF8
:1008300004707E3E3636F6C60C1C1818180C04F8E8
:10084000FC6E6666EECC040C1818181C0C06060626
:10085000E6761E0600001C1C0000009CFE66666614
:10086000FE9C0C1C1818181C0C3C7E666666FCF876
:100870000C1C18181C0C0418181818181858384094
:10088000E0F0F8FCFEFF0000040C1C3C7CD8D8D83B
:10089000D8D8D8D800000000000000FFFEFCF8F017
:1008A000E0407C3C1C0C040000080C06C6E6763CCC
:1008B000180000001818000000E03008C4F63A1ACA
:1008C0001AF2FA7E0408F00C30604C9C98988C9CCC
:1008D0009C90484C2000C0F8BE86BEF8C000181C92
:1008E00004040404041C18FEFE66666666FEDC1C36
:1008F0001C181818181C0CF8FC0E06060E9C080490
:100900000C1C18181C0C04FEFE0606060EFCF81C37
:100910001C1818181C0C04FEFE66666666661C1C15
:100920001818181818FEFE66666666061C1C00007D
:10093000000000F8FC0E0606C6CEDCC8040C1C182D
:100940001818180C04FEFE60606060FEFE1C1C009F
:100950000000001C1CFEFE1C1C8080000000FEFE2F
:100960000C1C1818181C0CFEFE603078EC86021C5B
:100970001C000000041C18FEFE00000000001C1CEF
:100980001818181818FEFE0E7CE000E07C0EFEFE23
:100990001C1C00000C1C0C00001C1CFEFE1C78E043
:1009A00080FEFE1C1C0000040C1C1CF8FC0E06063D
:1009B000060EFCF8040C1C1818181C0C04FEFE662D
:1009C00066667E3C1C1C0000000000F8FC0E0686DB
:1009D000060EFCF8040C1C18181C0C1C24FEFE66E9
:1009E00066E6E6BE1C001C1C0000000C1C18103C37
:1009F0007E666666EECC0C1C1818181C0C060606E3
:100A0000FEFE0606060000001C1C000000FEFE00A4
:100A1000000000FEFE040C1C18181C0C04021EFC36
:100A2000E000E0FC1E020000001C1C1C0000000690
:100A3000FEF800F0FE0EFEF000F8FE0600001C1CA2
:100A40001C0000001C1C1C0000060EF8F0F80E062E
:100A5000181C0400041C18060E38F0F0380E0600AE
:100A600000001C1C000000060686E6761E0E061816
:100A70001C1C1818181818FEFE0606FCFCC0C00640
:100A800038C000000004180606FEFEC0C0FCFC20B2
:100A9000380E0E38200000000000000000000000AA
:100AA000000000808080808080808002060400003A
:100AB000001098D858F8F0000C1C18180C1C10FEE8
:100AC000FE301838F0E01C1C0C181C0C04E0F01868
:100AD000183830040C18181C0CE0F0381830FEFEE2
:100AE000040C1C180C1C1CE0F0D8D8D8F0E0040C46
:100AF000181818180818FCFE1A1A001C1C0000E030
:100B0000F0381830F8F864ECDCD8CCFC7CFEFE3011
:100B10001818F8F01C1C0000001C1CFAFA1C1C0021
:100B2000FAFAC0FC7CFEFEE0F098081C1C00041CD5
:100B300018FEFE1C1CF8F81018F8F01818F8F01C35
:100B40001C00001C1C00001C1CF8F8301818F8F0E1
:100B50001C1C0000001C1CE0F0381838F0E0040CED
:100B60001C181C0C04F8F8301838F0E0FCFC0C18C9
:100B70001C0C04E0F0381830F8F8040C1C180CFCBD
:100B8000FCF8F83018181C1C00000070F8D8D8D8F1
:100B900090081818181C0C18FCFE1818000C1C18CB
:100BA00018F8F8000000F8F80C1C18180C1C1C3879
:100BB000F8C000C0F83800001C1C1C000018F8E049
:100BC00000F038F000E0F81800001C1C0C000C1CB1
:100BD0001C00001838E0E03818181C04041C181811
:100BE000F8E000E0F8180084FCF83C04001898D8FD
:100BF00078381C1C18181880FC7E0606007CFCC087
:100C0000C0FEFC06067EFC80C0C0FC7C006030306C
:100C10007060603000000000000000FE020202026E
:100C20000202FE1C1010101010101C009F0A052B51
:100C3000030A0A0AF8F8F8F8F8F8F8F8F870F8F87B
:100C4000F8F8F8888888F870F8888888888888880C
:100C5000F8700D600A152B100D060604090C0C0C1B
:100C60000C0C0C0C0C0C0C0400000000000000002C
:100C70000000000000000000000000000000000074
:100C80000000000000000000000000000000000064
:100C900000000000000080E0E0E020C0F8781800CC
:100CA000000000000000000707070707070000001A
:100CB00000000000000000E0E0E0E0080808080094
:100CC000000000E0FCFF1F030080F0FF7F0F00002A
:100CD00000607878180000000000E0F8FCFE1E0EAE
:100CE0000E1EFEFCF8E01F7FFFFFE0C0C0E0FFFF2C
:100CF0007F1F0000000808080808080000000038EE
:100D00003838FEFEFEFE0000000000C0C0C0FFFF3D
:100D1000FFFFC0C0C000000808080808080808084D
:100D200008001C1E0E0E0E0E1EFEFCFCF000C0E0A5
:100D3000F0F8F8FEDFCFC7C3C0C0080808080808ED
:100D40000808080808081C1E0E0E8E8E8ECEFEFCAB
:100D50007C38E0E0C0C0C3C3C3E7FFFE7E3C0008B0
:100D6000080808080808080000000000C0E0381C57
:100D7000FEFEFEFE00001E1F1D1C1C1CFFFFFFFFD1
:100D80001C1C00000000000008080808000000FE0D
:100D9000FEFEFE8E8E8E8E0E0E0EE0E3C3C3C3C328
:100DA000C3E7FFFF7F3E00080808080808080000A6
:100DB0000000C0F0F8FCBCDECECECECE8E001F7F91
:100DC000FFFFE1C1C1E3FFFF7F3E0000000808080C
:100DD0000808080000000E0E0E0E0E0ECEFEFEFEDF
:100DE0007E1E0000C0F0FCFF7F1F0701000000080E
:100DF0000808080800000000000078FCFCFECE8E09
:100E00008E8EFEFCFC3878FCFFFFE3C3C3C7FFFEF9
:100E1000FE3C000000080808080808000000F0F880
:100E2000FCFE1E0E0E1EFEFCF8E001E7CFCFCFCE7B
:100E3000EEF6FF7F3F0F00080808080808000000D2
:100E40000000E0E0E0E0E1E1E1E1080808080F89E6
:100E50000A102D130604001212121212121212128C
:100E600012101003030310C0C0C0C0C0C0010101B4
:100E700001010100000000E0E0E0E0FCFEFEFF0FE9
:100E800007070707070707070FFFFEFEFC3F7F7FE7
:100E90007FF0E0E0E0E0E0E0E0E0F0FF7F7F3F00B7
:100EA00007070707070FFEFEFEFC0000000000001A
:100EB0000000000000000000FFFFFFFF0000000036
:100EC00000000080C0C7E7E7E7E7E7E7E7E7E7E715
:100ED000E7FF7E7E3CFFFFFFFFE1E0E0E0E0E0E0D7
:100EE000E0E0E0E0E0E0E00707C7C7C7C7C7C7C763
:100EF000C7C7C7C7C7FFFEFEFCE0E0E1E1E1E1E1F3
:100F0000E1E1E1E1E1E1E1FF7F7F3FFFFFFFFF8002
:100F10000000000000000000F8F8F80000010103E4
:100F200003070707070707070707FFFFFF07073F35
:100F30007F7F7FF7E7E7E7E7E7E7E7E7E7E7E7E769
:100F4000E7E0E0E0E0E0E0E0E0E0E0E0E0E0F07FEB
:100F50007F3F1FFCFEFEFFE7E7E7E7E7E7E7E7E79E
:100F6000E7E7C7C0803F7F7FFFF1E0E0E0E0E0E03F
:100F7000E0E0F17F7F7F3F07070707070707078745
:100F8000C7E7F7FF7F3F1F0F0780C0E0F0F87C3E08
:100F90001F0F070301000000000000FCFEFEFFC75A
:100FA000C7C7C7C7C7C7C7C7C7FFFEFEFC3F7F7F0E
:100FB000FFE1E1E1E1E1E1E1E1E1E1FF7F7F3FFC30
:100FC000FEFEFF8F07070707070707078FFFFEFED5
:100FD000FC0103E3E3E7E7E7E7E7E7E7E7E7F7FF36
:100FE0007F7F3F00000000000000000000000000C4
:100FF000000000E0A0A0A0A0A0A0A0A0A0A0A0A091
:10100000A0A0A00000000000000000000000000000
:10101000000000A0A0A0A0A0A0A0A0A0A0A0A0A0B0
:10102000A0A0E0FF01FFFF00FFFF00FFFF80FFFF28
:1010300000FFFF00FF0000000000000000000000B3
:101040000000000000A0A0A0A0A0A0A0A0A0A0A0C0
:10105000A0A0A0A0A0024A0A102B04050D0909BCFB
:10106000A0BC043CF784B794F41F1010001F1111AA
:101070001F001F11151D00000000000000000000EF
:101080000000001D151517001F11110E00000000B3
:1010900000000000001115151F001F11110E0000A7
:1010A00000000000000000013D053E2B01051C086A
:1010B0000808C83D253D2525C0404040C0EB2AEA30
:1010C0004A2BBDA5BD2525080808050278407808EB
:1010D000783C202C243C31C80A2B300A1E151E1ED9
:1010E000221E1F1D1E1F000080C0F0F8F8FCFEFE2F
:1010F000FE7F3F3F3F3F3F3F7FFEFEFEFCF8F0E0BC
:10110000C0000000C0FCFFFFFFFFFFFF3F03000027
:101110000000000000000000031FFFFFFFFFFFFFB3
:10112000FCC0FFFFFFFFFFFFFFFF0000000000000B
:101130000000000000000000FFFFFFFFFFFFFFFFB7
:101140001FFFFFFFFFFFFFFFE000000000000000A7
:101150000000000000E0FFFFFFFFFFFFFF1F000196
:10116000071F3F7FFFFFFFFEF8F0F0E0E0E0E0E068
:10117000F0F8FEFFFFFF7F3F1F07010000000000A7
:1011800000000020206060E0E0E0E0E0E0E0E060FF
:1011900060202000000000000000000000000000AF
:1011A0000000000080C0E0F8FCFEFFFFFFFEFCE056
:1011B000F0F0F8F8FCFCFE7F7F3F1F0FFFFFFFFF02
:1011C000FFFFFFFF01030303030101000000000014
:1011D00000FFFFFFFFFFFFFFFF0000000000000017
:1011E000000000000000FFFFFFFFFFFFFFFF000007
:1011F0000000000000000000000000FFFFFFFFFFF4
:10120000FFFFFF00000000000000000000000000E1
:101210002060E0E0E0E0602000C0E0F0F8FCFCFED0
:10122000FEFE7F7F3F3F3F3F3F7F7FFEFEFEFCFC99
:10123000F8F0E0C000003E7FFFFFFF7F3F070100A6
:101240000000000000000000000083FFFFFFFFFF20
:10125000FFFFFE0000000000000000000000000092
:101260000080C0E0E0F0FCFEFFFFFF7F3F1F0F03A8
:1012700000000000000080C0E0F0F8FCFEFEFFFF70
:101280007F3F1F0F0F070301000000000000000058
:10129000F0FCFEFFFFFFFFFFFFFFF7F3F1F0F0F0C0
:1012A000F0F0F0F0F0F0F0F0F0F0F0F0E0C02060DE
:1012B000E0E0E0E0E0E0E0E0E0E0E0E0E0E0E0E02E
:1012C000E0E0E0E0E0E0E0E0E0E060200000C0E03E
:1012D000F0F8FCFCFEFE7E3F3F3F3F3F3F7F7FFE3E
:1012E000FEFEFCFCF8F0E000000000070F1F1F1FCF
:1012F0001F070100000000000000000080C1FFFF88
:10130000FFFFFFFFFF1F00000000000000000000C3
:10131000387C7E7E7E7E7E7E7F7FFFFFFFFFFFF735
:10132000F3E1C0800000C0E0F0F0F0E0C000000099
:10133000000000000000000000000107FFFFFFFFA9
:10134000FFFFFFFC030F1F7FFFFFFFFFFCF8F0F024
:10135000E0E0E0E0E0F0F0F8FCFEFFFFFF7F3F1F81
:101360000F0100000000000020206060E0E0E0E0ED
:10137000E0E0E0E0E06060602020000000000000AD
:1013800000000000000000000000000000000080DD
:10139000C0E0F8FCFEFFFFFFFFFFFEFC00000000C6
:1013A000000000000000000000000080C0F0F8FC19
:1013B000FEFF7F3F0F07FFFFFFFFFFFFFFFF000064
:1013C0000000000000000080C0F0F8FCFFFFFF3FBD
:1013D0001F07030000000000FFFFFFFFFFFFFFFFEC
:1013E000000000000000F8FCFFFFFFFFFFFFF3F12B
:1013F000F0F0F0F0F0F0F0F0F0F0FFFFFFFFFFFF93
:10140000FFFFF0F0F0F0F0E000010303030303033B
:10141000030303030303030303030303FFFFFFFFAC
:10142000FFFFFFFF030303030301000000000000B0
:10143000000000000000000000000000000020602C
:10144000E0E0E0E06020000000000000000000C0DC
:10145000FCFEFFFFFFFF7F7F7F7F7F7F7F7F7F7FA0
:101460007F7F7F7F7F7F7F3E1C000000F8FFFFFFB4
:10147000FFFFFF1F808080C0C0C0C0C0C0C0808090
:101480008000000000000000007EFFFFFFFFFF7FE4
:101490003F3F1F0F0F0F0F0F0F1F1F3F7FFFFFFF5C
:1014A000FEFEFCF0E000C0E0E0E0E0C080000000F4
:1014B000000000000000000000000001FFFFFFFF2F
:1014C000FFFFFFFF071F3F7FFFFFFFFEFCF8F0F06D
:1014D000E0E0E0E0E0F0F0F8FCFFFFFFFF7F3F0F0F
:1014E000070000000000002020606060E0E0E0E015
:1014F000E0E0E0E0E060606020000000000000004C
:1015000000000080C0F0F0F8FCFCFEFE7F7F3F3F53
:101510003F3F3F7F7FFEFEFEFCF8F0E0C000000092
:10152000F0FEFFFFFFFFFFFF0F0300000080808041
:10153000808080808103070F0F0F0F070000FFFFDF
:10154000FFFFFFFFFFFFF1F8FC7E3F3F1F1F1F1F44
:101550001F3F7FFFFFFFFEFEFCF8F0C0001FFFFFF4
:10156000FFFFFFFFFFFF030000000000000000007E
:1015700000000003FFFFFFFFFFFFFFFE0001071F4A
:101580003F7FFFFFFFFFFCF8F0F0E0E0E0E0E0F07D
:10159000F8FCFFFFFFFF7F3F1F0701000000000076
:1015A00000002020606060E0E0E0E0E0E0E0E0607B
:1015B000606020200000000000001E3E7F7F7F7FD3
:1015C0007F7F7F7F7F7F7F7F7F7F7F7F7F7FFFFF2B
:1015D000FFFFFFFFFF7E1C00000000000000000076
:1015E000000000000080C0F0FCFEFFFFFF3F1F076F
:1015F000030000000000000000000000000080E088
:10160000F8FEFFFFFFFF3F070100000000000000A1
:10161000000000000000000080F0FEFFFFFFFFFF61
:10162000FF0F0000000000000000000000000000AC
:1016300000000000F8FFFFFFFFFFFFFF7F01000039
:10164000000000000000000000000000000000009A
:10165000000060E0E0E0E06020000000000000002A
:101660000000000000000000000080E0F0F8FCFC3A
:10167000FEFEFF7F3F3F3F3F3F3F7FFEFEFEFCFC05
:10168000F8F0E0800000000C7FFFFFFFFFFFFFC1CC
:1016900080000000000000000080C3FFFFFFFFFF8C
:1016A000FF7F0000000080C1E3E7F7FFFFFFFFFFBF
:1016B0007E7E7E7E7E7EFFFFFFFFFFF7E7E3C18039
:1016C0000000F8FFFFFFFFFFFFFF07010000000021
:1016D0000000000000000107FFFFFFFFFFFFFFF811
:1016E000030F3F7FFFFFFFFFFEFCF8F0E0E0E0E0CC
:1016F000E0E0F0F8FCFEFFFFFFFF7F3F0F0300007C
:101700000000002020606060E0E0E0E0E0E0E0E079
:10171000E0E0606060202000000000000000C0E009
:10172000F0F8FCFCFEFEFE7F3F3F3F3F3F7F7FFE29
:10173000FEFEFCFCF8F0E0C0000000F8FFFFFFFF39
:10174000FFFFFF0701000000000000000000000193
:101750000FFFFFFFFFFFFFFFFCC0073F7FFFFFFF03
:10176000FFFFFCF0E0C08080808080C0C0E0F0FC23
:10177000FFFFFFFFFFFFFFFFFF0000000103070760
:101780000F0F1F1F1F1F1F1F1F0F0F0F070301FC2E
:10179000FFFFFFFFFFFF7F0700001E7FFFFFFFFE31
:1017A000FCF8F0F0E0E0E0E0E0F0F0F8FCFFFFFF34
:1017B0007F7F1F0F030000000000000020206060FA
:1017C00060E0E0E0E0E0E0E0E0E0606020200000D9
:1017D0000000000000003E002020202020202000EB
:1017E000466C75677A6569742E2E2E3A2020202566
:1017F0003032643A253032643A25303264004D612B
:1018000078686F6568652E2E2E2E3A2020202532AE
:101810002E3066004D61787374656967656E2E3A87
:1018200020202025322E3166004D617873696E6B61
:10183000656E2E2E2E3A20202025322E3166002570
:10184000730025302E31660025730025302E316659
:1018500000257300256400257300256400257300AE
:1018600025302E31660025730025302E3166002587
:10187000730025640025730025640025730025642A
:101880000025730045494E0041555300257300441F
:10189000495200475A004449522F475A004249478B
:1018A0000025302E31660025302E3166002564007B
:1018B00025640025640045494E004155530041759B
:1018C00073005465737400496E666F00456D6572F0
:1018D00067656E63790044495200475A0044495293
:1018E0002F475A004249470024504D4C522C49443E
:1018F0004750532C30312C564152494F2D2C534BCD
:101900005954524158582D2C30303030303030300E
:1019100030312C312E33304745524D414E59303104
:101920002F30392F30362A3536005452415858203E
:101930002020202020204155534C4553454E005631
:101940004F4D0025732E202020253032642E253067
:1019500032642E25303264005370656963686572A5
:101960002020206973742020206C6565722021007E
:10197000417573736368616C74656E3F004F4B20F3
:101980003D20204A410045696E736368616C74654F
:101990006E3F004F4B203D20204A41003300330072
:1019A00025730025322E3066002B002B003A003FB5
:1019B000003F003F003F003F003F003B003A003F38
:1019C000003F003F003F003F003F003B0025322E1C
:1019D0003066002E002D002C0025322E3066002DA2
:1019E000202D202D00253032640025303264002E59
:1019F000002E0025312E30660025312E316600255F
:101A0000312E30660025312E31660025322E3066AB
:101A10000025322E30660025322E3166002D202D15
:101A2000202D00253032643A25322E3466002530D0
:101A300032643A25322E346600536174733A2020A2
:101A4000253032640025322E306620206B6D002553
:101A50006420206D00416B6B753A20202D2D2D00E8
:101A6000416B6B753A202564202068002530326474
:101A70002E25732E25640025303264002530326413
:101A8000003A002D002C002B002B0020545241580E
:101A90005800205345545550002053595354454D38
:101AA00000526573657420202020425400466972FC
:101AB0006D776172650056657273696F6E202020C4
:101AC00020312E332E35004D656E7565746173744B
:101AD0006520202020332020205365632E00676579
:101AE00064727565636B7420202068616C74656E28
:101AF0002021005570646174652020202020206C16
:101B00006165756674210024003031323334353616
:101B10003738394142434445460011241FBECFEFB8
:101B2000D0E1DEBFCDBF14E0A0E0B1E0E4E3FAED28
:101B300000E00BBF02C007900D92AC32B107D9F79D
:101B40001DE0ACE2B4E001C01D92A535B107E1F79C
:101B50000C94CE410C940000CF92DF92EF92FF9252
:101B60000F931F93CF93DF936C017B01EA018DE606
:101B700091E0489F9001499F300D589F300D1124EE
:101B8000C9019A0157FF02C02D5F3F4F3595279538
:101B900035952795280F391FCE0164E670E00E9425
:101BA000536C261B370BCE0160E971E00E94536C29
:101BB000260F371FC901AA2797FDA095BA2F8C01C0
:101BC0009D01F701EE0DFF1DEA5FFE4F80819181BF
:101BD000AA2797FDA095BA2F080F191F2A1F3B1F90
:101BE00093E0E916F104FCF0CE0183709070892B2C
:101BF00021F40F5F1F4F2F4F3F4FCE0164E670E07F
:101C00000E94536C892B21F4015010402040304039
:101C1000CE0160E971E00E94536C892B21F40F5FC3
:101C20001F4F2F4F3F4F0894C108D108C601AA2764
:101C300097FDA095BA2F080F191F2A1F3B1FC90136
:101C4000B801DF91CF911F910F91FF90EF90DF903E
:101C5000CF9008959F92AF92BF92CF92DF92EF9272
:101C6000FF920F931F93CF93DF93CDB7DEB72197EA
:101C70000FB6F894DEBF0FBECDBF982EEE24FF2422
:101C8000670157E0A52E6C2D892D0E94A043BB242F
:101C9000092D112780E890E0801B910B181619067A
:101CA000D4F4C7018B0D911D845F9E4F41E050E03D
:101CB000BC01CE01840F951F0E94C36589810E94DB
:101CC0001344B3942B2D332780E890E0801B910BB5
:101CD0002817390734F3AA9488E090E0C80ED91E7B
:101CE00080E890E0E80EF91EA7FECDCF21960FB652
:101CF000F894DEBF0FBECDBFDF91CF911F910F9142
:101D0000FF90EF90DF90CF90BF90AF909F9008959D
:101D1000CF92DF92EF92FF920F931F93CF93C82E33
:101D2000D62EE42EF22EC0E0C417D0F41C2FCC1611
:101D300049F4812F8F0D682F8D2D0E94A04386EDD1
:101D400097E108C0812F8F0D682F8D2D0E94A04331
:101D500088ED97E10E94F645CF5F100FCE1538F35E
:101D6000CF911F910F91FF90EF90DF90CF9008954A
:101D7000E199FECFF894E3E5F7E0A0E0B0E08FE072
:101D8000182E0E94FC6C789408958CB39927DC017E
:101D9000A270B07081FDF9CFE3E5F7E08FE0182E77
:101DA0000E94F76C089520ED37E040E050E020936A
:101DB000A5073093A6074093A7075093A807209143
:101DC000A5073091A6074091A7075091A807E22FD9
:101DD000F32F3197F1F78A95D1F708958CB39927AE
:101DE000DC01A270B07081FDF9CF0E94EF6C802DF4
:101DF00099270895EF92FF920F931F93E090B907F0
:101E0000F090BA070091BB071091BC078091B5070D
:101E10009091B607A091B707B091B8079C01AD01AA
:101E2000C801B7010E941369181694F420E030E04D
:101E300040E05FE3C801B7010E946168DC01CB01AB
:101E40008093B5079093B607A093B707B093B807F0
:101E5000E090A107F090A2070091A3071091A407BA
:101E60008091620790916307A0916407B091650724
:101E70009C01AD01C801B7010E941369181644F412
:101E8000E0926207F092630700936407109365077E
:101E90008091D00B9091D10BA091D20BB091D30B2C
:101EA0009C01AD01C801B7010E941069882344F468
:101EB000E092D00BF092D10B0093D20B1093D30B86
:101EC0001F910F91FF90EF9008958EE481BF8FE0F6
:101ED00083BF87B7826087BF789408959C01892F5C
:101EE00099278BBD2ABD0895DC01CB019C01AD0172
:101EF000BC01CD010E946168DC01CB019C01AD01F8
:101F000060E074E284EF9AE40E94A368DC01CB01F4
:101F1000BC01CD010E94E968DC01CB010E946E0F7B
:101F20000895CF93DF939C01FB01EA01809120018A
:101F3000882341F1C901AA2797FDA095BA2F2091C6
:101F4000C7073091C8074091C9075091CA07280FA9
:101F5000391F4A1F5B1F80914B0790914C07A0913E
:101F60004D07B0914E0782179307A407B50738F4C1
:101F700080E48FBDBE01CF010E94740F03C01FBC5F
:101F80001092D90BDF91CF9108958BB38A7F8BBBD1
:101F90008BB3897F8BBB8BB3887F8BBB1FBC0895B2
:101FA0003F924F925F926F927F928F929F92AF92E9
:101FB000BF92CF92DF92EF92FF920F931F93CF9336
:101FC000DF93CDB7DEB7C854D0400FB6F894DEBF6C
:101FD0000FBECDBF7AE5E72EF12C6E010894C11C2F
:101FE000D11C88E4E6E2F1E0D60101900D928A95D9
:101FF000E1F74090A1075090A2076090A30770906E
:10200000A40720E030E040EC50E4C301B2010E949C
:10201000136918161CF48CE390E04FC020E030E008
:1020200040EA50E4C301B2010E94136918162CF46F
:10203000F0923504E092340444C020E030E040E8FF
:1020400050E4C301B2010E94136918161CF488E71A
:1020500090E033C020E030E040E450E4C301B2013E
:102060000E94136918161CF484EB90E026C020E04F
:1020700030E040E050E4C301B2010E941369181639
:102080001CF480EF90E019C020E030E040E85FE30E
:10209000C301B2010E94136918161CF48CE291E08E
:1020A0000CC02DEC3CEC4CEC5DE3C301B2010E9492
:1020B0001369181634F488E691E090933504809300
:1020C000340400913404109135040B35110508F4E3
:1020D00078018091530790915407A0915507B091D2
:1020E00056079C01AD01C301B2010E941069181688
:1020F0001CF081E080933204809153079091540743
:10210000A0915507B091560720E030E040E05FE332
:10211000BC01CD010E946168DC01CB019C01AD01D5
:10212000C301B2010E941369882314F01092320493
:102130008091570790915807A0915907B0915A077D
:102140009C01AD01C301B2010E94136988231CF0F8
:1021500081E0809333048091570790915807A091B4
:102160005907B0915A072DEC3CEC4CEC5DE3BC01F7
:10217000CD010E946068DC01CB019C01AD01C3016F
:10218000B2010E941069181634F08091310488233E
:1021900011F48093330430903304B1E03B1609F01E
:1021A00063C080913104882389F5C701AA2797FD70
:1021B000A095BA2F2091360430913704409138040D
:1021C00050913904280F391F4A1F5B1F80914B071C
:1021D00090914C07A0914D07B0914E0728173907F1
:1021E0004A075B0798F480914B0790914C07A091A8
:1021F0004D07B0914E078093360490933704A09317
:102200003804B0933904309231042EC0C801AA2793
:10221000BB27209136043091370440913804509107
:102220003904280F391F4A1F5B1F80914B0790917B
:102230004C07A0914D07B0914E07281739074A0760
:102240005B0790F480914B0790914C07A0914D074C
:10225000B0914E078093360490933704A0933804CE
:10226000B0933904109231044601860104C0E8E0BD
:10227000F0E08E0E9F1ED801AD90BD90CD90DC9009
:10228000085F1F4FA3019201C601B5010E941369A7
:1022900018166CF3A6019501C301B2010E94606893
:1022A0007B018C01E8EFFFEF8E0E9F1EF401808111
:1022B0009181A281B38128E030E0820E931EA601B5
:1022C0009501BC01CD010E946068DC01CB019C013D
:1022D000AD01C801B7010E94A3685B016C01F40164
:1022E000B291A291929182914F0124E030E0820E4E
:1022F000931EF401E480F58006811781A8019701FF
:10230000BC01CD010E946068DC01CB019C01AD01E4
:10231000C601B5010E94C069DC01CB019C01AD0181
:10232000C801B7010E9461687B018C0160933A0487
:1023300070933B0480933C0490933D04A090220151
:10234000B0902301C0902401D09025019B01AC01E5
:10235000C601B5010E94106988234CF425E236E0DD
:1023600041E85FE3C601B5010E94C0691AC023E3DA
:1023700033E343E95FE3C601B5010E94A368DC01D2
:10238000CB01A8019701BC01CD010E941369181669
:1023900094F425E236E041E85FE3C601B5010E940E
:1023A000A368DC01CB018093220190932301A093C9
:1023B0002401B093250180913204813039F0F1E09D
:1023C0003F1641F5809131048F1721F580915D070B
:1023D000813019F48BB385608BBB80915D078230AF
:1023E00019F48BB386608BBB80915D07833019F441
:1023F0008BB387608BBB80E48FBD8091220190916D
:102400002301A0912401B0912501BC01CD010E94BE
:10241000740F02C00E94C50FC85BDF4F0FB6F8945F
:10242000DEBF0FBECDBFDF91CF911F910F91FF9007
:10243000EF90DF90CF90BF90AF909F908F907F9064
:102440006F905F904F903F9008951F920F920FB63C
:102450000F9211242F933F934F935F936F937F932A
:102460008F939F93AF93BF93EF93FF9380914B070D
:1024700090914C07A0914D07B0914E070A96A11D6F
:10248000B11D80934B0790934C07A0934D07B093D9
:102490004E078091490C90914A0CA0914B0CB09141
:1024A0004C0C0196A11DB11D8093490C90934A0CD0
:1024B000A0934B0CB0934C0C80912101813039F5E5
:1024C0008091D90B882319F580914B0790914C0787
:1024D000A0914D07B0914E07BC01CD012EE130E037
:1024E00040E050E00E94666CDC01CB010097A10542
:1024F000B10569F480912001882349F080912C0472
:1025000090912D04806190932D0480932C048091F0
:10251000D7069091D806A091D906B091DA068C59C9
:10252000964EAF4FBF4F20914B0730914C074091D3
:102530004D0750914E0782179307A407B50748F43B
:1025400080912C0490912D04846090932D048093AD
:102550002C0480918A0790918B07A0918C07B091F1
:102560008D078854944FAF4FBF4F20914B07309148
:102570004C0740914D0750914E0782179307A407CF
:10258000B50748F480912C0490912D0480649093B9
:102590002D0480932C048091470790914807A091C7
:1025A0004907B0914A078053984FAF4FBF4F2091D2
:1025B0004B0730914C0740914D0750914E078217C1
:1025C0009307A407B50748F480912C0490912D043B
:1025D000806890932D0480932C048091490C9091F5
:1025E0004A0CA0914B0CB0914C0C4F97A109B1092A
:1025F000893A9105A105B10548F480912C04909188
:102600002D04916090932D0480932C048091D90B1C
:10261000882341F040E050E06CED73E482E390E009
:102620000E94910F21B120953091D40B23279091D6
:102630003E049223909590933E0480913F04822320
:10264000892780933F0498232923932F92279093DF
:10265000D40B92238091C207892B8093C207FF91EC
:10266000EF91BF91AF919F918F917F916F915F910A
:102670004F913F912F910F900FBE0F901F90189583
:10268000E0EDF7E011928BE0EF3CF807D9F3D4F3DB
:102690000895FF920F931F93CF9381E080939A0741
:1026A000FF240F2D1127C801B3E0880F991FBA9599
:1026B000E1F7682F80E00E94A043C0E0F801F695A2
:1026C000FE2FEE27F795E795EC0FF11DE053F84F3D
:1026D00080810E941344CF5FC7FFF0CFF39487E05F
:1026E0008F15F8F610929A07CF911F910F91FF90D6
:1026F000089580E090E0A0E0B0E08093B50790936B
:10270000B607A093B707B093B8078093D00B909308
:10271000D10BA093D20BB093D30B8093620790930D
:102720006307A0936407B09365078091E60B9091CF
:10273000E70BA091E80BB091E90B8093CC07909345
:10274000CD07A093CE07B093CF0780912C04909132
:102750002D049D7F90932D0480932C0408954F9217
:102760005F926F927F928F929F92AF92BF92CF9221
:10277000DF92EF92FF920F931F93CF93C0E06C2EE6
:10278000DC2E80E40E944D5B8823A9F081E08093D9
:10279000D90B80914B0790914C07A0914D07B091B8
:1027A0004E078093C7079093C807A093C907B093BB
:1027B000CA070E94791380912E04882309F4F0C07F
:1027C000E090E60BF090E70B0091E80B1091E90B1D
:1027D000C801B70120E137E240E050E00E94666C9A
:1027E000C22EC801B70124E630E040E050E00E946C
:1027F000666CDC01CB01D82EC801B70120E137E2BD
:1028000040E050E00E94666CDC01CB01ED2CFF241F
:10281000002711278E199F09A00BB10BBC01CD0118
:1028200024E630E040E050E00E94666CD22E8C2D11
:102830009927AA27BB27BC01CD0120E13EE040E05B
:1028400050E00E94146C3B014C018D2D9927AA2762
:10285000BB27BC01CD012CE330E040E050E00E94FA
:10286000146CDC01CB01680E791E8A1E9B1E6E0C57
:102870007F1C801E911EE090CC07F090CD07009148
:10288000CE071091CF07C801B70120E137E240E041
:1028900050E00E94666C422EC801B70124E630E089
:1028A00040E050E00E94666CDC01CB01D82EC801EC
:1028B000B70120E137E240E050E00E94666CDC01A5
:1028C000CB01AD2CBB24CC24DD248A199B09AC0997
:1028D000BD09BC01CD0124E630E040E050E00E949B
:1028E000666C522E842D9927AA27BB27BC01CD01E7
:1028F00020E13EE040E050E00E94146C7B018C013E
:10290000852D9927AA27BB27BC01CD012CE330E0F8
:1029100040E050E00E94146CDC01CB01E80EF91E8F
:102920000A1F1B1FAE0CBF1CC01ED11E6A187B08DD
:102930008C089D08C401B30120E13EE040E050E076
:102940000E94666CD22E822F9927AA27BB27BC0132
:10295000CD0120E13EE040E050E00E94146C7B019C
:102960008C01D401C3018E199F09A00BB10BBC01CE
:10297000CD012CE330E040E050E00E94666CC22FB5
:102980006E18822F9927AA27BB27BC01CD012CE303
:1029900030E040E050E00E94146CDC01CB01681A8A
:1029A0004FEF6CEA72E48FEF96E00E94B04260E075
:1029B00085E00E94A043862D99279F938F938C2FAB
:1029C00099279F938F938D2D99279F938F9380EEB7
:1029D00097E19F938F930E94D36662E185E00E9406
:1029E000A0438DB79EB708960FB6F8949EBF0FBE52
:1029F0008DBF8091B5079091B607A091B707B091B0
:102A0000B807BF93AF939F938F938EEF97E19F93F8
:102A10008F930E94D36664E285E00E94A0438DB745
:102A20009EB706960FB6F8949EBF0FBE8DBF8091DD
:102A3000620790916307A0916407B0916507BF9307
:102A4000AF939F938F9384E198E19F938F930E941C
:102A5000D36665E385E00E94A0438DB79EB70696D6
:102A60000FB6F8949EBF0FBE8DBF8091D00B909192
:102A7000D10BA091D20BB091D30BBF93AF939F9387
:102A80008F9389E298E19F938F930E94D3668DB7CD
:102A90009EB706960FB6F8949EBF0FBE8DBFCF911E
:102AA0001F910F91FF90EF90DF90CF90BF90AF906C
:102AB0009F908F907F906F905F904F90089580E4EB
:102AC0008FBD89E08EBD1FBC80914B0790914C0754
:102AD000A0914D07B0914E078093C7079093C80708
:102AE000A093C907B093CA07D59AD69AD79A80916E
:102AF0005D07882311F48093200190915D07913048
:102B000021F480E28BBB9093200180915D0782309D
:102B100029F480E68BBB81E08093200180915D07E2
:102B2000833029F480EE8BBB81E0809320010895EF
:102B30001F93CF9310E0812F9927C3E0880F991F2F
:102B4000CA95E1F7682F80E00E94A043C0E080E0D2
:102B50000E941344CF5FC7FFFACF1F5F183058F3AE
:102B6000CF911F9108952F923F924F925F926F9253
:102B70007F928F929F92AF92BF92CF92DF92EF920D
:102B8000FF920F931F938091460D9091470DA09156
:102B9000480DB091490D20E030E54DE754E4BC010B
:102BA000CD010E94A368DC01CB0122E534ED42E4B3
:102BB0005EE3BC01CD010E94086ADC01CB019C01EF
:102BC000AD0160E070E080E89FE30E946068DC0196
:102BD000CB0124EC3AE24DE257E4BC01CD010E9466
:102BE000C069DC01CB018093D3069093D406A093F7
:102BF000D506B093D606209081073090820740908A
:102C0000830750908407A2019101BC01CD010E946D
:102C100061687B018C016093B9077093BA07809358
:102C2000BB079093BC078091F60B9091F70B03972D
:102C300009F066C08091EF0B9091F00BA091F10B21
:102C4000B091F20B20E030E040E450E4BC01CD0153
:102C50000E94C0693B014C019B01AC01C801B70156
:102C60000E946168DC01CB01A090B00CB090B10C67
:102C7000C090B20CD090B30CA6019501BC01CD015F
:102C80000E941369181694F420E030E040E85FE3F6
:102C9000C201B1010E946068DC01CB018093810711
:102CA00090938207A0938307B0938407A4019301B4
:102CB000C801B7010E946068DC01CB01A601950143
:102CC000BC01CD010E9410698823D4F48091810752
:102CD00090918207A0918307B091840720E030E0B3
:102CE00040E85FE3BC01CD010E946168DC01CB01DB
:102CF0008093810790938207A0938307B093840702
:102D00001F910F91FF90EF90DF90CF90BF90AF9009
:102D10009F908F907F906F905F904F903F902F90FB
:102D200008958F929F92AF92BF92CF92DF92EF92CF
:102D3000FF920F931F93CF93DF930F2EF0E08F2E10
:102D4000F0E09F2EF0E0AF2EF0E0BF2EF02D80914E
:102D500040048F5F68E20E94336C90934004092F17
:102D60001127000F111F000F111F0F5B1B4FC09089
:102D7000D306D090D406E090D506F090D606809188
:102D8000850790918607A0918707B09188079C01DD
:102D9000AD01C701B6010E946068DC01CB01F801FA
:102DA00080839183A283B383C0928507D0928607E4
:102DB000E0928707F0928807C1E4D4E08991999165
:102DC000A991B9919C01AD01C501B4010E9461684E
:102DD0004B015C01F4E0CD3DDF0781F37CF32DEC8A
:102DE0003CEC4CEC5DE30E9410698823A4F42DECCC
:102DF0003CEC4CEC5DEBC501B4010E941369181664
:102E000054F40F2EF0E08F2EF0E09F2EF0E0AF2E66
:102E1000F0E0BF2EF02D20E030E040EF51E4C5019E
:102E2000B4010E941369181654F40F2EF0E08F2E8F
:102E3000F0E09F2EF0EFAF2EF1E4BF2EF02D20E05A
:102E400030E040EF51ECC501B4010E9410698823C5
:102E500054F40F2EF0E08F2EF0E09F2EF0EFAF2E07
:102E6000F1ECBF2EF02D8092A1079092A207A092C4
:102E7000A307B092A407DF91CF911F910F91FF900C
:102E8000EF90DF90CF90BF90AF909F908F9008957C
:102E9000AF92BF92CF92DF92EF92FF920F931F9368
:102EA000E090D306F090D4060091D5061091D60696
:102EB0008091E1049091E204A091E304B091E404D4
:102EC0009C01AD01C801B7010E9460685B016C0103
:102ED000E092E104F092E2040093E3041093E4042E
:102EE000E090F40CF090F50C0091F60C1091F70CBA
:102EF00020E030E040E050E0C801B7010E941069D6
:102F0000882399F18091A1079091A207A091A3072E
:102F1000B091A4072DEC3CEC4CE45FEBBC01CD017F
:102F20000E94106988230CF5809161078130E9F0D7
:102F30002DEC3BE34EE85EE3C801B7010E94C06997
:102F40007B018C0120E030E040E450ECC601B5018B
:102F50000E94A368DC01CB019C01AD01C801B7014F
:102F60000E94A368DC01CB0104C080E090E0A0E0F7
:102F7000B0E08093D50B9093D60BA093D70BB09372
:102F8000D80B1F910F91FF90EF90DF90CF90BF90E3
:102F9000AF9008952F923F924F925F926F927F92DF
:102FA0008F929F92AF92BF92CF92DF92EF92FF9259
:102FB0000F931F93CF93DF93CDB7DEB7C059D040A7
:102FC0000FB6F894DEBF0FBECDBF80E090E0A0EA60
:102FD000B1E4C358DF4F88839983AA83BB83CD575D
:102FE000D040ED968CAF9DAFAEAFBFAFED9780E018
:102FF00090E0A0EFB1E4CF57DF4F88839983AA8395
:10300000BB83C158D0400F2EF0E0AF2EF0E0BF2EB2
:10301000F0E0CF2EF0E0DF2EF02D2501360180E02C
:1030200090E0A0E0B0E4CB57DF4F88839983AA8378
:10303000BB83C558D04080E090E0A0EAB0E4C75719
:10304000DF4F88839983AA83BB83C958D04080E02F
:1030500090E0A0E8B0E4C357DF4F88839983AA8348
:10306000BB83CD58D0403324E32CF32C11E0912EB8
:10307000832C88E7EEE6F1E0A1E0B0E0AC0FBD1FE5
:1030800001900D928A95E1F7232C80915E078915B6
:1030900009F4292C0E94C50E90929A070E944013B1
:1030A0000E9498154FEF6CEA72E48FEF96E00E9451
:1030B000B042632D8DE00E94A04381E090E08C0F30
:1030C0009D1F9F938F938FE398E19F938F930E940F
:1030D000D366632D86E60E94A0430F900F900F9059
:1030E0000F908091530790915407A0915507B0918C
:1030F0005607BF93AF939F938F9382E498E19F937A
:103100008F930E94D36660E18DE00E94A043ADB72B
:10311000BEB716960FB6F894BEBF0FBEADBF80E126
:1031200090E08C0F9D1F9F938F9388E498E19F936D
:103130008F930E94D36660E186E60E94A0430F90C1
:103140000F900F900F908091570790915807A09182
:103150005907B0915A07BF93AF939F938F938BE416
:1031600098E19F938F930E94D36660E28DE00E9466
:10317000A043ADB7BEB716960FB6F894BEBF0FBE4C
:10318000ADBF8FE190E08C0F9D1F9F938F9381E5E2
:1031900098E19F938F930E94D36660E280E70E943C
:1031A000A0430F900F900F900F9080915B0799278D
:1031B0009F938F9384E598E19F938F930E94D366AA
:1031C00060E38DE00E94A0430F900F900F900F904E
:1031D000AEE2B0E0AC0FBD1FBF93AF9387E598E1BF
:1031E0009F938F930E94D36660E380E70E94A04381
:1031F0000F900F900F900F9080915C0799279F93ED
:103200008F938AE598E19F938F930E94D36600E1A4
:10321000232D44E0692D832D0E94880E0F900F907E
:103220000F900F90FF2009F03FC280E80E944D5B95
:10323000882309F042C380E40E944D5B082F882355
:1032400069F121E02093D90B80914B0790914C07B5
:10325000A0914D07B0914E078093C7079093C80780
:10326000A093C907B093CA07EE2051F4B2E09B16B1
:1032700009F0B0C0922EB3E0EB2E0E949815AEC0BC
:1032800081E0981611F4EA94A9C0EE2009F4A2C0D6
:1032900092E0991609F09EC0EA9457C180E20E941C
:1032A0004D5B182F882391F181E08093D90B809199
:1032B0004B0790914C07A0914D07B0914E0780931A
:1032C000C7079093C807A093C907B093CA07A3E0A4
:1032D000EA1649F4B1E09B1631F4A2E09A2E0E945E
:1032E0009815E02E32C181E0981631F492E09E15D7
:1032F00008F474C0E80E72C0A2E09A1609F06AC021
:10330000B1E0BE1508F421C1EB0E1FC180E10E949F
:103310004D5B882309F45EC081E08093D90B8091D6
:103320004B0790914C07A0914D07B0914E078093A9
:10333000C7079093C807A093C907B093CA0782E054
:10334000981619F4F0E18F2E01C0812EEE2029F499
:1033500091E09916F1F4F92C41C0A1E0EA1629F4A4
:103360009A1601F5E2E0FE2E39C0B2E0EB1631F418
:1033700081E0981601F573E0F72E30C093E0E9166E
:1033800031F4A1E09A1601F564E0F62E27C0EE2094
:1033900031F4B2E09B16F1F455E0F52ED6C081E091
:1033A000E81631F492E09916A9F446E0F42ECDC067
:1033B000A2E0EA1631F4B2E09B1661F438E0F32E95
:1033C000C4C083E0E81631F492E0991619F427E0BE
:1033D000F22EBBC0A1E09A1609F0B3C060E08DE008
:1033E0000E94A04381E090E08C0F9D1F9F938F93DC
:1033F0008DE598E19F938F930E94D36660E086E607
:103400000E94A0430F900F900F900F908091530750
:1034100090915407A0915507B0915607BF93AF9371
:103420009F938F9380E698E19F938F930E94D3663A
:1034300060E18DE00E94A043ADB7BEB716960FB60F
:10344000F894BEBF0FBEADBF80E190E08C0F9D1F12
:103450009F938F9386E698E19F938F930E94D36604
:1034600060E186E60E94A0430F900F900F900F90AE
:103470008091570790915807A0915907B0915A072A
:10348000BF93AF939F938F9389E698E19F938F9318
:103490000E94D36660E28DE00E94A043ADB7BEB744
:1034A00016960FB6F894BEBF0FBEADBF8FE190E089
:1034B0008C0F9D1F9F938F938FE698E19F938F931F
:1034C0000E94D36660E280E70E94A0430F900F90B5
:1034D0000F900F9080915B0799279F938F9382E7BE
:1034E00098E19F938F930E94D36660E38DE00E94E2
:1034F000A0430F900F900F900F90AEE2B0E0AC0F92
:10350000BD1FBF93AF9385E798E19F938F930E9470
:10351000D36660E380E70E94A0430F900F900F9066
:103520000F9080915C0799279F938F9388E798E18C
:103530009F938F930E94D3660F900F900F900F90E0
:10354000ABC0B2E09B1609F0A7C060E08DE00E941E
:10355000A043CE01CD969F938F938BE798E19F93E5
:103560008F930E94D36660E080E70E94A0430F9093
:103570000F900F900F9080915D0799279F938F93E5
:103580008EE798E19F938F930E94D36660E18DE070
:103590000E94A0430F900F900F900F90CE01845B7C
:1035A0009F4F9F938F9381E898E19F938F930E9401
:1035B000D36660E184E60E94A04380915E070F908D
:1035C0000F900F900F90813041F484E898E19F9321
:1035D0008F930E94D3660F900F9080915E0788238F
:1035E00041F488E898E19F938F930E94D3660F90EF
:1035F0000F9060E28DE00E94A043CE0186599F4F5C
:103600009F938F938CE898E19F938F930E94D3664A
:10361000809161070F900F900F900F90813061F4AF
:1036200060E283E60E94A0438FE898E19F938F9326
:103630000E94D3660F900F9080916107823061F4F1
:1036400060E285E60E94A04383E998E19F938F930F
:103650000E94D3660F900F9080916107833061F4D0
:1036600060E28AE40E94A04386E998E19F938F93E9
:103670000E94D3660F900F9080916107843061F4AF
:1036800060E283E60E94A0438DE998E19F938F93C7
:103690000E94D3660F900F9000E120E044E061E0CB
:1036A0008E2D0E94880EBECD81E0F81609F01BC158
:1036B00080E10E944D5B8823A1F0FF2481E080938C
:1036C000D90B80914B0790914C07A0914D07B09179
:1036D0004E078093C7079093C807A093C907B0937C
:1036E000CA0780E80E944D5B80E20E944D5B882300
:1036F00009F44BC081E08093D90B80914B079091E6
:103700004C07A0914D07B0914E078093C707909347
:10371000C807A093C907B093CA0780915307909137
:103720005407A0915507B09156072DEC3CEC4CEC9A
:103730005DE3BC01CD010E946168DC01CB01809397
:10374000530790935407A0935507B0935607809161
:10375000530790915407A0915507B091560720E068
:1037600030E040E050E0BC01CD010E941369181622
:1037700064F480E090E0A0E0B0E080935307909381
:103780005407A0935507B093560780E40E944D5B01
:10379000882309F44BC081E08093D90B80914B07BB
:1037A00090914C07A0914D07B0914E078093C707A9
:1037B0009093C807A093C907B093CA078091530795
:1037C00090915407A0915507B09156072DEC3CEC11
:1037D0004CEC5DE3BC01CD010E946068DC01CB01D3
:1037E0008093530790935407A0935507B0935607BF
:1037F0008091530790915407A0915507B0915607B7
:1038000020E030E040EA50ECBC01CD010E9410699C
:10381000882364F480E090E0A0E0B0E08093530758
:1038200090935407A0935507B09356078091530780
:1038300090915407A0915507B0915607ED962CAD85
:103840003DAD4EAD5FADED97BC01CD010E9410695D
:103850008823A9F000E02AE049E1602F86E60E9473
:1038600027478091530790915407A0915507B09135
:103870005607ED968CAF9DAFAEAFBFAFED97809181
:103880004B0790914C07A0914D07B0914E07BC019A
:10389000CD0128E532E040E050E00E94666CDC019A
:1038A000CB01883C9105A105B10550F4FF2041F002
:1038B00000E02AE049E1602F26C191E0392EF4CEE4
:1038C00060E086E60E94A0438091530790915407E0
:1038D000A0915507B0915607BF93AF939F938F93D5
:1038E00081EA98E126C1B2E0FB1609F02FC180E120
:1038F0000E944D5B8823A1F0FF2481E08093D90BC7
:1039000080914B0790914C07A0914D07B0914E07C5
:103910008093C7079093C807A093C907B093CA07BD
:1039200080E80E944D5B80E20E944D5B882309F491
:103930004BC081E08093D90B80914B0790914C074D
:10394000A0914D07B0914E078093C7079093C80789
:10395000A093C907B093CA07809157079091580761
:10396000A0915907B0915A072DEC3CEC4CEC5DE36B
:10397000BC01CD010E946168DC01CB018093570737
:1039800090935807A0935907B0935A07809157070F
:1039900090915807A0915907B0915A0720E030E064
:1039A00040EA50E4BC01CD010E941369181664F48A
:1039B00080E090E0A0E0B0E0809357079093580734
:1039C000A0935907B0935A0780E40E944D5B882367
:1039D00009F44BC081E08093D90B80914B07909103
:1039E0004C07A0914D07B0914E078093C707909365
:1039F000C807A093C907B093CA0780915707909151
:103A00005807A0915907B0915A072DEC3CEC4CECAB
:103A10005DE3BC01CD010E946068DC01CB018093B5
:103A2000570790935807A0935907B0935A0780916E
:103A3000570790915807A0915907B0915A0720E075
:103A400030E040E050E0BC01CD010E9410698823C5
:103A500064F480E090E0A0E0B0E08093570790939A
:103A60005807A0935907B0935A0780915707909130
:103A70005807A0915907B0915A07C358DF4F2881C2
:103A800039814A815B81CD57D040BC01CD010E9474
:103A900010698823C9F080E1881900E02AE049E133
:103AA000682F86E60E942747809157079091580714
:103AB000A0915907B0915A07C358DF4F8883998363
:103AC000AA83BB83CD57D04080914B0790914C0780
:103AD000A0914D07B0914E07BC01CD0128E532E021
:103AE00040E050E00E94666CDC01CB01883C91050F
:103AF000A105B10550F4FF2041F080E1881900E0F4
:103B00002AE049E1682F86E611C580E18819682F0F
:103B100086E60E94A0438091570790915807A09194
:103B20005907B0915A07BF93AF939F938F9387EA3A
:103B300098E19F938F930E94D366ADB7BEB7169658
:103B40000FB6F894BEBF0FBEADBF33C5B3E0FB16D2
:103B500009F0D3C080E10E944D5B8823A1F0FF24CF
:103B600081E08093D90B80914B0790914C07A091F5
:103B70004D07B0914E078093C7079093C807A09355
:103B8000C907B093CA0780E80E944D5B80E20E949B
:103B90004D5B8823F1F081E08093D90B80914B0736
:103BA00090914C07A0914D07B0914E078093C707A5
:103BB0009093C807A093C907B093CA0780915B0789
:103BC0008F5F80935B0780915B07893110F01092C3
:103BD0005B0780E40E944D5B8823E1F081E08093E5
:103BE000D90B80914B0790914C07A0914D07B09154
:103BF0004E078093C7079093C807A093C907B09357
:103C0000CA0780915B07882329F080915B07815068
:103C100080935B0780915B079927AA2797FDA09562
:103C2000BA2FBC01CD010E940669DC01CB01CF5740
:103C3000DF4F288139814A815B81C158D040BC0166
:103C4000CD010E941069882379F180E2881900E093
:103C50002AE049E1682F86E60E94274710915B071A
:103C6000812F992787FD9095A92FB92FBC01CD01F0
:103C70000E940669CF57DF4F688379838A839B83CD
:103C8000C158D04017FF10C020E030E040E853E4B6
:103C90000E946168DC01CB01CF57DF4F8883998395
:103CA000AA83BB83C158D04080914B0790914C07A9
:103CB000A0914D07B0914E07BC01CD0128E532E03F
:103CC00040E050E00E94666CDC01CB01883C91052D
:103CD000A105B10520F4FF2011F080E20FCF80E2B2
:103CE0008819682F80E70E94A04380915B0799277D
:103CF0009F938F938DEA98E1C6C084E0F81609F08F
:103D0000CBC080E10E944D5B8823A1F0FF2481E0BD
:103D10008093D90B80914B0790914C07A0914D0750
:103D2000B0914E078093C7079093C807A093C90727
:103D3000B093CA0780E80E944D5B80E20E944D5B11
:103D40008823F1F081E08093D90B80914B0790910B
:103D50004C07A0914D07B0914E078093C7079093F1
:103D6000C807A093C907B093CA0780915C078F5F0B
:103D700080935C0780915C078D3310F010925C0794
:103D800080E40E944D5B8823F1F021E02093D90B61
:103D900080914B0790914C07A0914D07B0914E0731
:103DA0008093C7079093C807A093C907B093CA0729
:103DB00080915C07815080935C0780915C07882329
:103DC00011F420935C0780915C079927AA2797FD3F
:103DD000A095BA2FBC01CD010E940669DC01CB0180
:103DE000A3019201BC01CD010E941069882319F141
:103DF00080E3881900E02AE043E1682F8CE60E9406
:103E0000274710915C07812F992787FD9095A92F4F
:103E1000B92FBC01CD010E9406692B013C0117FF9F
:103E20000AC020E030E040E853E40E946168DC0111
:103E3000CB012C013D0180914B0790914C07A09143
:103E40004D07B0914E07BC01CD0128E532E040E0BE
:103E500050E00E94666CDC01CB01883C9105A10515
:103E6000B10520F4FF2011F080E348CE80E38819EB
:103E7000682F80E70E94A04380915C0799279F9359
:103E80008F9380EB98E19F938F930E94D3660F905E
:103E90000F900F900F908DC395E0F91609F0F2C0C6
:103EA00080E10E944D5B8823A1F0FF2481E0809394
:103EB000D90B80914B0790914C07A0914D07B09181
:103EC0004E078093C7079093C807A093C907B09384
:103ED000CA0780E80E944D5B80915D078F5F8093E9
:103EE0005D0780E20E944D5B882359F180915D0758
:103EF0008F5F80935D0780915D07853018F081E0CA
:103F000080935D0780915D07815080935D070E94DB
:103F10005F1580915D078F5F80935D0781E08093DF
:103F2000D90B80914B0790914C07A0914D07B09110
:103F30004E078093C7079093C807A093C907B09313
:103F4000CA0780E40E944D5B882359F180915D0788
:103F5000815080935D0780915D07882319F484E088
:103F600080935D0780915D07815080935D070E947B
:103F70005F1580915D078F5F80935D0781E080937F
:103F8000D90B80914B0790914C07A0914D07B091B0
:103F90004E078093C7079093C807A093C907B093B3
:103FA000CA0780915D079927AA2797FDA095BA2F88
:103FB000BC01CD010E940669DC01CB01A60195017F
:103FC000BC01CD010E941069882309F100E02AE0BC
:103FD00043E1602F8CE60E94274710915D07812FF7
:103FE000992787FD9095A92FB92FBC01CD010E947B
:103FF00006695B016C0117FF0AC020E030E040E871
:1040000053E40E946168DC01CB015C016D01809189
:104010004B0790914C07A0914D07B0914E07BC0102
:10402000CD0128E532E040E050E00E94666CDC0102
:10403000CB01883C9105A105B10550F4FF2041F06A
:1040400000E02AE049E1602F86E60E94274714C07D
:1040500060E080E70E94A04380915D079927019767
:104060009F938F9383EB98E19F938F930E94D366E6
:104070000F900F900F900F9080915D07815080936B
:104080005D0797C2A6E0FA1609F0AAC080E10E9477
:104090004D5B8823A1F0FF2481E08093D90B8091B0
:1040A0004B0790914C07A0914D07B0914E0780931C
:1040B000C7079093C807A093C907B093CA0780E8C1
:1040C0000E944D5B80E20E944D5B882319F081E0E5
:1040D00080935E0780E40E944D5B882311F010926C
:1040E0005E0780915E079927AA2797FDA095BA2FB2
:1040F000BC01CD010E940669DC01CB01CB57DF4F2B
:10410000288139814A815B81C558D040BC01CD01ED
:104110000E941069882369F100E02AE043E160E130
:104120008CE60E94274710915E07812F992787FD13
:104130009095A92FB92FBC01CD010E940669CB57DC
:10414000DF4F688379838A839B83C558D04017FFEC
:1041500010C020E030E040E853E40E946168DC01D8
:10416000CB01CB57DF4F88839983AA83BB83C55884
:10417000D04080914B0790914C07A0914D07B09192
:104180004E07BC01CD0128E532E040E050E00E943E
:10419000666CDC01CB01883C9105A105B10540F4BA
:1041A000FF2031F000E02AE04BE160E184E6BEC18F
:1041B00060E184E60E94A04380915E07813041F473
:1041C00086EB98E19F938F930E94D3660F900F9098
:1041D00080915E07882309F0ECC18AEB98E1E3C186
:1041E000B7E0FB1609F0D4C080E10E944D5B882344
:1041F000A1F0FF2481E08093D90B80914B0790912F
:104200004C07A0914D07B0914E078093C70790933C
:10421000C807A093C907B093CA0780E80E944D5B06
:1042200080E20E944D5B882361F080915F078330BC
:1042300030F480915F078F5F80935F0702C0109218
:104240005F0780E40E944D5B882359F080915F07EF
:10425000882321F080915F07815001C083E0809323
:104260005F0780915F079927AA2797FDA095BA2F2E
:10427000BC01CD010E940669DC01CB01C757DF4FAD
:10428000288139814A815B81C958D040BC01CD0168
:104290000E941069882369F100E02EE048E460E2A2
:1042A00087E30E94274710915F07812F992787FD99
:1042B0009095A92FB92FBC01CD010E940669C7575F
:1042C000DF4F688379838A839B83C958D04017FF67
:1042D00010C020E030E040E853E40E946168DC0157
:1042E000CB01C757DF4F88839983AA83BB83C95803
:1042F000D04080914B0790914C07A0914D07B09111
:104300004E07BC01CD0128E532E040E050E00E94BC
:10431000666CDC01CB01883C9105A105B10540F438
:10432000FF2031F000E02EE048E460E287E3FEC0C9
:1043300060E287E30E94A04380915F07882341F4F5
:104340008EEB98E19F938F930E94D3660F900F900E
:1043500080915F07813041F482EC98E19F938F93C5
:104360000E94D3660F900F9080915F07823041F4D6
:1043700087EC98E19F938F930E94D3660F900F90E4
:1043800080915F07833009F014C18CEC98E10BC178
:1043900088E0F81609F00DC180E10E944D5B88238A
:1043A000A1F0FF2481E08093D90B80914B0790917D
:1043B0004C07A0914D07B0914E078093C70790938B
:1043C000C807A093C907B093CA0780E80E944D5B55
:1043D00080E20E944D5B8823F9F0809161078F5F36
:1043E0008093610780916107853018F081E08093A8
:1043F000610781E08093D90B80914B0790914C0726
:10440000A0914D07B0914E078093C7079093C807BE
:10441000A093C907B093CA0780E40E944D5B88232C
:10442000F9F0809161078150809361078091610765
:10443000882319F484E08093610781E08093D90B8D
:1044400080914B0790914C07A0914D07B0914E077A
:104450008093C7079093C807A093C907B093CA0772
:10446000809161079927AA2797FDA095BA2FBC01D3
:10447000CD010E940669DC01CB01C357DF4F2881C3
:1044800039814A815B81CD58D040BC01CD010E9469
:104490001069882369F100E02AE049E360E286E4DC
:1044A0000E94274710916107812F992787FD9095DA
:1044B000A92FB92FBC01CD010E940669C357DF4F58
:1044C000688379838A839B83CD58D04017FF10C0BF
:1044D00020E030E040E853E40E946168DC01CB0159
:1044E000C357DF4F88839983AA83BB83CD58D040BD
:1044F00080914B0790914C07A0914D07B0914E07CA
:10450000BC01CD0128E532E040E050E00E94666C3D
:10451000DC01CB01883C9105A105B10550F4FF20D9
:1045200041F000E02AE049E360E286E40E94274788
:1045300040C080916107813061F460E283E60E94AF
:10454000A04386ED98E19F938F930E94D3660F90CE
:104550000F9080916107823061F460E285E60E94ED
:10456000A0438AED98E19F938F930E94D3660F90AA
:104570000F9080916107833061F460E28AE40E94C9
:10458000A0438DED98E19F938F930E94D3660F9087
:104590000F9080916107843061F460E283E60E94AD
:1045A000A04384EE98E19F938F930E94D3660F906F
:1045B0000F9091E0391611F00C9412190E94B80E68
:1045C0000E94C50E80915E07882321F480915F07C9
:1045D0008823B1F080915E07882319F030926C0730
:1045E00002C080936C07222071F49698899A88EC17
:1045F0000E94D30E919888EC0E94D30E919A03C02A
:1046000080936C07969A0E945F1510929A07C05784
:10461000DF4F0FB6F894DEBF0FBECDBFDF91CF9155
:104620001F910F91FF90EF90DF90CF90BF90AF90D0
:104630009F908F907F906F905F904F903F902F90C2
:1046400008954F925F926F927F928F929F92AF9256
:10465000BF92CF92DF92EF92FF920F931F93CF936F
:10466000DF93CDB7DEB72C970FB6F894DEBF0FBE41
:10467000CDBF2B013C0129833A834B835C83ED82C0
:10468000FE820F831887A986BA86CB86DC8620E156
:1046900037E240E050E00E94666CDA01C90197FF02
:1046A00003C0309521953F4F4901AA2497FCA0945F
:1046B000BA2CC301B20124E630E040E050E00E9491
:1046C000666C6B017C01C301B20120E137E240E07E
:1046D00050E00E94666CDC01CB018C199D09AE098B
:1046E000BF09BC01CD0124E630E040E050E00E946B
:1046F000666C89019A01C6018053984FAC01B801DC
:10470000C4010E94AC0D7B018C014CEB57E061E0D1
:1047100070E086E090E00E94AC0DDC01CB01E81A6D
:10472000F90A0A0B1B0BC801B70120E831E541E08B
:1047300050E00E94146C7B018C0169817A818B812D
:104740009C8120E13EE040E050E00E94146CDC01DE
:10475000CB01E80EF91E0A1F1B1F6D817E818F8120
:1047600098852CE330E040E050E00E94146CDC01BE
:10477000CB01E80EF91E0A1F1B1F89859A85AB85A0
:10478000BC85E80EF91E0A1F1B1F80E891E5A1E019
:10479000B0E0E80EF91E0A1F1B1FC801B7012C96D6
:1047A0000FB6F894DEBF0FBECDBFDF91CF911F9142
:1047B0000F91FF90EF90DF90CF90BF90AF909F90C0
:1047C0008F907F906F905F904F9008952F923F92BF
:1047D0004F925F926F927F928F929F92AF92BF9211
:1047E000CF92DF92EF92FF920F931F93E090DA0B3C
:1047F000F090DB0B0091DC0B1091DD0B20E030E042
:1048000040E050E0C801B7010E941069882309F414
:10481000A1C08091A80C9091A90CA091AA0CB09174
:10482000AB0C9C01AD01C801B7010E946068DC01BE
:10483000CB0120E030E04EED52E4BC01CD010E94FE
:10484000C0691B012C01E090C307F090C4070091E0
:10485000C5071091C6078091AC0C9091AD0CA0914A
:10486000AE0CB091AF0C9C01AD01C801B7010E9424
:104870006068DC01CB0120E030E04EE852E4BC018E
:10488000CD010E94C0693B014C0120918E073091FF
:104890008F07409190075091910757FD05C0CA01BD
:1048A000B9010E94066916C0DA01C90181709070D1
:1048B000A070B0705695479537952795822B932B0E
:1048C000A42BB52BBC01CD010E9406699B01AC0154
:1048D0000E9461685B016C01A2019101C201B101FA
:1048E0000E94C0697B018C01A4019301C401B30142
:1048F0000E94C069DC01CB019C01AD01C801B70178
:104900000E946168DC01CB01BC01CD010E94516AAB
:10491000DC01CB0120E030E04AE754E4BC01CD01EA
:104920000E94C069DC01CB019C01AD01C601B5014B
:104930000E946168DC01CB01BC01CD010E94E968E5
:10494000DC01CB0180938E0790938F07A093900793
:10495000B09391078091CF069091D006A091D10697
:10496000B091D2062091BE073091BF074091C00799
:104970005091C10760906D0770906E0780906F072F
:10498000909070072090EB0B3090EC0B4090ED0B6B
:104990005090EE0B5C016D0179018A01A401930135
:1049A000C201B1010E9421237B018C018091A80CDE
:1049B0009091A90CA091AA0CB091AB0C21E63BE020
:1049C00046E35BE4BC01CD010E94C069DC01CB0180
:1049D000BC01CD010E94E968DC01CB018093750721
:1049E00090937607A0937707B09378078091AC0CEB
:1049F0009091AD0CA091AE0CB091AF0C21E63BE0D4
:104A000046E35BE4BC01CD010E94C069DC01CB013F
:104A1000BC01CD010E94E968DC01CB0180937107E4
:104A200090937207A0937307B09374078091B907AE
:104A30009091BA07A091BB07B091BC0720E030E08D
:104A400040E251E4BC01CD010E94C069DC01CB0110
:104A5000BC01CD010E94E968DC01CB01809379079C
:104A600090937A07A0937B07B0937C07E0927D0731
:104A7000F0927E0700937F071093800780919B0739
:104A800090919C07A0919D07B0919E0704E0880F2C
:104A9000991FAA1FBB1F0A95D1F700E110E020E083
:104AA00030E0AC01BD0181E797E00E94E6578091BC
:104AB0009B0790919C07A0919D07B0919E0701963E
:104AC000A11DB11DBC01CD0120E038E041E050E066
:104AD0000E94666CDC01CB0180939B0790939C073E
:104AE000A0939D07B0939E078091A80C9091A90C6C
:104AF000A091AA0CB091AB0C8093DA0B9093DB0BD6
:104B0000A093DC0BB093DD0B8091AC0C9091AD0CBD
:104B1000A091AE0CB091AF0C8093C3079093C407E3
:104B2000A093C507B093C6071F910F91FF90EF9018
:104B3000DF90CF90BF90AF909F908F907F906F90BD
:104B40005F904F903F902F90089562E080E00E9428
:104B5000135362E580E00E94135366E280E00E94F6
:104B6000135360E0862F0E94135360E0862F0E944B
:104B7000135368E780E00E94135363E080E00E94D3
:104B800013538AEF0E94D30E62E080E00E94135319
:104B900062E580E00E94135363E280E00E941353B9
:104BA00061E080E00E94135360E0862F0E9413535F
:104BB00066E780E00E94135365E080E00E94135393
:104BC00063E080E00E9413538AEF0E94D30E62E0FC
:104BD00080E00E94135362E580E00E94135366E276
:104BE00080E00E94135360E0862F0E94135360E020
:104BF000862F0E94135368E780E00E94135363E0FE
:104C000080E00E94135388EC0E94D30E40E056E9E6
:104C100060E070E080E00E947652089562E080E0FB
:104C20000E94135362E580E00E94135366E280E025
:104C30000E94135360E0862F0E94135360E0862F7A
:104C40000E94135368E780E00E94135363E080E002
:104C50000E9413538AEF0E94D30E62E080E00E940C
:104C6000135362E580E00E94135364E080E00E94E9
:104C7000135364E180E00E94135360E0862F0E948A
:104C800013536AE680E00E94135363E180E00E94C0
:104C9000135363E580E00E9413536BE480E00E94AD
:104CA000135369E580E00E94135364E580E00E949D
:104CB000135362E580E00E94135361E480E00E9498
:104CC000135368E580E00E94135368E580E00E947A
:104CD000135360E280E00E94135360E280E00E9480
:104CE000135360E280E00E94135360E280E00E9470
:104CF000135360E280E00E94135360E280E00E9460
:104D0000135360E280E00E94135360E280E00E944F
:104D1000135360E280E00E94135360E280E00E943F
:104D2000135360E0862F0E94135363E080E00E94DB
:104D300013538AEF0E94D30E62E080E00E94135367
:104D400062E580E00E94135366E280E00E94135304
:104D500060E0862F0E94135360E0862F0E94135359
:104D600068E780E00E94135363E080E00E941353E1
:104D700008958F929F92AF92BF92CF92DF92EF925F
:104D8000FF920F931F93CF93DF93CDB7DEB7E697D4
:104D90000FB6F894DEBF0FBECDBF81E0A82EB12CB8
:104DA000882499248091B1079091B207A091B3070C
:104DB000B091B4078F5F9F4FAF4FBF4F09F40BC245
:104DC0008AE090E09F938F930DE0E02EF12CFF920C
:104DD000EF9225E530E03F932F9382E090E09F93A0
:104DE0008F9344E550E05F934F933F932F9382E47A
:104DF00090E09F938F9385E490E09F938F9384E45A
:104E000090E09F938F93BF92AF925F934F93BF9227
:104E1000AF928BE890E09F938F9386EE91E09F9303
:104E20008F938E010A0D1B1D1F930F930E94F8662E
:104E3000A701B80180E00E94D753C090A907D09085
:104E4000AA07E090AB07F090AC078DB79EB74E96DF
:104E50000FB6F8949EBF0FBE8DBF8091AD079091A5
:104E6000AE07A091AF07B091B007C816D906EA0601
:104E7000FB0609F463C1D701C60114E0880F991F2E
:104E8000AA1FBB1F1A95D1F700E110E020E030E027
:104E9000AC01BD0181E797E00E945B596BE880E0BF
:104EA0000E9413530894A11CB11C8A2D99279C01C0
:104EB00020703170821B930B682F80E00E94135387
:104EC0008501107064E580E00E94135361E080E08A
:104ED0000E94135360E0862F0E94135361E080E02C
:104EE0000E9413530F511F4FC40101966FEF7FEFC4
:104EF0000E943F6C4C01292F3327020F111D080D12
:104F0000111D622F80E00E941353682D80E00E94E3
:104F1000135340917D0750917E0760917F077091F8
:104F200080074BAB5CAB6DAB7EAB9BA98CA9890FAB
:104F3000912D911D2DA9820F911D2EA9820F911DDA
:104F4000080F191F872F9927AA27BB27682F80E0F2
:104F50000E9413538BA99CA9ADA9BEA9CD01AA2774
:104F6000BB27682F80E00E9413538BA99CA9ADA991
:104F7000BEA9892F9A2FAB2FBB27682F80E00E94F4
:104F800013536BA980E00E94135340917507509111
:104F9000760760917707709178074BAB5CAB6DAB90
:104FA0007EAB9BA98CA9890F912D911D2DA9820FF4
:104FB000911D2EA9820F911D080F191F872F992768
:104FC000AA27BB27682F80E00E9413538BA99CA9B6
:104FD000ADA9BEA9CD01AA27BB27682F80E00E94FA
:104FE00013538BA99CA9ADA9BEA9892F9A2FAB2FCA
:104FF000BB27682F80E00E9413536BA980E00E94BA
:10500000135340917107509172076091730770912B
:1050100074074BAB5CAB6DAB7EAB9BA98CA9890FC6
:10502000912D911D2DA9820F911D2EA9820F911DE9
:10503000080F191F872F9927AA27BB27682F80E001
:105040000E9413538BA99CA9ADA9BEA9CD01AA2783
:10505000BB27682F80E00E9413538BA99CA9ADA9A0
:10506000BEA9892F9A2FAB2FBB27682F80E00E9403
:1050700013536BA980E00E9413534091790750911C
:105080007A0760917B0770917C074BAB5CAB6DAB93
:105090007EAB9BA98CA9890F912D911D2DA9820F03
:1050A000911D080F191FCB01AA27BB27682F80E08D
:1050B0000E9413538BA99CA9ADA9BEA9892F9A2F31
:1050C000AB2FBB27682F80E00E9413536BA980E0B1
:1050D0000E94135360E0862F0E941353C801AA2731
:1050E000BB279C01AD012070307041705070821B55
:1050F000930BA40BB50B8C01892F9927682F80E0A7
:105100000E941353602F80E00E9413536DE080E0F3
:105110000E9413536AE080E00E9413530894C11C5C
:10512000D11CE11CF11CC701B60120E038E041E0D0
:1051300050E00E94886C6B017C018FCE6BE880E0B0
:105140000E9413530894A11CB11C8A2D99279C011D
:1051500020703170821B930B682F80E00E941353E4
:105160009FEFA922BB2464E580E00E94135361E015
:1051700080E00E94135366E480E00E94135369E4C8
:1051800080E00E9413536EE480E00E9413538DEB85
:1051900091E0A80EB91EC501AA27BB279C01AD014D
:1051A0002070307041705070821B930BA40BB50BB4
:1051B0008C01892F9927682F80E00E941353602F5C
:1051C00080E00E9413536DE080E00E9413536AE078
:1051D00080E00E941353E6960FB6F894DEBF0FBE30
:1051E000CDBFDF91CF911F910F91FF90EF90DF9096
:1051F000CF90BF90AF909F908F900895CF92DF9205
:10520000EF92FF920F931F93CF93DF93EC0110E087
:105210008C819D81892B09F491C060E070E0CE0102
:105220000E94564A843241F0CE010E940F4A8C817E
:105230009D81892B91F74CC021E0E22EF12C8C81CD
:105240009D810197E816F90608F078C0B701CE01F4
:105250000E94564A8D30C1F5C7010196BC01CE01AE
:105260000E94564A8A3081F5CE010E940F4A00E022
:1052700010E067010894C108D1080C151D05C0F4A1
:1052800093EFE92E96E0F92E0F34110530F4CE019C
:105290000E940F4AF701808303C0CE010E940F4A8B
:1052A0000F5F1F4F0894E11CF11C0C151D0560F3E6
:1052B0000D50194FF8011082CE010E940F4ACE0105
:1052C0000E940F4A1AE006C00894E11CF11CB7CFF7
:1052D0001123A1F142E150E061E072E083EF96E03A
:1052E0000E94FB65892B39F488EE98E10E94C84F33
:1052F0000E94DF4F2DC044E150E064E172E083EF93
:1053000096E00E94FB65892B51F044E150E069E290
:1053100072E083EF96E00E94FB65892BC9F48AEF67
:105320000E94D30E8AEF0E94D30E8AEF0E94D30E02
:105330008AEF0E94D30E0E94B9260AC02C813D81BB
:105340008A819B812817390718F0CE010E94994A5B
:10535000812F9927DF91CF911F910F91FF90EF90AF
:10536000DF90CF9008953F924F925F926F927F921D
:105370008F929F92AF92BF92CF92DF92EF92FF9265
:105380000F931F93CF934B015C01CC24DD24760156
:10539000C0E03C2E2B013C01F4E0440C551C661C83
:1053A000771CFA95D1F7D301C2014097A109B10941
:1053B00000E110E020E030E0AC01BD0181E797E0C2
:1053C0000E945B5980917D0790917E07A0917F0795
:1053D000B09180078F5F9F4FAF4FBF4F19F4C70148
:1053E000B60177C100E110E020E030E0B301A20196
:1053F00081E797E00E945B598092AD079092AE07DB
:10540000A092AF07B092B00780917D0790917E0780
:10541000A0917F07B09180078093B1079093B20766
:10542000A093B307B093B40780917D0790917E0756
:10543000A0917F07B0918007BC01CD0120E831E544
:1054400041E050E00E94666C29013A017501640157
:105450000894C108D108E108F108C114D104E1049D
:10546000F10461F481E0381639F4C12CE8E0DE2E55
:10547000E1E0EE2EF12C02C071E0372ECC2309F0D2
:1054800044C098EEC91693E0D90690E0E90690E092
:10549000F906C8F188E19CEFAFEFBFEFC80ED91E47
:1054A000EA1EFB1ED701C60164E0880F991FAA1FE0
:1054B000BB1F6A95D1F700E110E020E030E0AC01BD
:1054C000BD0181E797E00E945B5980917D07909133
:1054D0007E07A0917F07B0918007BC01CD0120E835
:1054E00031E541E050E00E94666C24153505460523
:1054F000570509F4C5C088EE93E0A0E0B0E0C80EFF
:10550000D91EEA1EFB1EC1E003C0C13009F041C034
:1055100094E6C916D104E104F104C8F18CE99FEFC7
:10552000AFEFBFEFC80ED91EEA1EFB1ED701C601A2
:1055300054E0880F991FAA1FBB1F5A95D1F700E1AD
:1055400010E020E030E0AC01BD0181E797E00E946F
:105550005B5980917D0790917E07A0917F07B09164
:105560008007BC01CD0120E831E541E050E00E9418
:10557000666C241535054605570509F481C084E697
:1055800090E0A0E0B0E0C80ED91EEA1EFB1EC2E00B
:1055900003C0C23009F040C09AE0C916D104E1044A
:1055A000F104C0F186EF9FEFAFEFBFEFC80ED91E39
:1055B000EA1EFB1ED701C60144E0880F991FAA1FEF
:1055C000BB1F4A95D1F700E110E020E030E0AC01CC
:1055D000BD0181E797E00E945B5980917D07909122
:1055E0007E07A0917F07B0918007BC01CD0120E824
:1055F00031E541E050E00E94666C24153505460512
:105600005705F1F18AE090E0A0E0B0E0C80ED91EA5
:10561000EA1EFB1EC3E002C0C33091F50894C10826
:10562000D108E108F108D701C60134E0880F991FBD
:10563000AA1FBB1F3A95D1F700E110E020E030E04F
:10564000AC01BD0181E797E00E945B5980917D0725
:1056500090917E07A0917F07B0918007BC01CD019A
:1056600020E831E541E050E00E94666C99EEC916F1
:1056700093E0D90690E0E90690E0F90608F0C0E072
:10568000241535054605570509F4E7CEA0E0CA16EE
:10569000A8E0DA06A1E0EA06A0E0FA0671F00894B4
:1056A000C11CD11CE11CF11CC092A907D092AA0711
:1056B000E092AB07F092AC0708C01092A9071092D5
:1056C000AA071092AB071092AC0761E070E080E08F
:1056D00090E0CF911F910F91FF90EF90DF90CF90CE
:1056E000BF90AF909F908F907F906F905F904F9002
:1056F0003F9008952F923F924F925F926F927F92C8
:105700008F929F92AF92BF92CF92DF92EF92FF92D1
:105710000F931F93CF933B014C01AA24BB24650137
:10572000C0E0DC01CB0154E0880F991FAA1FBB1F0A
:105730005A95D1F700E110E020E030E0AC01BD0166
:1057400081E797E00E945B5980917D0790917E07E9
:10575000A0917F07B09180078F5F9F4FAF4FBF4FE2
:1057600019F4C601B50185C181E0681688E07806A4
:1057700081E0880680E0980611F435014601D401E5
:10578000C30144E0880F991FAA1FBB1F4A95D1F798
:1057900000E110E020E030E0AC01BD0181E797E0DE
:1057A0000E945B596092A9077092AA078092AB078A
:1057B0009092AC0780917D0790917E07A0917F0722
:1057C000B09180078093B1079093B207A093B3077D
:1057D000B093B40780917D0790917E07A0917F07D9
:1057E000B0918007BC01CD0120E831E541E050E0F7
:1057F0000E94666C19012A0179018A016401530132
:10580000C601B5012FEF37E041E050E00E94666C21
:105810005B016C01CC2309F046C098E1A91694E025
:10582000B90691E0C90690E0D906D8F588EE93E074
:10583000A0E0B0E0A80EB91ECA1EDB1ED601C5014D
:1058400034E0880F991FAA1FBB1F3A95D1F700E1DA
:1058500010E020E030E0AC01BD0181E797E00E945C
:105860005B5980917D0790917E07A0917F07B09151
:105870008007BC01CD0120E831E541E050E00E9405
:10588000666C79018A01221533054405550509F432
:10589000C7C088E19CEFAFEFBFEFA80EB91ECA1ECC
:1058A000DB1EC1E003C0C13009F046C09CE9A91667
:1058B00097E0B90691E0C90690E0D906D8F584E6EC
:1058C00090E0A0E0B0E0A80EB91ECA1EDB1ED60113
:1058D000C50124E0880F991FAA1FBB1F2A95D1F785
:1058E00000E110E020E030E0AC01BD0181E797E08D
:1058F0000E945B5980917D0790917E07A0917F0760
:10590000B0918007BC01CD0120E831E541E050E0D5
:105910000E94666C79018A012215330544055505FC
:1059200009F47EC08CE99FEFAFEFBFEFA80EB91E60
:10593000CA1EDB1EC2E003C0C23009F045C096EFAC
:10594000A91697E0B90691E0C90690E0D906D0F50E
:105950008AE090E0A0E0B0E0A80EB91ECA1EDB1EEF
:10596000D601C50104E0880F991FAA1FBB1F0A9525
:10597000D1F700E110E020E030E0AC01BD0181E7AB
:1059800097E00E945B5980917D0790917E07A091DE
:105990007F07B0918007BC01CD0120E831E541E0EF
:1059A00050E00E94666C79018A0122153305440596
:1059B0005505B1F186EF9FEFAFEFBFEFA80EB91E0F
:1059C000CA1EDB1EC3E002C0C33051F50894A11CFF
:1059D000B11CC11CD11CD601C50114E0880F991F50
:1059E000AA1FBB1F1A95D1F700E110E020E030E0BC
:1059F000AC01BD0181E797E00E945B5980917D0772
:105A000090917E07A0917F07B0918007BC01CD01E6
:105A100020E831E541E050E00E94666C79018A019E
:105A2000E214F3040405150509F4EACEA114B10447
:105A3000C104D10471F00894A108B108C108D108CB
:105A4000A092AD07B092AE07C092AF07D092B00758
:105A50000CC080E098E0A1E0B0E08093AD079093A7
:105A6000AE07A093AF07B093B00761E070E080E0AD
:105A700090E0CF911F910F91FF90EF90DF90CF902A
:105A8000BF90AF909F908F907F906F905F904F905E
:105A90003F902F9008956F927F928F929F92AF9236
:105AA000BF92CF92DF92EF92FF920F931F93CF930B
:105AB000DF93CDB7DEB7CA54D0400FB6F894DEBF3F
:105AC0000FBECDBF11E0E3E36E2E712C6C0E7D1E78
:105AD00088E1EEE3F2E0D30101900D928A95E1F7BF
:105AE0000E9440138CE30E94D30E4FEF6CEA72E4E5
:105AF0008FEF96E00E94B042109221011FBC80E11E
:105B00000E944D5B882309F4B3C182E30E94D30E47
:105B1000AFC1112309F427C10E9440136AE084E059
:105B20000E94A0438AE299E19F938F930E94D366DB
:105B300069E180E30E94A0430F900F908FE399E109
:105B40009F938F930E94D366802F0E9401530E94DF
:105B5000FE2847EE56E06091B1077091B207809140
:105B6000B3079091B4070E94B75A6DE281E10E9499
:105B7000A0438091B1079091B207A091B307B09173
:105B8000B4070F900F908F5F9F4FAF4FBF4F49F1FA
:105B90008091EC069091ED069F938F938091EB0698
:105BA00099279F938F938091EA0699279F938F93CC
:105BB0009091EE0683E0989FC0011124860D971DF9
:105BC0009F938F9383E499E19F938F930E94D36671
:105BD0008DB79EB70A960FB6F8949EBF0FBE8DBFC5
:105BE00008C088E599E19F938F930E94D3660F9038
:105BF0000F908091A9079091AA07A091AB07B0914F
:105C0000AC07BF93AF939F938F9386E592E09F93EA
:105C10008F934E010894811C911C9F928F920E9439
:105C2000F866C4010E94814F8091AD079091AE0744
:105C3000A091AF07B091B007BF93AF939F938F939D
:105C400089E692E09F938F939F928F920E94F866CD
:105C5000C4010E94814F8091A9079091AA07A09149
:105C6000AB07B091AC0774E0880F991FAA1FBB1F48
:105C70007A95D1F700E110E020E030E0AC01BD0101
:105C800081E797E00E945B59A0907D07B0907E0766
:105C9000C0907F07D09080078091AD079091AE07AC
:105CA000A091AF07B091B00764E0880F991FAA1FB9
:105CB000BB1F6A95D1F700E110E020E030E0AC01B5
:105CC000BD0181E797E00E945B59E0907D07F0906D
:105CD0007E0700917F0710918007EA18FB080C09E6
:105CE0001D09C801B70120E13EE040E050E00E94FC
:105CF000666CD22E822F9927AA27BB27BC01CD0123
:105D000020E13EE040E050E00E94146CDC01CB0159
:105D1000E81AF90A0A0B1B0BC801B7012CE330E0A3
:105D200040E050E00E94666CDA01C90199279F9318
:105D30008F938D2D99279F938F938CE792E09F935C
:105D40008F939F928F920E94F866C4010E94814FA8
:105D500010E00E944913ADB7BEB758960FB6F8943D
:105D6000BEBF0FBEADBF8091B1079091B207A091A9
:105D7000B307B091B4078F5F9F4FAF4FBF4F09F488
:105D800072C080E40E944D5B882361F181E08093C2
:105D9000D90B80914B0790914C07A0914D07B09182
:105DA0004E078093C7079093C807A093C907B09385
:105DB000CA076091A9077091AA078091AB079091DB
:105DC000AC07611571058105910529F0615070409E
:105DD0008040904004C060E078E081E090E00E9464
:105DE000B32911E080E20E944D5B882311F111E09C
:105DF0001093D90B80914B0790914C07A0914D07C0
:105E0000B0914E078093C7079093C807A093C90726
:105E1000B093CA078091AD079091AE07A091AF07EC
:105E2000B091B0070196A11DB11DBC01CD010E942A
:105E30007A2B80E10E944D5B8823A9F081E080935A
:105E4000D90B80914B0790914C07A0914D07B091D1
:105E50004E078093C7079093C807A093C907B093D4
:105E6000CA070E94B92680E00E9401530E94FE28C2
:105E700080E80E944D5B082F882309F44ACE0E94D7
:105E80004013C65BDF4F0FB6F894DEBF0FBECDBF29
:105E9000DF91CF911F910F91FF90EF90DF90CF9006
:105EA000BF90AF909F908F907F906F9008950E94C9
:105EB000C50E0E94EE0E8F3F51F580E090E0A0E00D
:105EC000B0EC8093530790935407A0935507B09379
:105ED00056078AE999E9A9E1BFE3809357079093B0
:105EE0005807A0935907B0935A0791E090935B0726
:105EF00085E080935C0790935D0790935E07109216
:105F00005F0710926007909361070E94B80E80911E
:105F10005E07882321F480915F07882389F08091B0
:105F20005E07811181E080936C079698899A88ECCE
:105F30000E94D30E919888EC0E94D30E919A01C0D2
:105F4000969A0E945F150895CF92DF92EF92FF928A
:105F50000F931F93CF93DF930E94C65680E00E9459
:105F6000E5568C01C801AA2797FDA095BA2FBC0160
:105F7000CD010E94066917FF06C020E030E040E82E
:105F800057E40E9461682DEC3CEC4CE45EE30E9417
:105F9000C0696B017C0100919C0210919D02C801B7
:105FA000AA2797FDA095BA2FBC01CD010E940669D2
:105FB00017FF06C020E030E040E857E40E94616827
:105FC0002DEC3CEC4CE45FE30E94C069DC01CB01AA
:105FD0009C01AD01C701B6010E946168DC01CB01E3
:105FE000BC01CD010E94E9687B018C01EB010E949C
:105FF000D456F0929D02E0929C028091E504863096
:1060000018F48F5F8093E5048E0100571340C80198
:10601000AA2797FDA095BA2FBC01CD010E94066961
:1060200017FF06C020E030E040E857E40E946168B6
:1060300020E030E040E250E40E94A368DC01CB01A4
:1060400020E030E040E850E4BC01CD010E946168EE
:10605000DC01CB01BC01CD010E94E968DC01CB0170
:10606000982F82E0CC3BD80710F490E010C083E07A
:10607000C634D80710F491E00AC083E0CC35D807C5
:1060800010F492E004C0C057D34008F493E080912C
:10609000E504863008F494E6849B08C080919B0256
:1060A000891710F4982F02C090939B029093CE060C
:1060B000DF91CF911F910F91FF90EF90DF90CF90E4
:1060C00008950F931F93CF93DF93CDB7DEB7E29779
:1060D0000FB6F894DEBF0FBECDBF8D9A959A129A77
:1060E0001A9886E90E94D30E1A9A40E855E260E0B9
:1060F00070E080E00E94765240E855E260E070E097
:1061000081E00E9476528E010F5F1F4F84E1EEE91D
:10611000F2E0D80101900D928A95E1F7C8010E9442
:10612000814F8AEF0E94D30E8FE1E2EBF2E0D801BB
:1061300001900D928A95E1F7C8010E94814F8AEF84
:106140000E94D30E87E2E1EDF2E0D80101900D92BA
:106150008A95E1F7C8010E94814FE2960FB6F89444
:10616000DEBF0FBECDBFDF91CF911F910F9108957C
:106170004F925F926F927F928F929F92AF92BF9257
:10618000CF92DF92EF92FF920F931F93CF93DF9303
:10619000CDB7DEB728970FB6F894DEBF0FBECDBFE0
:1061A0002FEF37E041E050E02D833E834F83588747
:1061B00019821A821B821C828FEF9FEFAFEFBFEF15
:1061C0008093B1079093B207A093B307B093B4073D
:1061D00000E110E020E030E040E050E060E070E0FE
:1061E00081E797E00E945B5980917D0790917E073F
:1061F000A0917F07B09180078F5F9F4FAF4FBF4F38
:1062000009F49FC0C0907D07D0907E07E0907F0783
:10621000F090800700E110E020E030E040EF5FE721
:1062200060E170E081E797E00E945B5980917D0713
:1062300090917E07A0917F07B0918007C816D9067C
:10624000EA06FB0630F48F5F9F4FAF4FBF4F09F058
:1062500078C089809A80AB80BC808D819E81AF811F
:10626000B885880E991EAA1EBB1EB694A794979453
:106270008794D501C40114E0880F991FAA1FBB1F82
:106280001A95D1F700E110E020E030E0AC01BD014B
:1062900081E797E00E945B5940907D0750907E0710
:1062A00060907F077090800789819A81AB81BC8163
:1062B000F4E0880F991FAA1FBB1FFA95D1F700E1E0
:1062C00010E020E030E0AC01BD0181E797E00E94E2
:1062D0005B59C0907D07D0907E07E0907F07F090DB
:1062E00080074C145D046E047F0470F09FEF491624
:1062F0009FEF59069FEF69069FEF790629F0898283
:106300009A82AB82BC8204C08D829E82AF82B886A4
:1063100089819A81AB81BC810196A11DB11D2D811E
:106320003E814F815885281739074A075B0709F0D6
:1063300090CF20939B0730939C0740939D075093E9
:106340009E0749815A816B817C81CB01BA012896D5
:106350000FB6F894DEBF0FBECDBFDF91CF911F9176
:106360000F91FF90EF90DF90CF90BF90AF909F90F4
:106370008F907F906F905F904F9008958091660707
:106380008F5F80936607833010F01092660781E07C
:106390008093D90B80914B0790914C07A0914D07AA
:1063A000B0914E078093C7079093C807A093C90781
:1063B000B093CA07089580E090E0A0EFB1E4809325
:1063C000A1079093A207A093A307B093A40780E02E
:1063D0000E942A0E0E94491305C00E94625685E061
:1063E0000E94D30E8091A1079091A207A091A307CC
:1063F000B091A40720E030E040E050E0BC01CD01C6
:106400000E941069882349F708950E9440139598C7
:1064100012988A988B988998969A10981198C79A8A
:10642000B998BA98BB98BE9888980E94D45614BA66
:10643000D098D198D298D398D498BD98D598D6981A
:10644000D7981B9808950F931F93CF9300E0C02F08
:10645000102F0E94C50F849BAAC00F9998C0CB3003
:1064600008F4CF5F84E60E94D30ECB3018F40F9B64
:10647000F6CF8DC001E00E9440134FEF6CEA72E44A
:106480008FEF96E00E94B0426AE084E10E94A04350
:1064900080E799E19F938F930E94D3666EE188E233
:1064A0000E94A0430F900F908DE799E19F938F93E7
:1064B0000E94D3660E9449130F900F9080E20E94C1
:1064C0004D5B8823A1F000E011E01093D90B80917F
:1064D0004B0790914C07A0914D07B0914E078093C8
:1064E000C7079093C807A093C907B093CA0780E86D
:1064F0000E944D5B8823A1F000E011E01093D90BBE
:1065000080914B0790914C07A0914D07B0914E0799
:106510008093C7079093C807A093C907B093CA0791
:1065200080E10E944D5B8823A1F002E011E010930E
:10653000D90B80914B0790914C07A0914D07B091DA
:106540004E078093C7079093C807A093C907B093DD
:10655000CA0780E40E944D5B8823A9F000E011E0A7
:106560001093D90B80914B0790914C07A0914D0748
:10657000B0914E078093C7079093C807A093C907AF
:10658000B093CA0707C0112309F498CF03C081E074
:106590008093CB070E9440130E9498150E944913D4
:1065A000023041F40F9B06C00E94053203C081E017
:1065B0008093CB07CF911F910F9108951F93CF9395
:1065C000DF9310E0849B67C00E94401381E08093BA
:1065D000D90B80914B0790914C07A0914D07B0913A
:1065E0004E078093C7079093C807A093C907B0933D
:1065F000CA074FEF6CEA72E48FEF96E00E94B04258
:106600006AE084E10E94A04386E899E19F938F931A
:106610000E94D3666EE188E20E94A0430F900F9023
:1066200083E999E19F938F930E94D3660E94491357
:106630000F900F900F9BFECFC0E0D0E082E30E944E
:10664000D30E80E10E944D5B882379F42196C436F5
:10665000D105A4F30E9440130E9498150E9449138B
:106660001123E1F40E94053219C011E00E94401389
:106670001093D90B80914B0790914C07A0914D0737
:10668000B0914E078093C7079093C807A093C9079E
:10669000B093CA07DFCF81E080933004DF91CF91C0
:1066A0001F910895CF9380912F04882329F580911D
:1066B000F40C9091F50CA091F60CB091F70C20E041
:1066C00030E040E051E4BC01CD010E94136918168E
:1066D0009CF48091E60B9091E70BA091E80BB091B0
:1066E000E90B8093430790934407A0934507B09329
:1066F000460781E080932F04C091BD07C630F8F4AF
:106700008091F40C9091F50CA091F60CB091F70CDF
:1067100020E030E040E051E4BC01CD010E9413696B
:1067200018166CF480912F04813049F48091F60B97
:106730009091F70B039719F4CF5FC093BD07809139
:10674000BD078530F0F08091E60B9091E70BA091AA
:10675000E80BB091E90B2091430730914407409139
:10676000450750914607821B930BA40BB50B079767
:10677000A105B10530F481E080932E040E947913C5
:106780001CC08091E60B9091E70BA091E80BB091B3
:10679000E90B209143073091440740914507509100
:1067A0004607821B930BA40BB50B0697A105B105F9
:1067B00020F01092BD0710922F04CF910895CF9230
:1067C000DF92EF92FF920F931F93CF93DF93C82E28
:1067D000D62E89014FEF6CEA72E48CEC96E00E94B1
:1067E000B0421016110614F4780104C0EE24FF2400
:1067F000E01AF10A6D2D8C2D0E94A0438CE999E1DD
:106800009F938F930E94D366C0E0D0E00F900F90CB
:10681000CE15DF05C4F4101611061CF48D2D8C1B4B
:1068200002C08D2D8C0F682F8C2D0E94A0438EE905
:1068300099E19F938F930E94D3660F900F902196BA
:10684000CE15DF0544F3DF91CF911F910F91FF909B
:10685000EF90DF90CF9008954F925F926F927F926A
:106860008F929F92AF92BF92CF92DF92EF92FF9260
:106870000F931F93CF93DF93CDB7DEB764970FB617
:10688000F894DEBF0FBECDBF9B01AC012E01089472
:10689000411C511C84E1D2011D928A95E9F7809137
:1068A0008805882381F480938705E6EEF4E0219340
:1068B0003193419351938F5F8832C8F3809387055A
:1068C00081E08093880580908605E82DFF27EE0FF4
:1068D000FF1FEE0FFF1FEA51FB4F208331834283DE
:1068E0005383109287059924520138EF632E32E0CA
:1068F000732E882D99278C01000F111F000F111F77
:106900000A511B4FF30121913F01C22EDD248C1946
:106910009D09889668E270E00E94536CFC01EE0FBE
:10692000FF1FEE0FFF1FEA51FB4FD801ED90FD90C6
:106930000D911C9180819181A281B3819C01AD0157
:10694000C801B7010E9460687B018C01C601AA27BB
:1069500097FDA095BA2FBC01CD010E940669DC010C
:10696000CB019C01AD01C801B7010E94A368DC0105
:10697000CB01F50181939193A193B1935F0193941E
:10698000F4E0F91508F0B5CF10928705EE240E2D2E
:106990001127000F111F000F111F040D151DF80105
:1069A00080819181A281B38120E030E040E251E416
:1069B000BC01CD010E94C069DC01CB01F8018083DC
:1069C0009183A283B38320E030E040E251E4BC0134
:1069D000CD010E94136918164CF480E090E0A0E20B
:1069E000B1E4F80180839183A283B383F8018081AD
:1069F0009181A281B38120E030E040E151ECBC0103
:106A0000CD010E94106988234CF480E090E0A0E161
:106A1000B1ECF80180839183A283B3838E2D8F5FC5
:106A2000E82E853008F4B3CF8093870589819A8159
:106A3000AB81BC81BC01CD010E94E968DC01CB01C6
:106A40009C014AE060E284E30E94DF338D819E81F5
:106A5000AF81B885BC01CD010E94E968DC01CB01A2
:106A60009C014AE060E289E20E94DF3389859A85D1
:106A7000AB85BC85BC01CD010E94E968DC01CB017E
:106A80009C014AE060E28EE10E94DF338D859E85A5
:106A9000AF85B889BC01CD010E94E968DC01CB015A
:106AA0009C014AE060E283E10E94DF3389899A8990
:106AB000AB89BC89BC01CD010E94E968DC01CB0136
:106AC0009C014AE060E288E00E94DF338091860505
:106AD0008F5F68E20E94336C9093860564960FB6D0
:106AE000F894DEBF0FBECDBFDF91CF911F910F9104
:106AF000FF90EF90DF90CF90BF90AF909F908F90DE
:106B00007F906F905F904F9008950F931F93CF9356
:106B1000DF93CDB7DEB7A4970FB6F894DEBF0FBEF4
:106B2000CDBF8E010F5F1F4F84E2EDEFF2E0D80181
:106B300001900D928A95E1F74FEF6CEA72E48CE0D8
:106B400095E00E94B0428091F00C9091F10CA091E0
:106B5000F20CB091F30C20E030E044EB51E4BC01C6
:106B6000CD010E946168DC01CB01BC01CD010E9416
:106B7000E968DC01CB019C0197FF03C030952195AA
:106B80003F4FC9016DE270E00E94536CDB0177FD5D
:106B90001796A87F6A1B7B0BDB01AA0FBB1FAA0FEE
:106BA000BB1FA00FB11FFD0101900020E9F7319735
:106BB000EA1BFB0B329718F461E086E602C061E045
:106BC0008AE50E94A0438091F00C9091F10CA09175
:106BD000F20CB091F30C20E030E044EB51E4BC0146
:106BE000CD010E946168DC01CB01BC01CD010E9496
:106BF000E968DC01CB019C0197FF03C0309521952A
:106C00003F4FC9016DE270E00E94536CCB0177FDEC
:106C10000796887F681B790B660F771F660F771FB3
:106C2000060F171F1F930F9380EA99E19F938F938D
:106C30000E94D3660F900F900F900F90A4960FB6FE
:106C4000F894DEBF0FBECDBFDF91CF911F910F91A2
:106C5000089562E080E00E94135362E580E00E94A4
:106C6000135366E280E00E94135360E0862F0E9477
:106C7000135360E0862F0E94135368E780E00E9460
:106C8000135363E080E00E9413538AEF0E94D30EF7
:106C90008AEF0E94D30E8AEF0E94D30E8AEF0E94E1
:106CA000D30E8AEF0E94D30E8AEF0E94D30E62E0C9
:106CB00080E00E94135362E580E00E94135367E175
:106CC00080E00E94135365E080E00E94135360E06F
:106CD000862F0E9413536EE680E00E94135364E0F7
:106CE00080E00E9413536FEF80E00E9413536FEF18
:106CF00080E00E9413536FEF80E00E9413536FEF08
:106D000080E00E94135363E080E00E9413538AEFF7
:106D10000E94D30E8AEF0E94D30E8AEF0E94D30EF8
:106D20008AEF0E94D30E8AEF0E94D30E8AEF0E9450
:106D3000D30E62E080E00E94135362E580E00E947F
:106D4000135366E280E00E94135360E0862F0E9496
:106D5000135360E0862F0E94135368E780E00E947F
:106D6000135363E080E00E941353089562E080E0D3
:106D70000E94135362E580E00E94135366E280E0B4
:106D80000E94135360E0862F0E94135360E0862F09
:106D90000E94135368E780E00E94135363E080E091
:106DA0000E9413538AEF0E94D30E62E080E00E949B
:106DB000135362E580E00E9413536AE180E00E9471
:106DC000135360E0862F0E94135360E0862F0E94C9
:106DD00013536CE680E00E94135363E080E00E944E
:106DE00013538AEF0E94D30E62E080E00E94135397
:106DF00062E580E00E94135366E280E00E94135334
:106E000060E0862F0E94135360E0862F0E94135388
:106E100068E780E00E94135363E080E00E94135310
:106E200008950E94D00F80912C0490912D048F7EA4
:106E300090932D0480932C0408950E94A42F809198
:106E40002C0490912D048B7F90932D0480932C041F
:106E500080914B0790914C07A0914D07B0914E0740
:106E60008093D7069093D806A093D906B093DA06FC
:106E700008950E94481780912C0490912D048F7BD7
:106E800090932D0480932C0480914B0790914C0794
:106E9000A0914D07B0914E0780938A0790938B077E
:106EA000A0938C07B0938D0708950E94FA0E8091ED
:106EB0002C0490912D048F7790932D0480932C04B3
:106EC00080914B0790914C07A0914D07B0914E07D0
:106ED0008093470790934807A0934907B0934A07C8
:106EE000089581E00E9401530E947D4E80912C0400
:106EF00090912D048F7D90932D0480932C04089500
:106F0000CF93DF93CDB7DEB7E2970FB6F894DEBF2D
:106F10000FBECDBF8BE293E50E94764FAE014F5F6F
:106F20005F4F84E121E233E0DA01F90101900D9233
:106F30008A95E1F7CA010E94814F86E293E50E949B
:106F4000764FE2960FB6F894DEBF0FBECDBFDF914D
:106F5000CF9108958F929F92AF92BF92CF92DF927E
:106F6000EF92FF920F931F93CF93DF93CDB7DEB7CE
:106F7000E4970FB6F894DEBF0FBECDBF4E01089464
:106F8000811C911C84E3E5E3F3E0D40101900D92B0
:106F90008A95E1F780918B05893018F48F5F809393
:106FA0008B0580918B058830A1F48091A80C90917D
:106FB000A90CA091AA0CB091AB0C20E030E040E00D
:106FC00050E0BC01CD010E941069882311F40E9499
:106FD00080370E94401390916607992309F068C09A
:106FE00080916107843009F063C0849B04C081E014
:106FF0008093210104C0909321010E94C50F4FEF9F
:107000006CEA72E486ED90E10E94B0428091B9078B
:107010009091BA07A091BB07B091BC0720E03CE378
:107020004CE156E4BC01CD010E941369181664F4CA
:1070300080E09CE3ACE1B6E48093B9079093BA0793
:10704000A093BB07B093BC078091B9079091BA0792
:10705000A091BB07B091BC0720E030E04AE754E4C0
:10706000BC01CD010E94106988231CF46AE082E112
:1070700002C06AE081E00E94A0438091B90790912C
:10708000BA07A091BB07B091BC07BF93AF939F9382
:107090008F9383EA99E19F938F930E94D3662DB7D4
:1070A0003EB72A5F3F4F0FB6F8943EBF0FBE2DBFCD
:1070B00090916607992309F033C480916107843069
:1070C00009F42EC4849B04C081E08093210104C094
:1070D000909321010E94C50F4FEF6CEA72E487EA9A
:1070E00090E10E94B04260E0862F0E94A04389EAAE
:1070F00099E19F938F930E94D3668091F60B9091B4
:10710000F70B0F900F90039799F44FEF6CEA72E42E
:1071100085E590E10E94B04260E086E00E94A043D5
:107120008BEA99E19F938F930E94D3660F900F9003
:107130004FEF6CEA72E48EE49EE00E94B04266E09B
:1071400088E00E94A0438DEA99E19F938F930E946B
:10715000D36666E088E10E94A0430F900F908FEA0B
:1071600099E19F938F930E94D36666E088E20E9424
:10717000A0430F900F9081EB99E19F938F930E9412
:10718000D36666E088E30E94A0430F900F9083EBE4
:1071900099E19F938F930E94D36666E088E40E94F2
:1071A000A0430F900F9085EB99E19F938F930E94DE
:1071B000D36666E088E50E94A0430F900F9087EBAE
:1071C00099E19F938F930E94D36666E080E60E94C8
:1071D000A0430F900F9089EB99E19F938F930E94AA
:1071E000D36666E080E70E94A0430F900F908BEB80
:1071F00099E19F938F930E94D3666DE188E00E948E
:10720000A0430F900F908DEB99E19F938F930E9475
:10721000D3666DE188E10E94A0430F900F908FEB41
:1072200099E19F938F930E94D3666DE188E20E945B
:10723000A0430F900F9081EC99E19F938F930E9450
:10724000D3666DE188E30E94A0430F900F9083EC1A
:1072500099E19F938F930E94D3666DE188E40E9429
:10726000A0430F900F9085EC99E19F938F930E941C
:10727000D3666DE188E50E94A0430F900F9087ECE4
:1072800099E19F938F930E94D3666DE180E60E94FF
:10729000A0430F900F9089EC99E19F938F930E94E8
:1072A000D3666DE180E70E94A0430F900F908BECB6
:1072B00099E19F938F930E94D3664FEF6CEA72E43B
:1072C00082E59CE00E94B0428091B9079091BA0794
:1072D000A091BB07B091BC070F900F9020E03CE35A
:1072E0004CE156E4BC01CD010E941369181664F408
:1072F00080E09CE3ACE1B6E48093B9079093BA07D1
:10730000A093BB07B093BC0760E08EE00E94A0434F
:107310008091B9079091BA07A091BB07B091BC07C3
:10732000BF93AF939F938F938DEC99E19F938F932E
:107330000E94D3668091D3069091D406A091D50681
:10734000B091D606BC01CD010E942C348091F60B81
:107350009091F70BADB7BEB716960FB6F894BEBFB7
:107360000FBEADBF039799F44FEF6CEA72E485E569
:1073700090E10E94B04269E182E40E94A04383ED63
:1073800099E19F938F930E94D3660F900F90809105
:10739000F60B9091F70B029799F44FEF6CEA72E4B9
:1073A00085E590E10E94B04269E182E40E94A04339
:1073B00085ED99E19F938F930E94D3660F900F9074
:1073C00080912E048823C9F08091F60B9091F70BE1
:1073D00002979CF04FEF6CEA72E485E590E10E9421
:1073E000B04262E282E40E94A04387ED99E19F935C
:1073F0008F930E94D3660F900F904FEF6CEA72E468
:1074000082E59CE00E94B0428091F40C9091F50CD2
:10741000A091F60CB091F70C20E030E046E953E47F
:10742000BC01CD010E941369181664F480E090E05D
:10743000A6E9B3E48093F40C9093F50CA093F60CBA
:10744000B093F70C6FE28EE00E94A0438091F60BA0
:107450009091F70B0397E4F08091F40C9091F50C68
:10746000A091F60CB091F70CBF93AF939F938F93BD
:1074700089ED99E19F938F930E94D3662DB73EB714
:107480002A5F3F4F0FB6F8943EBF0FBE2DBF0CC012
:107490006DE283E10E94A0438FED99E19F938F936A
:1074A0000E94D3660F900F908091E60B9091E70BAE
:1074B000A091E80BB091E90B0097A105B10509F483
:1074C00056C04FEF6CEA72E482E59CE00E94B04245
:1074D0006FE282E40E94A04390916D0780915B0768
:1074E000890F68E10E94336C892F99279F938F93AE
:1074F00085EE99E19F938F930E94D3666FE285E6B4
:107500000E94A0430F900F900F900F908091BE07A4
:1075100099279F938F938AEE99E19F938F930E946F
:10752000D366809189050F900F900F900F90813056
:10753000D9F46DE28FE50E94A0438FEE99E19F930D
:107540008F930E94D36665E28FE50E94A0430F905F
:107550000F9081EF99E19F938F930E94D3661092D1
:1075600089050F900F9003C081E0809389054FEF4C
:107570006CEA72E482E59CE00E94B0428091A1072F
:107580009091A207A091A307B091A4072DEC3CEC29
:107590004CEC5EE3BC01CD010E94C0697B018C0113
:1075A00080918C0590918D05A0918E05B0918F05ED
:1075B0002AE939E949E15FE3BC01CD010E94C069D4
:1075C000DC01CB019C01AD01C801B7010E946168DB
:1075D0007B018C01609390057093910580939205D7
:1075E0009093930560938C0570938D0580938E0521
:1075F00090938F052DEC3CEC4CE45DE30E94106908
:107600008823B4F42DEC3CEC4CE45DEBC801B701ED
:107610000E941369181664F480E090E0A0E0B0E0E6
:107620008093900590939105A0939205B093930554
:10763000E0909005F09091050091920510919305CE
:1076400026E636E64EE151ECC801B7010E9410690A
:1076500088239CF467E18AE50E94A043809190050D
:1076600090919105A0919205B0919305BF93AF932E
:107670009F938F9383EF99E16FC020E030E040E06B
:1076800050E0C801B7010E9410698823FCF467E14B
:107690008AE50E94A0438091900590919105A09168
:1076A0009205B0919305BF93AF939F938F9389EF0A
:1076B00099E19F938F930E94D366ADB7BEB716969C
:1076C0000FB6F894BEBF0FBEADBF52C026E636E679
:1076D0004EE151E4C801B7010E941369181604F580
:1076E00067E181E60E94A043809190059091910509
:1076F000A0919205B0919305BF93AF939F938F9301
:107700008FEF99E19F938F930E94D3662DB73EB779
:107710002A5F3F4F0FB6F8943EBF0FBE2DBF28C063
:1077200020E030E040E050E0C801B7010E9413695A
:107730008823F4F067E181E60E94A04380919005E0
:1077400090919105A0919205B0919305BF93AF934D
:107750009F938F9385E09AE19F938F930E94D366C6
:107760008DB79EB706960FB6F8949EBF0FBE8DBF1D
:107770004FEF6CEA72E482E59CE00E94B042809197
:10778000F60B9091F70B03975CF18091F40C9091BC
:10779000F50CA091F60CB091F70C20E030E040E041
:1077A00050E0BC01CD010E9413691816CCF4809101
:1077B000D50B9091D60BA091D70BB091D80B20E0B0
:1077C00030E040E050E0BC01CD010E941069882308
:1077D00039F480916107823019F00E948535A0C08C
:1077E000E090D50BF090D60B0091D70B1091D80BF1
:1077F00020E030E040E050E0C801B7010E9413698A
:1078000018160CF081C080916107813009F47CC0AA
:1078100021EE3AEF47EC52E4C801B7010E94136928
:107820001816FCF460E087E50E94A0438091D50B18
:107830009091D60BA091D70BB091D80BBF93AF937B
:107840009F938F938BE09AE19F938F930E94D366CF
:10785000ADB7BEB716960FB6F894BEBF0FBEADBF9C
:107860005FC02AE037ED4FE151E4C801B7010E9443
:107870001369181654F520E030E048EC52E4C801D2
:10788000B7010E941069882304F560E085E60E9434
:10789000A0438091D50B9091D60BA091D70BB091BE
:1078A000D80BBF93AF939F938F9381E19AE19F93FE
:1078B0008F930E94D3662DB73EB72A5F3F4F0FB616
:1078C000F8943EBF0FBE2DBF2BC060E081E60E9442
:1078D000A0438091D50B9091D60BA091D70BB0917E
:1078E000D80BBF93AF939F938F9387E19AE19F93B8
:1078F0008F930E94D3668DB79EB706960FB6F89405
:107900009EBF0FBE8DBF0CC060E087E60E94A04303
:107910008DE19AE19F938F930E94D3660F900F9011
:1079200080916607813009F0D2C1E090A80CF090F8
:10793000A90C0091AA0C1091AB0CC801B7010E94D0
:10794000E9685B016C01CB01AA2797FDA095BA2FCE
:10795000BC01CD010E940669B7FE06C020E030E000
:1079600040E857E40E9461689B01AC01C801B7017F
:107970000E946068DC01CB0120E030E040E752E487
:10798000BC01CD010E94C0697B018C014FEF6CEA04
:1079900072E48FEF96E00E94B04262E180E00E94C4
:1079A000A0431F930F93FF92EF92BF92AF9283E297
:1079B0009AE19F938F930E94D366E090AC0CF09075
:1079C000AD0C0091AE0C1091AF0CC801B7010E9434
:1079D000E9685B016C01CB01AA2797FDA095BA2F3E
:1079E000BC01CD010E940669ADB7BEB718960FB6AF
:1079F000F894BEBF0FBEADBFB7FE06C020E030E0BA
:107A000040E857E40E9461689B01AC01C801B701DE
:107A10000E946068DC01CB0120E030E040E752E4E6
:107A2000BC01CD010E94C0697B018C0161E280E054
:107A30000E94A0431F930F93FF92EF92BF92AF92C9
:107A40008EE29AE19F938F930E94D36662E380E077
:107A50000E94A0432DB73EB7285F3F4F0FB6F89462
:107A60003EBF0FBE2DBF8091EA0B99279F938F9346
:107A700089E39AE19F938F930E94D36661E280E548
:107A80000E94A04320918E0730918F07409190076C
:107A9000509191070F900F900F900F90293E83E027
:107AA000380780E0480780E05807C0F157FD05C05F
:107AB000CA01B9010E94066916C0DA01C9018170C4
:107AC0009070A070B0705695479537952795822B8A
:107AD000932BA42BB52BBC01CD010E9406699B0101
:107AE000AC010E94616820E030E04AE754E40E9463
:107AF000A368DC01CB01BF93AF939F938F9385E481
:107B00009AE19F938F930E94D366ADB7BEB7169646
:107B10000FB6F894BEBF0FBEADBF10C080918E07E8
:107B200090918F079F938F938FE49AE19F938F9308
:107B30000E94D3660F900F900F900F9062E387E33F
:107B40000E94A0438091CE06843649F485E59AE1EF
:107B50009F938F930E94D3660F900F900DC099272B
:107B60009F938F9380E69AE19F938F930E94D366B1
:107B70000F900F900F900F908091F60B9091F70B54
:107B800002972CF48091EA0B882309F4A0C0E090BE
:107B9000EB0BF090EC0B0091ED0B1091EE0BC8018C
:107BA000B70120E137E240E050E00E94666CC22E4F
:107BB000C801B70124E630E040E050E00E94666C66
:107BC000DC01CB01D82EC801B70120E137E240E04B
:107BD00050E00E94666CDC01CB018D199109A1096E
:107BE000B109BC01CD0124E630E040E050E00E9444
:107BF000666C122F60E0862F0E94A0438D2D99277E
:107C00008053984F9F938F93812F9927880F991FA7
:107C1000880F991F880E991E2CEF3FEF820E931E3E
:107C20009F928F928C2D99279F938F938CE69AE148
:107C30009F938F930E94D36660E08AE50E94A043E1
:107C40008DB79EB708960FB6F8949EBF0FBE8DBF36
:107C500090916D0780915B07890F68E10E94336CFA
:107C6000892F99279F938F9387E79AE19F938F930B
:107C70000E94D36660E08EE60E94A0430F900F90B2
:107C80000F900F908091BE0799279F938F938CE759
:107C90009AE19F938F930E94D366809189050F90FC
:107CA0000F900F900F90813079F460E089E60E9488
:107CB000A04381E89AE19F938F930E94D36610922C
:107CC00089050F900F9003C081E080938905809112
:107CD0006607823011F40E94AF13009166070023FB
:107CE00009F050C084994EC010918A05112389F47F
:107CF0004FEF6CEA72E48BE29CE00E94B042612F8D
:107D000083E70E94A04383E89AE10E94F64581E060
:107D100012C0113099F44FEF6CEA72E48BE29CE0F0
:107D20000E94B042602F83E70E94A04385E89AE159
:107D30000E94F64582E080938A0513C0123089F4D0
:107D40004FEF6CEA72E48BE29CE00E94B042602F3D
:107D500083E70E94A04387E89AE10E94F6450093DA
:107D60008A05879B0FC04FEF6CEA72E48BE29CE0C0
:107D70000E94B04260E083E70E94A04389E89AE154
:107D80000E94F6450E944913E4960FB6F894DEBFB0
:107D90000FBECDBFDF91CF911F910F91FF90EF905C
:107DA000DF90CF90BF90AF909F908F90089580917B
:107DB000EA0B8330A0F480E090E0A0E0B0E0809394
:107DC000F40C9093F50CA093F60CB093F70C809301
:107DD000F00C9093F10CA093F20CB093F30C809103
:107DE0002E04882311F40E94523380915C07209165
:107DF000C8063091C9064091CA065091CB06280F9B
:107E0000311D411D511D2150304040405040809156
:107E1000E60B9091E70BA091E80BB091E90B2817C6
:107E200039074A075B07E0F480912E048823C1F0EC
:107E30008091F60B9091F70B029794F00E94E62345
:107E40008091E60B9091E70BA091E80BB091E90BC4
:107E50008093C8069093C906A093CA06B093CB0638
:107E60000E94AA378091490C90914A0CA0914B0C2A
:107E7000B0914C0C88539F4FAF4FBF4F8093490C2C
:107E800090934A0CA0934B0CB0934C0C80912C0413
:107E900090912D049E7F90932D0480932C0408953F
:107EA000EF92FF920F931F93CF93FF24CF2DEF2CD0
:107EB0000E9423321091CB07113009F065C287B7B9
:107EC0008F7E87BF0E945F15F09221011093D90B1E
:107ED00080914B0790914C07A0914D07B0914E07B0
:107EE0008093C7079093C807A093C907B093CA07A8
:107EF000F0929A0782E30E94D30EF092C2074FEFEE
:107F00006CEA72E48FEF96E00E94B0420E94401348
:107F100068E088E20E94A0438BE89AE19F938F93E8
:107F20000E94D36668E188E20E94A0430F900F9000
:107F300082E99AE19F938F930E94D36668E2862F2D
:107F40000E94A0430F900F9089E99AE19F938F932D
:107F50000E94D36600E128E043E069E18C2F0E9493
:107F6000880E80E40E944D5B0F900F908823F1F003
:107F700081E08093D90B80914B0790914C07A091A1
:107F80004D07B0914E078093C7079093C807A09301
:107F9000C907B093CA07CC2311F0C15001C0C2E099
:107FA00000E128E043E069E18C2F25C080E20E94D7
:107FB0004D5B882319F181E08093D90B80914B07A9
:107FC00090914C07A0914D07B0914E078093C70741
:107FD0009093C807A093C907B093CA07CF5F8C2FAF
:107FE0009927039663E070E00E94536CC82F00E16C
:107FF00028E043E069E10E94880E2BC080E10E94E6
:108000004D5B882309F121E02093D90B80914B0728
:1080100090914C07A0914D07B0914E078093C707F0
:108020009093C807A093C907B093CA07CC2311F453
:10803000F22E0FC0C13019F422E0F22E0AC0C23075
:1080400041F493E0F92E05C080E80E944D5B88233F
:1080500081F40E944913FF2009F458CF8F2D9927EE
:108060008230910519F183309105D4F40197D9F04C
:108070007FC181E08093D90B80914B0790914C0791
:10808000A0914D07B0914E078093C7079093C80702
:10809000A093C907B093CA078CE30E94D30EDECF2A
:1080A000039739F065C10E944B2D60C10E94CA1729
:1080B0005DC110922101FF24CF2D0E94401360E189
:1080C00088E20E94A04381EA9AE19F938F930E94E5
:1080D000D36660E288E20E94A0430F900F908DEA81
:1080E0009AE19F938F930E94D36600E1202F42E094
:1080F00069E18C2F0E94880E80E40E944D5B0F90F6
:108100000F908823F9F081E08093D90B80914B0781
:1081100090914C07A0914D07B0914E078093C707EF
:108120009093C807A093C907B093CA07C1508C2F7A
:10813000992702969C018E7F9170281B390BC901EB
:10814000C22F24C080E20E944D5B882329F181E088
:108150008093D90B80914B0790914C07A0914D07CC
:10816000B0914E078093C7079093C807A093C907A3
:10817000B093CA07CF5F8C2F992702969C018E7F00
:108180009170281B390BC901C22F00E1202F42E05A
:1081900069E10E94880E14C080E10E944D5B882333
:1081A00051F0CC2319F481E0F82E0AC0C13041F41B
:1081B00002E0F02E05C080E80E944D5B882329F480
:1081C0000E944913FF2009F478CF8F2D9927813021
:1081D000910521F0029709F478C0C6C011E0109310
:1081E000D90B80914B0790914C07A0914D07B0910E
:1081F0004E078093C7079093C807A093C907B09311
:10820000CA0740E855E260E070E080E00E947652E4
:108210000E940E261093D90B80914B0790914C072A
:10822000A0914D07B0914E078093C7079093C80760
:10823000A093C907B093CA070E94A52540E056E95C
:1082400060E070E080E00E9476520E940E2610935B
:10825000D90B80914B0790914C07A0914D07B0919D
:108260004E078093C7079093C807A093C907B093A0
:10827000CA070E94A525109360070E94B80E40E02F
:1082800056E960E070E080E00E9476526DC081E0C7
:1082900080939A070E94981569E18FE00E94A0439D
:1082A00083EF9AE19F938F930E94D36688E190E0D9
:1082B00029E00FB6F894A89581BD0FBE21BD84E6D4
:1082C0000E94D30E0F900F904FC021E02093D90B46
:1082D00080914B0790914C07A0914D07B0914E07AC
:1082E0008093C7079093C807A093C907B093CA07A4
:1082F00020939A070E94981565E082E10E94A043AE
:1083000086EB9AE19F938F930E94D36668E186E0A3
:108310000E94A0430F900F9087EC9AE19F938F9358
:108320000E94D3666AE286E00E94A0430F900F90FD
:108330008EED9AE19F938F930E94D3660F900F90DA
:1083400080E80E944D5B8823D9F30F990DC08EE120
:108350008E1508F0E39484E60E94D30E8EE18E150C
:1083600008F495CF0F9BF3CF10929A070E94503FCD
:1083700087B78F7E87BF0E945F1581E080932101C0
:1083800010929A07109266071092CB070E94AA37A4
:10839000CF911F910F91FF90EF900895CFEFD0E113
:1083A000DEBFCDBF80E783B980EF87BB109261004D
:1083B0001092620088E082B91B9A8E9A9698BF9AB2
:1083C000C79ABE9AC6980E94650F0E945F151092C8
:1083D00021010E94981580E00E9484430E94491365
:1083E00040E050E0BA018EEF94E40E941C660E94C7
:1083F000F1520E9440550E9485570E9431560E94BA
:108400006C5501E024E048E651E060E0862F0E94D0
:108410007E550E94572F0E94C6560E94DE3280E889
:108420000E944D5B0E94DB318BE293E50E94764F08
:108430000E94613086E293E50E94764F0E94B83038
:10844000DC01CB01BC01CD010E94B3290E94A42F05
:10845000009160070023D9F440E855E260E070E045
:10846000802F0E9476520E940E260E94A52540E091
:1084700056E960E070E0802F0E9476520E940E263E
:108480000E94A52581E0809360070E94B80E40E01D
:1084900056E960E070E080E00E94765285B7837E06
:1084A00085BF85B7806285BF889585B78F7D85BF7D
:1084B00080912C0490912D0480FF02C00E9462568E
:1084C00080912C0490912D0484FF02C00E941137EA
:1084D00080912C0490912D0490FF02C00E94D73E01
:1084E00080912C0490912D0482FF02C00E941D37C0
:1084F00080912C0490912D0486FF02C00E94393790
:1085000080912C0490912D0487FF02C00E94553762
:1085100080912C0490912D0485FF02C00E94713738
:1085200080E20E944D5B882331F00E94C50F0E94BB
:10853000BE310E94AA3780E80E944D5B882311F06B
:108540000E94503F80913004813009F0A7CF849B76
:10855000A5CF0E940532A2CFFC01849199270895EE
:108560009093E50B8093E40B7093E30B6093E20B25
:108570004093DE0B08950F931F93CF93182F00E0C5
:108580008091E40B9091E50BE091E20BF091E30B0D
:1085900004960995C82F8091E40B9091E50BE0912A
:1085A000E20BF091E30B059609951C17B8F0212F0B
:1085B00033278C0F912D911D281739077CF41C1B34
:1085C0008091E40B9091E50B810F911DE091E20BFE
:1085D000F091E30B06960995082F0F5F802F9927DE
:1085E000CF911F910F9108950F931F93CF93DF9316
:1085F000EC0100E010E08881882331F089910E942D
:10860000BB42080F111DF7CFC801DF91CF911F9119
:108610000F9108950F931F93CF93DF93EC0100E028
:1086200010E0FE018491882341F0FE01219684919F
:108630000E94BB42080F111DF4CFC801DF91CF91FA
:108640001F910F910895962F969596959695292F9F
:1086500033273695322F222737952795280F311D3E
:10866000C9010895CF93DF93CDB7DEB721970FB639
:10867000F894DEBF0FBECDBFDB9A00000000000003
:10868000DB9819828981883030F489818F5F8983F2
:1086900089818830D0F321960FB6F894DEBF0FBEE3
:1086A000CDBFDF91CF910895CF93DF93CDB7DEB7E4
:1086B00021970FB6F894DEBF0FBECDBF982F66236B
:1086C00019F4D898DC9A04C0613011F4DC98D89A77
:1086D000DA98D9988FEF84BB95BBDB9A0000000035
:1086E0000000DB9819828981883020F489818F5FAE
:1086F0008983F9CF15BA21960FB6F894DEBF0FBE65
:10870000CDBFDF91CF9108951092DF0B1092E00B57
:108710001092E10B809394058FEF8ABB6091E00B80
:108720008FE30E94544361E08FE30E94544360E072
:1087300080EC0E94544361E080EC0E945443089511
:108740001F9390E087FD892F603408F0692F809394
:10875000DF0B6093E00B6695669566956093E10B81
:10876000803410F0805491E0692F80640E9454435B
:108770001091E10B186B60E0812F0E94544361E07F
:10878000812F0E9454431F9108951F93CF93DF932D
:10879000CDB7DEB721970FB6F894DEBF0FBECDBFC1
:1087A000982F15BA14BA8091DF0B803418F4D8983A
:1087B000DC9A02C0DC98D89A803429F4992319F005
:1087C00061E00E945443DA9AD99ADB9A00000000D3
:1087D000000013B3DB9819828981883020F48981E5
:1087E0008F5F8983F9CF8FEF84BB6091E00B80911D
:1087F000DF0B0E94A0438091940581111095812F79
:10880000992721960FB6F894DEBF0FBECDBFDF913A
:10881000CF911F91089581E00E94C54380E00E949E
:10882000C54399270895DF92EF92FF920F931F930C
:10883000CF93DF93CDB7DEB721970FB6F894DEBFA5
:108840000FBECDBFF82E80919A07A091DF0B882331
:10885000A9F5AA230CF4C4C09091E00B892F86954A
:1088600086958695E82FFF27F695FE2FEE27F7953C
:10887000E795EA0FF11DE053F84F4F2D55279770FC
:10888000692F77279A01062E02C0220F331F0A9400
:10889000E2F78081822B8083E058FF4F88E090E0F0
:1088A000861B970B02C0559547958A95E2F7808104
:1088B000842B8083AF5FA093DF0B92C0AA230CF4BC
:1088C0008FC0A03418F4D898DC9A02C0DC98D89AEB
:1088D000A03421F461E08A2F0E945443DA9AD99897
:1088E0000FEF04BB1091E00B177009F461C0DBB20D
:1088F00081E00E94C54380E00E94C543DBBA04BB0F
:10890000EF2CFF24012F11279701002E02C0220F08
:10891000331F0A94E2F7982F922B809194058111CE
:10892000909595BBDB9A000000000000DB9819824F
:108930008981883020F489818F5F8983F9CF809184
:10894000E00B885F682F8091DF0B0E94A04381E0DD
:108950000E94C54380E00E94C543DBBA9FEF94BBF1
:1089600028E030E0201B310B02C0F594E7942A95F3
:10897000E2F7982F9E29809194058111909595BBDF
:10898000DB9A000000000000DB98198289818830A2
:1089900020F489818F5F8983F9CF8091E00B885023
:1089A0009091DF0B682F892F8F5F0E94A04317C023
:1089B000809194058111F094F5BADB9A00000000D3
:1089C0000000DB9819828981883020F489818F5FCB
:1089D0008983F9CF8091DF0B8F5F8093DF0B15BA0E
:1089E00021960FB6F894DEBF0FBECDBFDF91CF91B9
:1089F0001F910F91FF90EF90DF9008953F924F925B
:108A00005F926F927F928F929F92AF92BF92CF921E
:108A1000DF92EF92FF920F931F93CF93DF93182F64
:108A200055248091E40B9091E50BE091E20BF091DD
:108A3000E30B03960995882E9924C401079633E029
:108A4000959587953A95E1F7482E8091E40B9091A2
:108A5000E50BE091E20BF091E30B04960995C82F2A
:108A60008091E40B9091E50BE091E20BF091E30B28
:108A700005960995EE24FF247090DF0B3090E00BF3
:108A80001C1750F0212F3327C82EDD24C6018C0F70
:108A9000911D281739071CF081E090E095C01C1B40
:108AA000052D511698F4E7018091E40B9091E50BA8
:108AB0008C0F9D1FE091E20BF091E30B0696099558
:108AC000E80EF11C0F5F2196011770F3842D992792
:108AD000E89E9001E99E300DF89E300D1124790139
:108AE000EC0CFD1C86E090E0E80EF91E8091E40B92
:108AF0009091E50B810F911DE091E20BF091E30B5A
:108B000006960995582ECC24C41408F055C0CC27DD
:108B1000DD27C819D9092896AA24BB246C2CDD248A
:108B2000D51478F500E010E08091E40B9091E50B0E
:108B30008E0D9F1D860D911DE091E20BF091E30BD0
:108B4000800F911F0995282FC50108968816990650
:108B50004CF4822F99270C2E02C0959587950A9484
:108B6000E2F7282F8091DE0B8F3F11F4822F02C095
:108B7000822F80950E941344D3940F5F1F4FD5140A
:108B800098F28091DE0B8F3F11F480E001C08FEFEF
:108B90000E9413448091E00B885F682F872D0E940C
:108BA000A043C394650C28E030E0A20EB31EC20FB0
:108BB000D31FC41408F4B3CF750C632D872D8F5FBA
:108BC0000E94A04380E090E0DF91CF911F910F9130
:108BD000FF90EF90DF90CF90BF90AF909F908F90DD
:108BE0007F906F905F904F903F9008950F931F93E9
:108BF000CF93DF93EC018091DF0B082F1127FE014B
:108C000084918823E9F0FE0184918A3091F4809167
:108C1000E40B9091E50BE091E20BF091E30B0396EE
:108C200009959091E00B980F692F802F0E94A04327
:108C300002C00E94FE442196FE018491882319F708
:108C4000DF91CF911F910F9108950F931F93CF93B1
:108C5000DF93EC018091DF0B082F11278881882397
:108C6000D9F088818A3091F48091E40B9091E50BE2
:108C7000E091E20BF091E30B039609959091E00BE4
:108C8000980F692F802F0E94A04302C00E94FE44CB
:108C900021968881882329F7DF91CF911F910F9129
:108CA00008950F931F93962F042F162F1770911B63
:108CB000692F0E94A04381E00E94C54380E00E948A
:108CC000C543482F212F33270F3F49F481E090E01F
:108CD00002C0880F991F2A95E2F7482B09C081E04E
:108CE00090E002C0880F991F2A95E2F780954823EB
:108CF000842F0E9413441F910F910895AF92BF9249
:108D0000CF92DF92EF92FF920F931F93CF93B82EE3
:108D1000162FA42EC22EC394462F4770141B5FEF4C
:108D2000D52EEC2CFF24642F772728E030E0C901F2
:108D3000861B970BE816F90664F48FEF90E02E1966
:108D40003F0902C0959587952A95E2F7D82ECC2D3C
:108D500002C0C8E0C41B8D2D992702C0880F991F3F
:108D60006A95E2F7D82E612F8B2D0E94A04300E078
:108D700081E00E94C54380E00E94C543282F982FC0
:108D800090959D218D2D80958223892B0E941344DF
:108D90000F5FA01668F78C2F99270896E816F9063A
:108DA000A4F0C85F185F612F8B2D0E94A04300E0E4
:108DB00081E00E94C54380E00E94C54380950E94E7
:108DC00013440F5FA016A0F7E6CFCC1530F52C2D7D
:108DD00033272C1B31098FEF90E002C0880F991FB9
:108DE0002A95E2F7D82ED094185F612F8B2D0E9420
:108DF000A04300E081E00E94C54380E00E94C5439B
:108E0000282F982F90959D218D2D80958223892B39
:108E10000E9413440F5FA01668F7CF911F910F9126
:108E2000FF90EF90DF90CF90BF90AF900895CF93D9
:108E3000C82F809194058C1741F02FE34FE760E035
:108E4000862F0E947E46C0939405CF9108959F92ED
:108E5000AF92BF92CF92DF92EF92FF920F931F9348
:108E6000CF93B82E162F942EC22EA02EC394462F29
:108E70004770141B6FEFD62EEC2CFF24642F77273E
:108E800028E030E0C901861B970BE816F90664F468
:108E90008FEF90E02E193F0902C0959587952A958E
:108EA000E2F7D82ECC2D02C0C8E0C41B8D2D992727
:108EB00002C0880F991F6A95E2F7D82E612F8B2D7B
:108EC0000E94A04300E081E00E94C54380E00E9430
:108ED000C543982F8FEFA81611F49D2903C08D2D3F
:108EE00080959823892F0E9413440F5F901658F79E
:108EF0008C2F99270896E816F90674F0C85F185F5A
:108F0000612F8B2D0E94A04300E08A2D0E94134404
:108F10000F5F9016D0F7ECCFCC1540F52C2D3327F2
:108F20002C1B31098FEF90E002C0880F991F2A9502
:108F3000E2F7D82ED094185F612F8B2D0E94A043AA
:108F400000E081E00E94C54380E00E94C543982F65
:108F50008FEFA81611F49D2903C08D2D80959823BD
:108F6000892F0E9413440F5F901658F7CF911F91DD
:108F70000F91FF90EF90DF90CF90BF90AF909F90B8
:108F800008952F923F924F925F926F927F928F92AD
:108F90009F92AF92BF92CF92DF92EF92FF920F9388
:108FA0001F93CF93DF93CDB7DEB726970FB6F89414
:108FB000DEBF0FBECDBF282E362E49832A83602EFA
:108FC0007E2C402E55245E824D82C201840D951D5B
:108FD000E3E0AE2EB12CA81AB90A882499249C8209
:108FE0008B82032D060DE02E2D81E21A122D160D17
:108FF000C12EC818472D6E2D8C2D0E945146081980
:10900000D12E3D81D31A472D602F8D2D0E945146C0
:109010001981120D1619F12EF80C472D6E2D8F2D7A
:109020000E945146ED80E10E472D602F8E2D0E944B
:1090300051461A81130D16190D81010F472D602F0E
:109040008F2D0E945146180D472D612F8E2D0E94A5
:109050005146472D602F8C2D0E945146472D612F80
:109060008D2D0E945146B7FE09C08B819C81A80EB0
:10907000B91EE6E0F0E0AE0EBF1E13C0C4012D81A4
:109080003E81821B930B880F991F880F991FA80E92
:10909000B91E8AE090E0A80EB91E215030403E83F0
:1090A0002D830894811C911CEB81FC813496FC83F8
:1090B000EB832D813E81281539050CF092CF72018A
:1090C000E40CF51C19811E19D22CD60C072D20E0BA
:1090D000412F632D8D2D0E9427478A81830D20E02B
:1090E000412F682F8D2D0E9427471A811E19F32CBE
:1090F000F60C212F40E06F2D822D0E942747212F53
:1091000040E06F2D8981820D0E94274726960FB679
:10911000F894DEBF0FBECDBFDF91CF911F910F91AD
:10912000FF90EF90DF90CF90BF90AF909F908F9087
:109130007F906F905F904F903F902F900895CF92C7
:10914000DF92EF92FF920F931F93D82EF62EC42E2C
:10915000E22E20E00E9427478F2D8E0D20E04C2D1F
:10916000682F8D2D0E9427472E2D40E06F2D8D2DCD
:109170000E9427472E2D40E06F2D8D2D8C0D0E94D3
:1091800027471F910F91FF90EF90DF90CF900895A8
:109190008F929F92AF92BF92CF92DF92EF92FF9207
:1091A0000F931F93CF93D82EE62EF42E122FA02EBE
:1091B000841749F4261710F4E22E162F1E190A2DD3
:1091C000212F40E00AC0621769F4481710F4D42E2A
:1091D000F82EFD180A2D20E04F2D6E2D8D2D0E94AA
:1091E0002747ECC0622F77274E2D5527CB01841BD4
:1091F000950B2F2D33272D1931098217930734F43E
:10920000461B570B421753070CF46CC0FD1430F487
:109210008D2D9E2DDF2CE12EF82E192FCF2CCD1861
:10922000812F99278E1991094C2D552728EC30E074
:10923000829FB001839F700D929F700D1124CB010E
:10924000BA010E94536C4B01EE2DBB248B2D992744
:10925000889E9001899E300D989E300D1124C90181
:1092600068EC70E00E94536CCE2DC60FC90168EC0B
:1092700070E00E94536C8436910514F0CF5F09C0F2
:10928000C90168EC70E00E94536C8D599F4F0CF43B
:10929000C1508D2D8B0D0A2D2C2F482F6E2F0E9423
:1092A000C8486C2D7727412F55272E2D3327CA010B
:1092B000821B930B861797072CF0E11618F4EC2FFE
:1092C000EF5F0BC0241B350B261737072CF01E153C
:1092D00018F4EC2FE15001C0EC2FB394CB1408F03C
:1092E000B5CF6CC01E1530F48D2D9E2DDF2CE12ED8
:1092F000F82E192FC12ECE188F2D99278D1991096F
:109300004C2D552728EC30E0829FB001839F700DD3
:10931000929F700D1124CB01BA010E94536C4B0136
:10932000ED2DBB248B2D9927889E9001899E300DB1
:10933000989E300D1124C90168EC70E00E94536CB6
:10934000CD2DC60FC90168EC70E00E94536C8436C5
:10935000910514F0CF5F09C0C90168EC70E00E946C
:10936000536C8D599F4F0CF4C1508E2D8B0D0A2DCF
:10937000282F4C2F682F8E2F0E94C8486C2D7727DE
:109380004F2D55272D2D3327CA01821B930B86178E
:1093900097072CF0DF1418F4EC2FEF5F0BC0241BA1
:1093A000350B261737072CF0FD1418F4EC2FE1507D
:1093B00001C0EC2FB394CB1408F0B4CFCF911F9120
:1093C0000F91FF90EF90DF90CF90BF90AF909F9064
:1093D0008F9008951F93CF9310E0812F9927F3E08A
:1093E000880F991FFA95E1F7682F80E00E94A0434B
:1093F000C0E080E00E941344CF5FC7FFFACF1F5F39
:10940000183058F3CF911F910895FC017183608348
:109410005383428317821682158214820895CF9354
:10942000DF93EC01E0E02C813D8121153105B9F09D
:109430008E819F81E881F981E80FF91FE081019613
:109440009F838E836A817B818617970720F00E9415
:109450003F6C9F838E83215030403D832C838E2F21
:109460009927DF91CF910895CF93DF93FC01EB0112
:109470002481358162177307A0F486819781860F56
:10948000971F97838683628173818617970720F0E1
:109490000E943F6C978386832C1B3D0B358324836E
:1094A00002C015821482DF91CF910895FC0186815C
:1094B000978122813381860F971FB9010E943F6CEB
:1094C0000190F081E02DE80FF91F80819927089520
:1094D000CF93DF93EC01462F2C813D816A817B8104
:1094E0002617370798F48E819F81820F931F0E9461
:1094F0003F6CE881F981E80FF91F40838C819D81E1
:1095000001969D838C838FEF90E002C080E090E015
:10951000DF91CF910895FC0140E050E02481358136
:10952000828193812817390710F441E050E0CA0185
:109530000895FC01158214820895CF93FC010190D7
:109540000020E9F73197E81BF90B9F0144275527C5
:10955000C4E260E070E0211531054105510579F064
:10956000FC018191C8276F5F7F4FCB01AA2797FD30
:10957000A095BA2F82179307A407B50790F38C2FF5
:109580009927CF9108950F931F93CF93DF93CDB772
:10959000DEB7A0970FB6F894DEBF0FBECDBF8091A7
:1095A0006C07813009F070C08091A1079091A207EB
:1095B000A091A307B091A40720EC3FEC48EF5FE334
:1095C000BC01CD010E94C069DC01CB01BF93AF9308
:1095D0009F938F9389E693E09F938F938E010F5F04
:1095E0001F4F1F930F930E94F86648EF5BE0509364
:1095F000F50B4093F40B8AE02FE633E0DA01F90132
:1096000001900D928A95E1F7B801CA010E94E465C4
:1096100069E773E08091F40B9091F50B0E94E4658B
:109620006AE873E08091F40B9091F50B0E94E46579
:109630008091F40B9091F50B0E949D4A8093F30B5F
:1096400099279F938F938DE893E09F938F9308E4DE
:109650001CE01F930F930E94F866B8018091F40BF1
:109660009091F50B0E94E4658091F40B9091F50BBD
:109670000E94814F0E94DF4F8DB79EB70E960FB6A6
:10968000F8949EBF0FBE8DBFA0960FB6F894DEBFB4
:109690000FBECDBFDF91CF911F910F910895089517
:1096A0008DE49CE00895CF93DF93CDB7DEB722978A
:1096B0000FB6F894DEBF0FBECDBFDC0196E0FD0112
:1096C00086818C3221F487818C3209F450C0FD01EF
:1096D000E90FF11D9F5F80818C32C9F7FD01E90F11
:1096E000F11D9F5F80818C32C9F7FD01E90FF11DEB
:1096F0009F5F80818C32C9F7FD01E90FF11D9F5FEB
:1097000080818C32C9F7FD01E90FF11D9F5F8081D7
:109710008C32C9F7FD01E90FF11D9F5F80818C320A
:10972000C9F7FD01E90FF11D9F5F80818C32C9F7F8
:10973000FD01E90FF11D9F5F80818C32C9F7BE01E9
:109740006F5F7F4FA90FB11DCD010E94916ADC01AF
:10975000CB01BC01CD010E94E968DC01CB01809303
:10976000EB0B9093EC0BA093ED0BB093EE0B2296CA
:109770000FB6F894DEBF0FBECDBFDF91CF91089535
:10978000FF920F931F93CF93DF93CDB7DEB722974E
:109790000FB6F894DEBF0FBECDBF8C0186E0F82E69
:1097A000F80186818C3221F487818C3209F496C0CD
:1097B000F801EF0DF11DF39480818C32C9F7BE01E1
:1097C0006F5F7F4FC8018F0D911D0E94916ADC0170
:1097D000CB01BC01CD010E94E968DC01CB01909373
:1097E000F70B8093F60BF801EF0DF11DF3948081D8
:1097F0008C32C9F7F801EF0DF11DF39480818C32A2
:10980000C9F7F801EF0DF11DF39480818C32C9F78F
:10981000F801EF0DF11DF39480818C32C9F7F80146
:10982000EF0DF11DF39480818C32C9F7F801EF0D33
:10983000F11DF39480818C32C9F7F801EF0DF11D11
:10984000F39480818C32C9F7F801EF0DF11DF39488
:1098500080818C32C9F7F801EF0DF11DF3948081FE
:109860008C32C9F7F801EF0DF11DF39480818C3231
:10987000C9F7F801EF0DF11DF39480818C32C9F71F
:10988000F801EF0DF11DF39480818C32C9F7F801D6
:10989000EF0DF11DF39480818C32C9F7F801EF0DC3
:1098A000F11DF39480818C32C9F7F801EF0DF11DA1
:1098B000F39480818C32C9F7BE016F5F7F4FC8017E
:1098C0008F0D911D0E94916ADC01CB018093EF0BFB
:1098D0009093F00BA093F10BB093F20B22960FB67E
:1098E000F894DEBF0FBECDBFDF91CF911F910F91D6
:1098F000FF900895FF920F931F93CF93DF93CDB7FF
:10990000DEB722970FB6F894DEBF0FBECDBF8C0135
:1099100096E0F92E98012A5F3F4FF80186818C323C
:1099200021F487818C3209F44CC0BE016F5F7F4FF8
:10993000C9010E94916ADC01CB018093F00C9093E5
:10994000F10CA093F20CB093F30CF801EF0DF11DA4
:10995000F39480818C32C9F7F801EF0DF11DF39477
:1099600080818C32C9F7F801EF0DF11DF3948081ED
:109970008C32C9F7F801EF0DF11DF39480818C3220
:10998000C9F7F801EF0DF11DF39480818C32C9F70E
:10999000F801EF0DF11DF39480818C32C9F7BE01FF
:1099A0006F5F7F4FC8018F0D911D0E94916ADC018E
:1099B000CB018093F40C9093F50CA093F60CB0932C
:1099C000F70C22960FB6F894DEBF0FBECDBFDF9125
:1099D000CF911F910F91FF900895BF92CF92DF9288
:1099E000EF92FF920F931F93CF93DF93CDB7DEB724
:1099F00026970FB6F894DEBF0FBECDBF6C0126E0F0
:109A0000B22E9C012A5F3F4FFC0186818C3221F4EB
:109A100087818C3209F461C1BE016F5F7F4FC9013C
:109A20000E94916ADC01CB01BC01CD010E94E96872
:109A30007B018C016093E60B7093E70B8093E80B3E
:109A40009093E90B20E137E240E050E00E94666C21
:109A500020936D0730936E0740936F075093700704
:109A6000C801B70124E630E040E050E00E94666C97
:109A7000DC01CB018093CF069093D006A093D10652
:109A8000B093D206C801B70120E137E240E050E0D0
:109A90000E94666CDC01CB01BC01CD0124E630E004
:109AA00040E050E00E94666C2093BE073093BF07F1
:109AB0004093C0075093C107F601EB0DF11DB3941D
:109AC00080818C32C9F7BE016F5F7F4FC6018B0D5D
:109AD000911D0E94916ADC01CB018093A80C9093A8
:109AE000A90CA093AA0CB093AB0C20E030E048EC9A
:109AF00052E4BC01CD010E94A368DC01CB01AE01A0
:109B00004D5F5F4FBC01CD010E94906920E030E0C5
:109B100048EC52E40E94C069DC01CB0120E030E057
:109B200040E752E4BC01CD010E94A368DC01CB01F7
:109B3000EB80FC800D811E819C01AD01C801B70145
:109B40000E946168DC01CB018093A80C9093A90C62
:109B5000A093AA0CB093AB0CF601EB0DF11DB394DE
:109B600080818C32C9F7F601EB0DF11D80818335C0
:109B700089F48091A80C9091A90CA091AA0CB091A5
:109B8000AB0CB0588093A80C9093A90CA093AA0C8E
:109B9000B093AB0CF601EB0DF11DB39480818C32C8
:109BA000C9F7BE016F5F7F4FC6018B0D911D0E94EB
:109BB000916ADC01CB018093AC0C9093AD0CA09327
:109BC000AE0CB093AF0C20E030E048EC52E4BC01A6
:109BD000CD010E94A368DC01CB01AE014D5F5F4F58
:109BE000BC01CD010E94906920E030E048EC52E4D5
:109BF0000E94C069DC01CB0120E030E040E752E484
:109C0000BC01CD010E94A368DC01CB01EB80FC808C
:109C10000D811E819C01AD01C801B7010E946168E0
:109C2000DC01CB018093AC0C9093AD0CA093AE0CF7
:109C3000B093AF0CF601EB0DF11DB39480818C3223
:109C4000C9F7F601EB0DF11D8081873589F480910C
:109C5000AC0C9091AD0CA091AE0CB091AF0CB05883
:109C60008093AC0C9093AD0CA093AE0CB093AF0C62
:109C7000F601EB0DF11DB39480818C32C9F7F6012A
:109C8000EB0DF11DB39480818C32C9F7C6018B0DA9
:109C9000911D0E9496658093EA0BF601EB0DF11D74
:109CA000B39480818C32C9F7F601EB0DF11DB394AA
:109CB00080818C32C9F7BE016F5F7F4FC6018B0D6B
:109CC000911D0E94916ADC01CB018093B00C9093AE
:109CD000B10CA093B20CB093B30C26960FB6F894C7
:109CE000DEBF0FBECDBFDF91CF911F910F91FF90CF
:109CF000EF90DF90CF90BF900895CF92DF92EF92D8
:109D0000FF920F931F93CF93DF93EC0110E08C81B0
:109D10009D81892B09F4D5C060E070E0CE010E94DE
:109D2000564A843241F0CE010E940F4A8C819D81B7
:109D3000892B91F754C01092490C10924A0C109242
:109D40004B0C10924C0C41E0E42EF12C8C819D8147
:109D50000197E816F90608F0B4C0B701CE010E94D9
:109D6000564A8D30C1F5C7010196BC01CE010E9453
:109D7000564A8A3081F5CE010E940F4A00E010E079
:109D800067010894C108D1080C151D05C0F43DE415
:109D9000E32E3CE0F32E0F34110530F4CE010E9487
:109DA0000F4AF701808303C0CE010E940F4A0F5F64
:109DB0001F4F0894E11CF11C0C151D0560F3035B9B
:109DC000134FF8011082CE010E940F4ACE010E946B
:109DD0000F4A1FEF07C00894E11CF11CB7CF1123F5
:109DE00009F46FC045E050E064E973E08DE49CE065
:109DF0000E94FB65892BC9F48DE49CE00E94ED4C28
:109E000080916C07813009F066C084E20E947B4F2C
:109E10008DE49CE00E94814F8DE00E947B4F8AE0A0
:109E20000E947B4F0E94C34A56C045E050E06AE959
:109E300073E08DE49CE00E94FB65892B29F48DE49E
:109E40009CE00E947A4C0EC045E050E060EA73E06E
:109E50008DE49CE00E94FB65892BB1F48DE49CE0CD
:109E60000E94C04B80916C078130A9F584E20E946A
:109E70007B4F8DE49CE00E94814F8DE00E947B4FE0
:109E80008AE00E947B4F27C045E050E066EA73E01D
:109E90008DE49CE00E94FB65892BE9F48DE49CE055
:109EA0000E94534B80916C078130A9F487E09BE1BD
:109EB0000E94C84F8DE49CE00E94814F0E94DF4FBA
:109EC0000AC02C813D818A819B812817390718F0AF
:109ED000CE010E94994A812F9927DF91CF911F913E
:109EE0000F91FF90EF90DF90CF900895909396059B
:109EF000809395050895E0919505F0919605099553
:109F00000895CF93DF93EC01892B61F0888188233A
:109F100049F0E0919505F091960589910995888120
:109F20008823B9F7DF91CF910895EF92FF920F93B5
:109F30001F93CF93DF938C017A01C0E0D0E0892B8F
:109F400001F1CE0121968617970728F4F801819137
:109F50008F018823B1F7C0E0D0E0CE15DF0588F48B
:109F6000F8018081E0919505F0919605882319F01C
:109F70000F5F1F4F01C080E209952196CE15DF05C6
:109F800078F3DF91CF911F910F91FF90EF9008959B
:109F9000CF93DF93EC01009779F0FC012196849137
:109FA000882351F0E0919505F09196050995FE0101
:109FB000219684918823B1F7DF91CF910895E091A4
:109FC0009505F09196058DE00995E0919505F09144
:109FD00096058AE009950895E82FFF27EF70F07045
:109FE000E75FF44E8491E0919505F091960509950F
:109FF00008951F93182F82958F700E94EC4F812F28
:10A000000E94EC4F1F9108950F931F938C01812F95
:10A0100099270E94F94F802F0E94F94F1F910F91AD
:10A020000895EF92FF920F931F937B018C01C8015B
:10A03000AA27BB270E940450C7010E9404501F9109
:10A040000F91FF90EF9008952F923F924F925F9261
:10A050006F927F928F929F92AF92BF92CF92DF9238
:10A06000EF92FF920F931F93CF93DF93CDB7DEB79D
:10A07000A2970FB6F894DEBF0FBECDBF69A3242E02
:10A080002AA337014801442351F017FF08C0EE24EA
:10A09000FF248701E618F7080809190902C084019E
:10A0A000730199A1692F772761507040222011F028
:10A0B00061507040362E18A22FE1422E512C4C0ECA
:10A0C0005D1EA82EBB24CC24DD24C801B701A60147
:10A0D00095010E94666CDC01CB01FC01E75FF44E48
:10A0E00084918F8FC801B701A60195010E94666C0B
:10A0F00079018A013A94AFEF3A1639F1C20101971A
:10A10000E114F10401051105C1F02C01C801B701EA
:10A11000A60195010E94666CDC01CB01FC01E75FA2
:10A12000F44E8491F2018083C801B701A601950124
:10A130000E94666C79018A0104C02C01EAA1DC014D
:10A14000EC933A94FFEF3F16C9F62220B9F097FE40
:10A1500005C08DE2D2018E932D0110C0C20101977E
:10A1600016141704180419042CF42C018BE2F201C4
:10A17000808304C02C0180E2D2018C9339A03A94F0
:10A18000BFEF3B1661F0E0919505F0919605D20185
:10A190008D912D0109953A94BFEF3B16A1F7A29638
:10A1A0000FB6F894DEBF0FBECDBFDF91CF911F91E8
:10A1B0000F91FF90EF90DF90CF90BF90AF909F9066
:10A1C0008F907F906F905F904F903F902F90089569
:10A1D0006F927F928F929F92AF92BF92CF92DF92B7
:10A1E000EF92FF920F931F93CF93DF93682E7A0124
:10A1F0008B0177240F2EF0E0AF2EF0E0BF2EF0E8B9
:10A20000CF2EFFE3DF2EF02DC72D20E030E040E021
:10A2100050E0C801B7010E94106988230CF4C1E026
:10A2200020E030E040E050E0C801B7010E9413692F
:10A23000181624F017FB109517F91095872CA60116
:10A240009501C801B7010E94A368DC01CB0120E0A1
:10A2500030E040E251E4BC01CD010E94106987FD6D
:10A260000EC020E030E040E251E4C601B5010E949A
:10A27000C0695B016C0183948EE0881500F7E09162
:10A280009505F0919605CC2311F08DE201C08BE28B
:10A2900009958824861408F06BC0A6019501C801B1
:10A2A000B7010E94A368DC01CB01BC01CD010E9473
:10A2B000E968DC01CB01982E8729C82FDD2720E033
:10A2C00030E040E85FE3C601B5010E9410698823D1
:10A2D00011F0CD2B49F031E0732EE0919505F0910E
:10A2E0009605892D805D05C0E0919505F091960554
:10A2F00080E2099520E030E040E85FE3C601B50167
:10A300000E941069882331F4E0919505F09196053B
:10A310008EE20995892D9927AA2797FDA095BA2F36
:10A32000BC01CD010E940669DC01CB01A6019501AB
:10A33000BC01CD010E94C069DC01CB019C01AD01D3
:10A34000C801B7010E946068DC01CB017C018D016E
:10A3500020E030E040E251E4C601B5010E94A3686C
:10A36000DC01CB015C016D018394861408F495CF68
:10A37000DF91CF911F910F91FF90EF90DF90CF90E1
:10A38000BF90AF909F908F907F906F9008957F9235
:10A390008F929F92AF92BF92CF92DF92EF92FF92F5
:10A3A0000F931F93CF93DF93CDB7DEB77888C9881B
:10A3B000DA8873E1A72EB12CAC0EBD1E08C088232D
:10A3C00009F47FC0E0919505F091960509959601F5
:10A3D0002F5F3F4F772021F0F6016901849103C080
:10A3E000F60180816901853251F72F5F3F4F772059
:10A3F00021F0F6016901849103C0F60180816901B1
:10A40000282F33272436310591F02536310524F4E1
:10A410002336310529F0D6CF2837310581F0D2CF48
:10A42000F50122E030E0A20EB31E8081CBCF6AE0BE
:10A43000862E912C50E1E52E57E2F52E04C040E126
:10A44000E42EF12C4701F50122E030E0A20EB31E0C
:10A45000008111818436D9F417FF09C01095019548
:10A460001F4FE0919505F09196058DE2099532E038
:10A47000E316F10460F00E151F0548F4C7016AE009
:10A4800070E00E943F6C7B0162307105A0F7C8014B
:10A49000B7010E943F6CFB01E75FF44E8491E091AD
:10A4A0009505F09196050995C801B7010E943F6C8A
:10A4B0008C01C701B4010E943F6C7B01672B39F707
:10A4C00086CF80E090E0DF91CF911F910F91FF90B8
:10A4D000EF90DF90CF90BF90AF909F908F907F9044
:10A4E000089508958DE99CE0089508951F93182F0D
:10A4F000DB01CA0173E0880F991FAA1FBB1F7A9561
:10A50000D1F79C01AD01220F331F441F551F80500E
:10A510009E4EA548BF4FBC01CD010E94666CDA017A
:10A52000C9018150112319F08093990001C089B9A4
:10A530001F91089540E850E067E276E088E09DE0F2
:10A540000E94054A40E150E067EA76E08AE19DE03A
:10A550000E94054A08950E949A521092BA061092DB
:10A56000B90688ED80939A0040E855E260E070E01B
:10A5700081E00E94765281E08093FF0C1092110DD1
:10A580001092250D1092240D7894089540E850E023
:10A5900067E975E080E09DE00E94054A40E150E0F7
:10A5A00067E176E082E19DE00E94054A08950E94FD
:10A5B000C6521092B8061092B70688ED8AB940E8E4
:10A5C00055E260E070E080E00E94765281E0809386
:10A5D000FE0C1092100D1092230D1092220D789403
:10A5E00008950E94D7520E94AB520895823040F4E1
:10A5F000E82FFF27EE0FFF1FE954F94F71836083A7
:10A6000008959927E3E0880F991FEA95E1F78050B4
:10A61000934F08959927F3E0880F991FFA95E1F772
:10A620008E5E924F0895982FE82FFF27DF01A250EA
:10A63000B34F8C918823E9F3992319F060939C0020
:10A6400001C06CB9E250F34F10820895682F80E08A
:10A650000E9413530895682F81E00E9413530895B8
:10A66000CF93DF93EB01E82FFF27A3E0EE0FFF1F4F
:10A67000AA95E1F7E050F34F82819381009751F062
:10A6800084819581009731F0CF010E940F4A888321
:10A6900081E090E0DF91CF910895CF93DF93CDB724
:10A6A000DEB721970FB6F894DEBF0FBECDBFBE0157
:10A6B0006F5F7F4F81E00E943053882319F08981BA
:10A6C000992702C08FEF9FEF21960FB6F894DEBF57
:10A6D0000FBECDBFDF91CF910895CF93DF93CDB75C
:10A6E000DEB721970FB6F894DEBF0FBECDBFBE0117
:10A6F0006F5F7F4F80E00E943053882319F089817B
:10A70000992702C08FEF9FEF21960FB6F894DEBF16
:10A710000FBECDBFDF91CF9108959927B3E0880F89
:10A72000991FBA95E1F78050934F0E94994A089576
:10A7300020E030E0E82FFF2783E0EE0FFF1F8A952F
:10A74000E1F7E050F34F84819581892B11F421E0EA
:10A7500030E0C9010895992733E0880F991F3A9591
:10A76000E1F78E5E924F0E94684A0895682F80E05C
:10A770000E94AB530895682F81E00E94AB53089567
:10A780001F93182F9927FC01E05FF24F21E02083EF
:10A7900043E0880F991F4A95E1F78E5E924F0E9421
:10A7A0000F4A682F812F0E9413531F910895AF9273
:10A7B000BF92CF92DF92EF92FF920F931F93CF93AE
:10A7C000DF93B82E8B01C82EDD24F60163E0EE0F77
:10A7D000FF1F6A95E1F7EE5EF24F84819581840F49
:10A7E000951F228133818217930760F5411551052A
:10A7F00049F1F801A1908F01C0E0D0E07A010894FE
:10A80000E108F108CE15DF0580F4F80121918F01F0
:10A81000C60153E0880F991F5A95E1F7622F8E5EAB
:10A82000924F0E94684A2196EDCFEB2DFF27E05F03
:10A83000F24F81E080836A2D8B2D0E94135381E0BB
:10A8400090E002C080E090E0DF91CF911F910F91E6
:10A85000FF90EF90DF90CF90BF90AF900895CF938F
:10A86000DF93282FA82FBB27ED01C05FD24F88812F
:10A870008823E1F0FD0173E0EE0FFF1F7A95E1F709
:10A88000EE5EF24F84819581892B79F0222339F095
:10A890008AE19DE00E940F4A80939C000BC082E1F8
:10A8A0009DE00E940F4A8CB905C01882A250B34F98
:10A8B00081E08C93DF91CF910895E82F882329F0D0
:10A8C00080919C0080939C0002C08CB18CB9FF27C2
:10A8D000E250F34F81E0808308951F93CF93DF937D
:10A8E000882319F010919C0001C01CB1282F332738
:10A8F000E901C20FD31FFE01E954F94F8081918114
:10A90000892B31F00190F081E02D812F099520C035
:10A91000E3E0220F331FEA95E1F7612FC901805070
:10A92000934F0E94684A882341F4FE01EE5DF24F86
:10A93000808191810196918380831A3049F48091BE
:10A940002C0490912D04806290932D0480932C040C
:10A95000DF91CF911F9108951F920F920FB60F9222
:10A9600011242F933F934F935F936F937F938F9314
:10A970009F93AF93BF93EF93FF9380E00E942F5478
:10A98000FF91EF91BF91AF919F918F917F916F91C7
:10A990005F914F913F912F910F900FBE0F901F909D
:10A9A00018951F920F920FB60F9211242F933F9379
:10A9B0004F935F936F937F938F939F93AF93BF93C7
:10A9C000EF93FF9381E00E942F54FF91EF91BF918D
:10A9D000AF919F918F917F916F915F914F913F9137
:10A9E0002F910F900FBE0F901F9018951F920F92EE
:10A9F0000FB60F9211242F933F934F935F936F9352
:10AA00007F938F939F93AF93BF93EF93FF9380E0D8
:10AA10000E946D54FF91EF91BF91AF919F918F91E3
:10AA20007F916F915F914F913F912F910F900FBE4A
:10AA30000F901F9018951F920F920FB60F9211242E
:10AA40002F933F934F935F936F937F938F939F9336
:10AA5000AF93BF93EF93FF9381E00E946D54FF91FA
:10AA6000EF91BF91AF919F918F917F916F915F9186
:10AA70004F913F912F910F900FBE0F901F901895FF
:10AA8000C19AB99ABB98BA9AB89A6C9A689A699A14
:10AA900070986B986A986D986E9A8EB180912C041C
:10AAA00090912D04826090932D0480932C046F98D4
:10AAB0000895282F80912C0490912D048D7F9093E0
:10AAC0002D0480932C042FB9779BFECF08950E940C
:10AAD00059558FB1992708956B986A98BE9AC69870
:10AAE0008FEF0E9459558FEF0E9459558FEF0E94AA
:10AAF00059558FEF0E945955C69A0895CF92DF920B
:10AB0000FF920F931F93F82E6A01122F6B986A9889
:10AB1000BE9AC6981770812F80620E9459558D2D5C
:10AB200099278F70806C0E945955812F80630E94F5
:10AB300059558C2D0E945955812F80610E9459557D
:10AB40000295000F007EFF0CFF0C8CE1F822802F95
:10AB50008F290E945955C69A1F910F91FF90DF903F
:10AB6000CF900895EF92FF920F931F936B986A987E
:10AB7000C6988CE50E94595580E00E946755992738
:10AB8000AA27BB27EE24F82E092F1A2F80E00E9457
:10AB900067559927AA27BB27E82AF92A0A2B1B2BD6
:10ABA000102F0F2DFE2CEE2480E00E946755992770
:10ABB000AA27BB27E82AF92A0A2B1B2BC69AC80109
:10ABC000B7011F910F91FF90EF900895DC01CB0129
:10ABD00020E030E040EA50E4BC01CD010E94A368CF
:10ABE000DC01CB012CE53FE842EC5DE3BC01CD018B
:10ABF0000E946168DC01CB012AEF3DEE4BE65AE38F
:10AC0000BC01CD010E94A368DC01CB01BC01CD01D8
:10AC100008959B01AC0197FD03C00E94066916C010
:10AC2000DC01CB0181709070A070B0705695479593
:10AC300037952795822B932BA42BB52BBC01CD01E7
:10AC40000E9406699B01AC010E9461682CEC3CECFF
:10AC50004CE45AE40E94A368DC01CB01BC01CD01A5
:10AC60000895889880916A00826080936A0080913C
:10AC70006A008E7F80936A0089B7816089BF0895DA
:10AC800080912C0490912D048E7F90932D048093BD
:10AC90002C040E94B255DC01CB01BC01CD010E9405
:10ACA0000956DC01CB01BC01CD010E94E655DC0157
:10ACB000CB018093460D9093470DA093480DB09320
:10ACC000490D089580912C0490912D0480FF06C0B9
:10ACD0000E9440560E94B3150E94911608958091DB
:10ACE0002C0490912D048E7F90932D0480932C043E
:10ACF00080912C0490912D0480FFFACF80912C0438
:10AD000090912D048E7F90932D0480932C040895B0
:10AD10001F920F920FB60F9211248F939F938091E1
:10AD20002C0490912D04826090932D0480932C0428
:10AD30009F918F910F900FBE0F901F9018951F92AB
:10AD40000F920FB60F9211248F939F9380912C0432
:10AD500090912D04816090932D0480932C049F91F9
:10AD60008F910F900FBE0F901F90189596B1987FFE
:10AD7000982B96B9089527B12F73992736E0880F3D
:10AD8000991F3A95E1F7282B27B90895379A3598F6
:10AD900087E00E94B65680E00E94BB563D98339AE9
:10ADA00010924A0D7894089533983798089597B182
:10ADB000907E8F71982B97B90895349A369A08959A
:10ADC00086B1992780749070089510924A0D97B1BA
:10ADD000907E8F71982B97B9349A369A3699FECF18
:10ADE00084B1282F332785B19927982F8827822B64
:10ADF000932B08950E94E55696958795969587958D
:10AE0000992708951F920F920FB60F9211248F93D6
:10AE100081E080934A0D8F910F900FBE0F901F908D
:10AE200018950F931F93CF93DF938C01EB01672B42
:10AE300039F0F80181918F010E9459552197C9F786
:10AE4000DF91CF911F910F9108950F931F93CF938F
:10AE5000DF938C01EB0180E00E946755F80181933C
:10AE60008F01219741F080E00E946755F80181939E
:10AE70008F012197C1F7DF91CF911F910F91089515
:10AE8000EF92FF920F931F938091C4069091C50695
:10AE900009977C01002711278091C6069091C7066B
:10AEA0009C0144275527C801B7010E94146CDC019E
:10AEB000CB01BC01CD011F910F91FF90EF90089540
:10AEC000CF93DF93CDB7DEB721970FB6F894DEBFEF
:10AED0000FBECDBF1982C79861E070E084E094E0B6
:10AEE0000E94115761E070E0CE01860F971F0E940B
:10AEF0002557C79A8981992721960FB6F894DEBF06
:10AF00000FBECDBFDF91CF910895EF92FF920F93C7
:10AF10001F93CF936B9A6A9AC0E0BF9A0E946057C2
:10AF20008093BF06992788739070809769F488E0B2
:10AF300091E09093C5068093C40680E090E19093E1
:10AF4000C7068093C606C1E08091C4069091C506ED
:10AF50007C01002711278091C6069091C7069C01AD
:10AF600044275527C801B7010E94146CDC01CB01AE
:10AF70008093C0069093C106A093C206B093C30607
:10AF80008C2F9927CF911F910F91FF90EF900895EB
:10AF9000EF92FF920F931F93DC01CB012FEFE22E74
:10AFA000F12C012D112DBC01CD01A80197010E94AA
:10AFB000886CDC01CB01E81AF90A0A0B1B0BC801EB
:10AFC000B7011F910F91FF90EF9008952F923F923C
:10AFD0004F925F926F927F928F929F92AF92BF92A9
:10AFE000CF92DF92EF92FF920F931F93CF93DF9355
:10AFF000CDB7DEB768970FB6F894DEBF0FBECDBFF2
:10B000009A8789874B875C876D877E870F87188B28
:10B01000298B3A8B1B8A1C8A1D8A1E8A20E030E00D
:10B0200040E050E06F85788989899A89261737072B
:10B03000480759070CF01EC1EB84FC840D851E8562
:10B040008B899C89AD89BE89E80EF91E0A1F1B1FDA
:10B05000A091C406B091C506B88FAF8B5D01CC241A
:10B06000DD24C801B701A60195010E94886C190171
:10B070002A01C601B5010E94146CDC01CB01370125
:10B080004801681A790A8A0A9B0A2F8538894989F2
:10B090005A896B897C898D899E89261B370B480BC1
:10B0A000590BA216B306C406D50614F4A6019501E1
:10B0B000DA01C901860D971DA81DB91DEF89F88D0C
:10B0C0007F0100271127E816F9060A071B073CF441
:10B0D00057016801A618B708C808D90802C0590165
:10B0E0006A018091C0039091C103A091C203B09105
:10B0F000C3038201710149E0EE0CFF1C001F111F08
:10B100004A95D1F7A801970120703E7F4F7150708A
:10B11000822B932BA42BB52B89839A83AB83BC837F
:10B120006B9A6A9A0E9460578823E4F78C818D831A
:10B1300035E0432E512C4C0E5D1E8B818E838A810F
:10B140008F8389818887C79864E070E0C2010E947C
:10B150001157C79A8091D4039091D503A091D6033B
:10B16000B091D7032FEF31E040E050E0622273222C
:10B170008422952286299729A829B92989839A8327
:10B18000AB83BC830E9460578823E4F78C818D8356
:10B190008B81F20181838A81828389818383C7982D
:10B1A00064E070E0C2010E941157B50189859A855B
:10B1B0002B893C89820F931F0E9411574B895C8910
:10B1C0006D897E894A0D5B1D6C1D7D1D4B8B5C8BD3
:10B1D0006D8B7E8BC79A8091DE039091DF03A091E7
:10B1E000E003B091E10320E03EEF4FE150E0E222C6
:10B1F000F322042315238E299F29A02BB12B8983A9
:10B200009A83AB83BC838C818D838B81F201818394
:10B210008A81828389818383C79864E070E0C20158
:10B220000E941157C79A2B853C854D855E856B8999
:10B230007C898D899E89260F371F481F591F809151
:10B24000C0069091C106A091C206B091C30628170E
:10B2500039074A075B0774F48B899C89AD89BE89DD
:10B260002F85388949895A8982179307A407B5071A
:10B270000CF4E2CE0E9460578823E4F76B897C8946
:10B280008D899E8968960FB6F894DEBF0FBECDBF3C
:10B29000DF91CF911F910F91FF90EF90DF90CF90B2
:10B2A000BF90AF909F908F907F906F905F904F90E6
:10B2B0003F902F9008952F923F924F925F926F92FE
:10B2C0007F928F929F92AF92BF92CF92DF92EF9236
:10B2D000FF920F931F93CF93DF93CDB7DEB768979D
:10B2E0000FB6F894DEBF0FBECDBF9A8789874B8714
:10B2F0005C876D877E870F87188B298B3A8B1B8A1B
:10B300001C8A1D8A1E8A20E030E040E050E06F85F4
:10B31000788989899A8926173707480759070CF0D1
:10B32000D8C0EB84FC840D851E858B899C89AD89F2
:10B33000BE89E80EF91E0A1F1B1FA091C406B0911A
:10B34000C506B88FAF8B5D01CC24DD24C801B701E1
:10B35000A60195010E94886C39014A01C601B50118
:10B360000E94146CDC01CB0117012801281A390A4C
:10B370004A0A5B0A2F85388949895A896B897C89F1
:10B380008D899E89261B370B480B590BA216B306D5
:10B39000C406D50614F4A6019501DA01C901820D8F
:10B3A000931DA41DB51D6F89788D7B010027112782
:10B3B000E816F9060A071B072CF4E218F30804093B
:10B3C000150902C079018A016B9A6A9A0E94605736
:10B3D0008823E4F78091AC039091AD03A091AE0374
:10B3E000B091AF0359E0660C771C881C991C5A95E4
:10B3F000D1F720E03EEF4FE150E062227322842239
:10B40000952286299729A829B9294FEF51E060E0B4
:10B4100070E0242235224622572282299329A4292A
:10B42000B52989839A83AB83BC838C818D838B817F
:10B430008E838A818F8389818887C79864E070E0D2
:10B44000CE0105960E9411578091B003682F77278F
:10B45000CE0101960E941157B70189859A85AB8963
:10B46000BC898A0F9B1F0E942557C79A2B893C894C
:10B470004D895E892E0D3F1D401F511F2B8B3C8B2C
:10B480004D8B5E8B2B853C854D855E856B897C89DC
:10B490008D899E89260F371F481F591F8091C0062E
:10B4A0009091C106A091C206B091C3062817390732
:10B4B0004A075B0774F48B899C89AD89BE892F8507
:10B4C000388949895A8982179307A407B5070CF46C
:10B4D00028CF6B897C898D899E8968960FB6F894F0
:10B4E000DEBF0FBECDBFDF91CF911F910F91FF90B7
:10B4F000EF90DF90CF90BF90AF909F908F907F9014
:10B500006F905F904F903F902F900895DC01FC0169
:10B510002281538147813481832F8350883030F5D5
:10B52000852F9927841B910949973CF0442311F4F6
:10B53000223018F03A3019F408953330B9F02F5F03
:10B54000283179F420E04F5F473009F4422FE32F90
:10B55000FF27E65FFB4F8081581711F4522F3F5FA2
:10B560005F5FFD0134832283538347830895EF9205
:10B57000FF920F931F93CF93DF937B018C01EA011E
:10B580002CE330E040E050E00E94666CDC01CB012F
:10B590008883C801B7012CE330E040E050E00E940E
:10B5A000666C79018A01CA01B9012CE330E040E000
:10B5B00050E00E94666CDC01CB018983C801B701B1
:10B5C0002CE330E040E050E00E94666C79018A0193
:10B5D000CA01B90128E130E040E050E00E94666C09
:10B5E000DC01CB018A83C801B70128E130E040E0EB
:10B5F00050E00E94666C2B5F3F4FC901059667E0E3
:10B6000070E00E943F6C8F83E0E5F1E06DE671E051
:10B610004E2F5527CA0183709070892B61F46EE616
:10B6200071E0EE2321F0E43611F0E83C21F4F15012
:10B6300011F06DE671E02617370720F0261B370B57
:10B64000EF5FE4CF4459584F5E834D8360FF05C0E0
:10B650002B33310510F02F5F3F4F41E080910B04F9
:10B6600099272817390770F0E42FFF27E65FFB4F73
:10B670008081281B31094F5FE42FFF27E65FFB4FD6
:10B680008081EECF4C83822F8F5F8B83DF91CF91B0
:10B690001F910F91FF90EF900895982FF89480914B
:10B6A000C207982389278093C2077894892F992706
:10B6B0000895982FF894809189079823892780937B
:10B6C00089077894892F99270895982FF894809165
:10B6D000D40B809589230E944D5B992708950E9481
:10B6E000595B0E944D5B992708952F923F924F928C
:10B6F0005F926F927F928F929F92AF92BF92CF9202
:10B70000DF92EF92FF920F931F93CF93DF93CDB70A
:10B71000DEB72A970FB6F894DEBF0FBECDBF1C016F
:10B720005A016B012D831F830E8327FF02C01D82E8
:10B7300005C02D81263214F065E26D831886210143
:10B74000C10188969A87898720E030E040E050E088
:10B75000C601B5010E94106988235CF4EE81FF8167
:10B7600080819181826091838083D7FAD094D7F8C9
:10B77000D094AE014F5F5F4FC601B5010E94906942
:10B780005B016C0189819A81AB81BC8120E030E052
:10B7900040E050E0BC01CD010E941069882309F40B
:10B7A0004AC009851A852AC02DEC3CEC4CEC5DE3BF
:10B7B000C401B3010E94C069DC01CB01AE014F5F3F
:10B7C0005F4FBC01CD010E949069DC01CB012AE9E9
:10B7D00039E941E251E4BC01CD010E94C069DC01BC
:10B7E000CB01BC01CD010E94E968DC01CB01805D89
:10B7F000F80182938F01F885FF5FF88769807A806E
:10B800008B809C8020E030E040E050E0C401B30138
:10B810000E941069882319F02016310628F28985C4
:10B820009A850817190768F5F80181918F01F201CF
:10B8300081932F01F4CF20E030E040E050E0C601DA
:10B84000B5010E9413691816E4F405C05701680198
:10B8500098859150988720E030E040E251E4C6019D
:10B86000B5010E94C0697B018C0120E030E040E816
:10B870005FE30E94106987FDE9CFE982FA820B83BA
:10B880001C83EE81FF814081518153FF15C0F885F3
:10B89000FD3F94F02F2F332727FD30956D81862FA4
:10B8A000992787FD90950196281739072CF4546045
:10B8B000EE81FF8151834083EE81FF818081918100
:10B8C0009C012070347092FD03C0FD81FF5FFD83F9
:10B8D0006D81062F112707FD1095020D131D232BD7
:10B8E00039F0E8858E2F992787FD9095080F191F4D
:10B8F0000215130520F5F10158C089859A8548166F
:10B90000590600F520E030E040E251E4C601B501FF
:10B910000E94C069AE014F5F5F4F0E9490695B015A
:10B920006C0189819A81AB81BC81BC01CD010E94EF
:10B93000E968DC01CB01805DF20181932F010415E0
:10B940001505D8F6E985FA850E171F0718F0F101DD
:10B9500017A22CC02801F80180818B5F80838A3375
:10B960001CF120E331E3F80120832016310628F48E
:10B9700082918F018F5F808313C0F8013083F88537
:10B98000FF5FF887EE81FF818081918192FF08C07F
:10B990002414350410F4F20120830894411C511C36
:10B9A000F80180818A33FCF6F2011082F8858F2F2E
:10B9B000992787FD90952A960FB6F894DEBF0FBEA3
:10B9C000CDBFDF91CF911F910F91FF90EF90DF904E
:10B9D000CF90BF90AF909F908F907F906F905F902F
:10B9E0004F903F902F9008952F923F924F925F92E9
:10B9F0006F927F928F929F92AF92BF92CF92DF927F
:10BA0000EF92FF920F931F93CF93DF93CDB7DEB7E3
:10BA1000EE970FB6F894DEBF0FBECDBF88249924F1
:10BA200054013C0178AF6FAB1A011EAA1DAAFC019C
:10BA300017821682838181FD1EC48FEF9FEF2EC473
:10BA40008FA998AD019698AF8FAB6DA97EA960FFC5
:10BA5000FEC389AD80538A30C8F499AD903331F478
:10BA6000552021F463FD02C07160ABC18AE0589E8D
:10BA7000502C1124E9AD5E0EF0ED5F0E57FE02C0B2
:10BA80005FE7552E63FDF7C3452CF5C329AD255659
:10BA90002EAF233028F089AD8554833008F01EC1C5
:10BAA000F10184E090E0280E391EE080F1800281EF
:10BAB00013814701580163FD02C046E0542E37EB65
:10BAC000C32E3FEFD32EC622D722DEAACDAAC801AD
:10BAD000B7010E948069892BB9F08EE48B8389833A
:10BAE00081E48A83FE013496FCAFEBAFFEADF33008
:10BAF00008F0ADC28981805E89838A81805E8A83F5
:10BB00008B81805E8B83A3C2C801B7010E948769C5
:10BB1000892BC9F089E48B838EE48A8386E4898348
:10BB2000CE0104969CAF8BAF20E030E040E050E0C7
:10BB3000C801B7010E9410698823C4F68DE28C8386
:10BB4000FE013596D1CF80E092E0C82AD92ADEAA3C
:10BB5000CDAAE9AD8E2F992787FD90958734910561
:10BB600009F45CC0883491053CF48534910599F062
:10BB70008634910561F17FC38636910541F18736A0
:10BB8000910524F48536910531F075C3873691050A
:10BB900009F444C070C38E010B5C1F4F252DB50105
:10BBA000A401CE010D960E94755B8DAFFCEF4F0E88
:10BBB00015140CF44A94CE010D969CAF8BAFFC018A
:10BBC00001900020E9F731978E2E881ABFC18DA908
:10BBD0009EA994609EAB8DAB8E010B5C1F4F252DF3
:10BBE000B501A401CE010D960E94755B8DAF1514B1
:10BBF0000CF44A94FE013D96FCAFEBAFFDAD1F1671
:10BC000054F4EBADFCAD01900020E9F731978E2E96
:10BC10002BAD821A9BC1852C839498C18DA99EA9B6
:10BC200098609EAB8DAB252D552009F421E08E0147
:10BC30000B5C1F4FB501A401CE010D960E94755BF0
:10BC40008DAF8DA99EA992FF27C08DAD850D815026
:10BC5000882E87FD15C08DAD881694F09E012F5F4C
:10BC60003F4FE82DFF27E7FDF095E20FF31F848596
:10BC7000803331F48A9487FC03C09DAD89168CF71C
:10BC800087FC03C0EDAD8E1614F4552418C0582C53
:10BC9000FDAD5F1A539413C0852C15147CF49E01DE
:10BCA0002F5F3F4FE82DFF27E7FDF095E20FF31FD1
:10BCB0008485803319F48A941814A4F3582CE82D41
:10BCC000FF27E7FDF095EC0FFD1F16868DA99EA9B5
:10BCD00092FD8DCF29AD225029AF68CF63FF04C0FC
:10BCE000552011F421E0522EE9AD8E2F992787FDC2
:10BCF00090958936910509F4A5C08A3691057CF5A1
:10BD00008335910509F483C084359105BCF48B32E9
:10BD1000910509F443C08C3291054CF480329105B1
:10BD200009F43FC08332910509F443C08AC28D32C1
:10BD30009105E9F18E329105F1F183C283369105C7
:10BD400009F442C0843691052CF48835910509F434
:10BD5000AEC077C28436910509F474C072C28037D0
:10BD6000910509F49FC08137910544F48C36910503
:10BD700039F18F36910509F492C063C28537910578
:10BD800009F497C08637910524F48337910521F192
:10BD900058C28837910509F48AC053C260617EABEE
:10BDA0006DAB8DA99EA980629EAB8DAB64C26068AD
:10BDB00008C0606406C068607EAB6DAB55245BC292
:10BDC00064607EAB6DAB57C2F10182E090E0280E5B
:10BDD000391E80804A943BC1F10182E090E0280E38
:10BDE000391EA081B1814D0163FF09C0852D9927BE
:10BDF00087FD9095BC01CD010E9409661FC0FD0121
:10BE000001900020E9F73197EA1BEAAF18C0F10171
:10BE100082E090E0280E391E0190F081E02D4F0164
:10BE200063FF09C0852D992787FD9095BC01CF013F
:10BE30000E94D96503C0CF010E94D0658AAF9AAD38
:10BE4000491A05C162FF0AC0F10184E090E0280EA2
:10BE5000391E20813181428153810CC0F10182E081
:10BE600090E0280E391E808191819C01442737FD86
:10BE70004095542F49015A0157FF0BC062607EABB9
:10BE80006DABB094A09490948094811C911CA11CE3
:10BE9000B11C8DA99EA98F7B9EAB8DAB27C098E06E
:10BEA0009AAF07C060647EAB6DABE8E7E9AFF0E145
:10BEB000FAAF6DA97EA962FF0AC0F10184E090E0AB
:10BEC000280E391E20813181428153810AC0F1013F
:10BED00082E090E0280E391E808191819C014427E8
:10BEE000552749015A016F7C7EAB6DABFE0131963F
:10BEF000FCAFEBAF6F01FAADEF2EFF240027112747
:10BF0000C501B401A80197010E94666CDC01CB0158
:10BF1000EBADFCAD80838A3024F0F9AD8F0F8152F8
:10BF200001C0805DEBADFCAD8193FCAFEBAFC50113
:10BF3000B401A80197010E94666C49015A012115BC
:10BF4000310541055105E1F68BAC8C184DA95EA970
:10BF5000CA0182739070892B09F04A9446FF0DC084
:10BF6000842D992787FD9095FAADF03121F49EEF4D
:10BF7000492E480E02C0482E4A9443FF0EC0252D7C
:10BF8000332727FD3095882D99278217930724F0B2
:10BF9000477F5EAB4DAB01C058188DA99EA983FFAA
:10BFA00002C0451801C0481880789170892B51F45F
:10BFB000842D4A94181634F4B30180E290E00E9474
:10BFC000A666F6CF8DA99EA981FF04C0B3018DE2BC
:10BFD00090E00BC084FF04C0B3018BE290E005C089
:10BFE00085FF05C0B30180E290E00E94A6668DA99E
:10BFF0009EA986FF10C0B30180E390E00E94A66670
:10C000002AAD203141F4B301E9AD8E2F992787FD88
:10C0100090950E94A6668DA99EA990FF0AC0842DC6
:10C020004A94181634F4B30180E390E00E94A666A7
:10C03000F6CF8DA99EA983FF0AC0852D5A941816A4
:10C0400034F4B30180E390E00E94A666F6CF8DA998
:10C0500087FD0AC0842D4A94181634F4B30180E297
:10C0600090E00E94A666F6CFF9ADF33631F4882D44
:10C07000B301992787FD9095C0C029AD2337B9F446
:10C080008AAD81508AAF8F3F09F4CEC0F401808120
:10C090000894811C911CB301992787FD90950E94FB
:10C0A000A6669AAD91509AAF9F3F81F7BDC0E9ADAA
:10C0B000E33581F4FAADF150FAAFFF3F09F4B4C0B3
:10C0C000F4018491B30199270E94A6660894811C0B
:10C0D000911CF0CF8DA99EA991FF92C092FF1DC027
:10C0E0002DAD1216B4F421502DAF2F3F81F0EBADE2
:10C0F000FCAD8191FCAFEBAFB301992787FD909523
:10C100000E94A666FDADF150FDAFFF3F81F71DAE69
:10C110000FC0B30180E390E009C0EBADFCAD8191AD
:10C12000FCAFEBAFB301992787FD90950E94A666FF
:10C1300015142CF4B3018EE290E00E94A6668DA93E
:10C140009EA992FF20C08DADF82FFF5FFDAF0DC0FF
:10C15000852D5A941816BCF4B30180E390E00E9438
:10C16000A6668DAD282F2F5F2DAF88238CF30BC0D3
:10C17000852D5A9418167CF4882DB301992787FDD4
:10C1800090950E94A666EBADFCAD8191FCAFEBAF44
:10C19000882E882369F78DA99EA992FD45C0B30119
:10C1A000F9AD8F2F992787FD90950E94A6662DAD3A
:10C1B00021502DAF27FF09C0B3018DE290E00E940E
:10C1C000A6668DAD81958DAF05C0B3018BE290E081
:10C1D0000E94A6666AE070E0EDAD8E2F992787FD7C
:10C1E00090950E94536C4B015C01B301C401C09651
:10C1F0000E94A666B301C501C0960E94A66614C03F
:10C200008E010F5F1F4F8BAD9CAD8017910761F0C2
:10C21000EBADFCAD8291FCAFEBAFB301992787FD8D
:10C2200090950E94A666EFCF8DA987FF0DC0842D43
:10C230004A9418164CF4B30180E290E00E94A6667E
:10C24000F6CFB3010E94A6661EAA1DAA14C099AD1E
:10C25000953249F481E090E09EAB8DAB5524452C9E
:10C26000EAE0EAAF08C0B301F9AD8F2F992787FD47
:10C2700090950E94A666F301838183FF04C0EFA915
:10C28000F8ADF49103C0EFA9F8ADF081F9AF29AD95
:10C29000222309F0D5CBF30186819781EE960FB664
:10C2A000F894DEBF0FBECDBFDF91CF911F910F91EC
:10C2B000FF90EF90DF90CF90BF90AF909F908F90C6
:10C2C0007F906F905F904F903F902F9008952F92A6
:10C2D0003F924F925F926F927F928F929F92AF9216
:10C2E000BF92CF92DF92EF92FF920F931F93CF9363
:10C2F000DF93CDB7DEB7C254D0400FB6F894DEBF9F
:10C300000FBECDBFCC24DD2476011FAE1EAE4C0186
:10C3100078AF6FAB3A018EE0A7E1B4E0FE01319651
:10C320000D9001928A95E1F723961FAE23971BAEDD
:10C330001AAE00E010E02FEF3FEF3DAF2CAFF4015D
:10C340001783068322961FAF0EAF2297838180FD4D
:10C350009FC38FEF9FEFD0C34FA958AD4F5F5F4F83
:10C3600058AF4FAB23965FAD2397A52EBB2440E279
:10C37000242E312C2A203B20A5FEB7C08EE548167E
:10C3800041F40115110509F081C0A6FC7FC050647D
:10C3900025C19DE2491639F501151105A9F4842D31
:10C3A000869586958695FE013196E80FF11D27E06A
:10C3B000422281E090E002C0880F991F4A94E2F780
:10C3C0002685282B268707C023963FAD2397386004
:10C3D00023963FAF23970F5F1F4F5AC3B401C80185
:10C3E0000E9428674DC04DE5441609F04FC0011565
:10C3F0001105A9F2A3FE03C08C8980628C8BA6FE76
:10C400000EC0FE0131960FE110E08685809586878B
:10C4100001501040319617FFF8CF00E210E0A4FC65
:10C4200007C0F30182E090E0680E791EC080D180E1
:10C43000852D5A94181624F5C4010E9463668C0158
:10C440009FEF0F3F1907E1F0202F802F86958695EB
:10C450008695FE01E80FF11D8785992787FD909548
:10C46000277002C0959587952A95E2F780FFB6CF91
:10C47000A4FCDECFF60100830894C11CD11CD8CFE8
:10C480002396EFAD2397E4FDA3C207C1A3FE28C006
:10C490002396FFAD2397F77F2396FFAF23972EAD0B
:10C4A0002415F0F4BE016F5F7F4F41E050E08EAD88
:10C4B000982F969596959695FB01E90FF11D87703B
:10C4C0009A0102C0220F331F8A95E2F78685822BDC
:10C4D00086878EAD9FAD01969FAF8EAF841538F3E2
:10C4E000E42DFF27FFAFEEAF5ACFA0FE96C2F5E2D4
:10C4F0004F1641F423962FAD23972E7F23962FAF0F
:10C500002397B8C2942D90539A3058F43FE75316AE
:10C5100011F4552404C08AE0589E502C1124590E61
:10C52000B7C2842D992787FD90950E94E96C482E0B
:10C53000282F332727FD30952936310509F4C3C04C
:10C540002A363105DCF42436310509F4BCC0253621
:10C5500031057CF42B35310509F429C22C35310520
:10C5600024F42A32310571F133C223363105D1F179
:10C570002FC2283631050CF496C18AC22037310506
:10C5800009F498C02137310564F42E36310509F4D9
:10C5900076C12F3631050CF083C02C363105D1F031
:10C5A00017C22537310509F487C0263731052CF429
:10C5B0002337310509F43FC00BC22837310509F490
:10C5C00079C006C223964FAD2397406123964FAFA3
:10C5D00023975EC223965FAD2397546023965FAF87
:10C5E000239756C2A4FC07C0F30182E090E0680ED6
:10C5F000791EC080D1809FE7591611F431E0532E87
:10C60000852D5A9418160CF0E3C1C4010E9463668C
:10C610008C01EFEF8F3F9E0709F448C2A4FCF0CFD6
:10C62000F60180830894C11CD11CEACFB401C80173
:10C630000E9428672DC0A4FC07C0F30122E030E06F
:10C64000620E731EC080D180C4010E9463668C019B
:10C650000E94DA6C892BC1F73FEF0F3F130709F4F3
:10C6600025C2852D5A9418169CF4C8010E94DA6CD4
:10C67000892BE1F6A4FC05C0F60100830894C11CD7
:10C68000D11CC4010E9463668C018F5F9F4F49F7E4
:10C6900023965FAD239754FD9BC1F601108298C18C
:10C6A00088E089AF23969FAD2397926023969FAF32
:10C6B000239709C0E0E1E9AF2396FFAD2397F2602D
:10C6C0002396FFAF2397C4010E9463668C010E94EA
:10C6D000DA6C892BC1F72FEF0F3F120709F4E6C17F
:10C6E0000D3211F00B32A9F45A9415140CF0DEC17E
:10C6F0000D3239F423963FAD2397386023963FAF30
:10C700002397C4010E9463668C018F5F9F4F09F4D9
:10C71000CDC1003389F5CC24DD2476015A9415145B
:10C720000CF07DC0C4010E9463668C015FEF8F3FF7
:10C73000950709F474C00E94E96C8837C1F48FE64C
:10C74000481631F094E6491619F0E5E74E1629F43B
:10C75000B401C8010E94286762C0F0E1F9AFC401CA
:10C760000E9463668C018F5F9F4F31F458C039E699
:10C77000431611F448E049AFCC24DD247601C8010A
:10C780000E94E96CC0979FAF8EAF8A30910544F04C
:10C79000C1979FAF8EAF97FD03C00A969FAF8EAF34
:10C7A0008EAD9FAD97FD08C0E9AD8E2F99272EADB8
:10C7B0003FAD281739072CF0B401C8010E94286743
:10C7C00021C089AD282F332744275527C701B6013B
:10C7D0000E94146C6B017C01EEADFFADCF01AA2766
:10C7E00097FDA095BA2FC80ED91EEA1EFB1E5A94BB
:10C7F000151444F4C4010E9463668C018F5F9F4F3F
:10C8000009F0BDCF23962FAD239723FF08C0F094E6
:10C81000E094D094C094C11CD11CE11CF11C23965F
:10C820004FAD2397242F332724FDD2C0C901867032
:10C830009070069731F4F30182E090E0680E791E63
:10C840000EC021FF06C0F30122E030E0620E731E2D
:10C8500010C0C301029622FF0AC0F3013C010190FF
:10C86000F081E02DC082D182E282F382B1C0F30177
:10C870003C010190F081E02DD182C082A9C0A4FCCE
:10C88000A7C0F30142E050E0640E751EA081B181A3
:10C89000F401868197818D939C939AC0B401C8015D
:10C8A0000E9428675FC0C4010E9463668C010E94D9
:10C8B000DA6C892BC1F7FFEF0F3F1F0709F4F6C0B1
:10C8C0000D3211F00B3289F40D3239F423962FAD6D
:10C8D0002397286023962FAF2397C4010E94636695
:10C8E0008C018F5F9F4F09F4E1C02FE0C22ED12C45
:10C8F000CC0EDD1E760196E3A92EB12CAC0EBD1E2A
:10C90000CA14DB0478F515146CF5B801CE01019654
:10C910000E94EF65892B11F2053611F0053489F478
:10C920001B86F70101937F01C4010E9463668C019D
:10C93000FFEF8F3F9F07B1F08D3231F08B3221F046
:10C940000DC00E3209F41D86F70101937F01C40169
:10C950000E9463668C018F5F9F4F21F05A94EA1406
:10C96000FB0488F2F701108260E070E0C6010E94CB
:10C97000916ADC01CB016C017D012396FFAD239709
:10C98000F3FF04C0F7FAF094F7F8F094F30122E013
:10C9900030E0620E731E0190F081E02DC082D182E2
:10C9A000E282F38285E48B878EE28D8711C0239625
:10C9B0003FAD2397306223963FAF239781013FAE6F
:10C9C0002EAE80E2FE013F9611928A95E9F760C093
:10C9D000F4018681978122962EAD3FAD22972817CC
:10C9E000390774F423963FAD239734FD06C04AAD52
:10C9F0005BAD4F5F5F4F5BAF4AAF1DAE1CAE09C072
:10CA00005EE6451609F052C08FEF0F3F180709F494
:10CA10004DC023961FAE23973BC095E2491689F47B
:10CA2000E1E02396EFAF2397FAE0F9AFF401068037
:10CA3000F781E02D2296FFAFEEAF22978FE7582EB9
:10CA400027C0842D992787FD90950E94DA6C892B49
:10CA500089F0C4010E9463668C010E94DA6C892B04
:10CA6000C1F7FFEF0F3F1F0709F1B401C8010E9492
:10CA700028670EC0C4010E9463668C018F5F9F4FC0
:10CA8000A9F0842D992787FD90950817190771F44F
:10CA9000F401838183FF04C0EFA9F8AD449003C083
:10CAA000EFA9F8AD4080442009F056CC2396FFADA5
:10CAB00023972F2F332720FF13C0F40186819781FE
:10CAC00022964EAD5FAD2297481759074CF424FDCE
:10CAD00005C08AAD9BAD01969BAF8AAF1DAE1CAE63
:10CAE0000F5F1F4F39F4EAADFBADEF2B19F48CAD9E
:10CAF0009DAD02C08AAD9BADCE5BDF4F0FB6F89403
:10CB0000DEBF0FBECDBFDF91CF911F910F91FF9080
:10CB1000EF90DF90CF90BF90AF909F908F907F90DD
:10CB20006F905F904F903F902F900895FC01882761
:10CB30009927E89421912223F1F02032D9F329306A
:10CB4000C9F32A30B9F32C30A9F32D3099F32637E5
:10CB500089F32B3219F02D3221F46894219122238C
:10CB600051F0203344F02A3334F420530E941466E9
:10CB7000820F911DF3CF8115910521F01EF4809550
:10CB8000909501960895FB01DC0140FF05C002C0AD
:10CB900005900D9205900D9242505040C8F70895AF
:10CBA000FC0105900020E9F7809590958E0F9F1F5E
:10CBB0000895FC010590615070400110D8F78095F0
:10CBC00090958E0F9F1F0895FB01DC010D900020B2
:10CBD000E9F7119701900D920020E1F70895FC010B
:10CBE0000190061629F00020D9F788279927089583
:10CBF0003197CF010895FB01DC014150504030F0E6
:10CC00008D910190801919F40020B9F7881B990BB8
:10CC10000895FC016150704001900110D8F7809593
:10CC200090958E0F9F1F08957AE0979F902D879F74
:10CC3000802D910D112408950F931F93CF93DF93AF
:10CC40008C01EB01009711F4672BC1F16EE070E0ED
:10CC500081E090E00E944467FC01892B71F180E83B
:10CC60008383209771F0D387C28781E88383809183
:10CC70004B0D90914C0D892B21F4F0934C0DE093CA
:10CC80004B0D01151105C9F0118700878381826062
:10CC9000838380914D0D90914E0D892B71F4F0930B
:10CCA0004E0DE0934D0D80914F0D9091500D892BBD
:10CCB00021F4F093500DE0934F0DCF01DF91CF9110
:10CCC0001F910F910895CF93DF93EC014B81842F37
:10CCD000992780FF2EC086FF09C04F7B4B838E8132
:10CCE0009F8101969F838E838A812CC082FF11C011
:10CCF000E881F9818081282F332727FD3095211580
:10CD0000310519F440624B8314C03196F983E883EE
:10CD100013C0EA85FB85CE0109959C0197FF0CC0E5
:10CD20008B8199272F5F3F4F11F4806101C0806292
:10CD30008B838FEF9FEF07C08E819F8101969F832A
:10CD40008E83822F9927DF91CF9108950F931F93A0
:10CD5000CF93DF938C01EB018B81992781FF1CC05E
:10CD600082FF0DC02E813F818C819D81281739075C
:10CD700064F4E881F9810193F983E88306C0E885CA
:10CD8000F985802F0995892B39F48E819F81019631
:10CD90009F838E83C80102C08FEF9FEFDF91CF91F9
:10CDA0001F910F910895CF93DF93CDB7DEB745E084
:10CDB00050E04C0F5D1FFA0121913191AF01A0911C
:10CDC0004D0DB0914E0DFD01838188608383B901C3
:10CDD00080914D0D90914E0D0E94F45CE0914D0DAF
:10CDE000F0914E0D2381277F2383DF91CF9108950A
:10CDF0000F931F93CF93DF93CDB7DEB72E970FB668
:10CE0000F894DEBF0FBECDBF0D891E892F89388DE6
:10CE100086E08C831A8309838FEF9FE79E838D833F
:10CE2000AE01475E5F4FB901CE0101960E94F45CEE
:10CE3000EF81F885E00FF11F10822E960FB6F8945F
:10CE4000DEBF0FBECDBFDF91CF911F910F9108952F
:10CE5000AC01FB012381822F992780FF06C086FD4C
:10CE600004C08FEF4F3F580719F48FEF9FEF0895DD
:10CE7000428320642F7D2383868197810197978346
:10CE80008683842F992708950F931F93CF93DF9361
:10CE9000869F8001879F100D969F100D1124C80159
:10CEA0000E946067EC01009729F0A80160E070E043
:10CEB0000E945668CE01DF91CF911F910F91089586
:10CEC000CF93DF93AC01029710F442E050E020E0F2
:10CED00030E0A091530DB091540DBD01F9011097B0
:10CEE00009F44CC08D919C9111978417950731F1ED
:10CEF0004817590738F42115310519F0821793079F
:10CF000008F49C01FD01A281B381109759F7211506
:10CF10003105A1F1C901841B950B049708F4A901FF
:10CF2000DB01E0E0F0E0109749F18D919C911197C1
:10CF300082179307F9F44217530779F4ED018A81B8
:10CF40009B81309719F09383828304C09093540D92
:10CF50008093530DCD0102964AC0241B350BFD0171
:10CF6000E20FF31F41935193225030402D933C9395
:10CF7000CF013DC0FD01A281B381D5CF8091510D7C
:10CF80009091520D892B41F48091270490912804AF
:10CF90009093520D8093510DE0912504F091260459
:10CFA000309741F4EDB7FEB78091290490912A049F
:10CFB000E81BF90BA091510DB091520D9F012A1B56
:10CFC0003B0B2417350788F0CA010296281739074A
:10CFD00060F0CD01840F951F02969093520D8093BF
:10CFE000510D4D935D93CD0102C080E090E0DF9143
:10CFF000CF910895CF93DF93009709F454C0DC01DB
:10D000001297ED011B821A828091530D9091540D5D
:10D01000009721F1FC0140E050E0EA17FB0718F10E
:10D02000ED01FB83EA832D913C911197C20FD31F31
:10D03000CE0102968E179F0771F48A819B81280F7B
:10D04000391F2E5F3F4F11963C932E93828193811F
:10D05000FD01938382834115510559F4B093540D1A
:10D06000A093530D20C0AF010280F381E02D3097D3
:10D07000A1F6EA01BB83AA83CA01029628813981FD
:10D08000820F931F8A179B0771F48D919C911197C2
:10D09000280F391F2E5F3F4F39832883FD0182817E
:10D0A00093819B838A83DF91CF910895DC0140FFB8
:10D0B00003C001C06D936D9342505040D8F708955E
:10D0C0005058192EEFD001D0D2C0BA17620773079B
:10D0D00084079507B1F188F40EF410940B2EBA2F43
:10D0E000A02D062E622F202D072E732F302D082EF7
:10D0F000842F402D092E952F502DFF275523B9F051
:10D10000591B49F0573E98F0469537952795A795B6
:10D11000F0405395C9F776F0BA0F621F731F841F52
:10D1200030F4879577956795B795F040939517FA02
:10D130000F2E0895BF1BBB27BA0B620B730B840B1A
:10D14000F6CFDEF6DBC0AED001D091C0552359F04A
:10D15000992369F09F575F57951B33F442F4903839
:10D1600011F4915805C09BC091589F3F09F4C6C067
:10D17000BB27112462177307840730F4660F771FEB
:10D18000881FBB1F915098F311D00F920FD00F92B0
:10D190000DD0A0E82617370748071B0609F0A0485E
:10D1A000BA2F602D7F918F9100240895A0E800246C
:10D1B000621773078407B10528F0621B730B840B99
:10D1C000B1090A2A660F771F881FBB1FA69581F732
:10D1D000089597FB73D09F3738F0FEE9F91B982F1D
:10D1E000872F762F6B2F05C086C0969587957795EC
:10D1F0006795F150D0F73EF49095809570956195C4
:10D200007F4F8F4F9F4F0895E89403C097FB0EF414
:10D21000F3DFB62F672F782F892F9EE9002427C0D0
:10D220000ED05EF004C00BD026F001C008D019F07B
:10D2300020F48FEF089580E0089581E0089597FB32
:10D24000092E052600F8689430D0E89407FC07C042
:10D25000621773078407950721F008F40094079478
:10D26000989408959A95BB0F661F771F881F112405
:10D270009923A1F08823B2F79F3F59F0BB0F48F4E0
:10D2800021F4002011F460FF04C06F5F7F4F8F4FC7
:10D290009F4F881F9795879597F908952CC09FEF0A
:10D2A00080EC0895052E092607FA440F551F5F3FAD
:10D2B00079F0AA27A51708F051E04795880F991F24
:10D2C0009F3F31F0BB27B91708F091E0879508958B
:10D2D0009F919F911124E3CF97FB880F991F9F3F48
:10D2E00031F0BB27B91708F091E0879508959F9119
:10D2F0009F911124D4CF66277727882799270895EF
:10D300009F3F59F4803C49F481E099270895906843
:10D310008923872386238395B9F38827992708953E
:10D32000DBDFCF93DF93D52FC42F55274427332737
:10D3300022279923D9F09F37C8F0F92F98DF592F6A
:10D34000482F372F262FF63968F443DF5FDFC030D0
:10D35000CD0721F069937993899399939058DF9140
:10D36000CF91AFCE9927882777276627C030CD0782
:10D3700021F02993399349935993DF91CF9177CF36
:10D3800091DF01D074CF992339F0552329F09F57AD
:10D390005F57950F13F49AF1B1CF91589F3FE1F386
:10D3A000629FA12D0F92BB27639FA00DB11DEE2799
:10D3B000729FA00DB11DEE1FAF93AA27649FB00D01
:10D3C000E11D739FB00DE11DAA1F6627829FB00D5E
:10D3D000E11DA61F5527749FE00DA11D551F839FBA
:10D3E000E00DA11D561F849FA00D511D852F7A2F82
:10D3F0006E2F1F900F9088231AF4939539F44FCF16
:10D40000000C111CBB1F661F771F881F0128089581
:10D410003CD038F02ED060F186F021F436D009F0FF
:10D420003EF53DCF5F934F933F932F93CAD12F91FA
:10D430003F914F915F91A4DF2EC127D098F389F0DF
:10D440000894E795D901AA2329F4AB2FBE2FF85FE2
:10D45000D0F3E8CFFF5F30F7A695E0F7F73908F390
:10D4600009F09F779F939F77DDDFEF91E0789E270C
:10D470000895E894FC01EE0FFF1F309661057105D9
:10D4800019F0F395F14097FB0895E894FA01EE0F37
:10D49000FF1F30962105310519F0F395F14057FB38
:10D4A000089597FDFCCE992309F40895482F14DFC1
:10D4B000F92FFF57F5959F1B9F1BFF93D8DEFF9217
:10D4C000EF92DF92CF92BF92AF929F928F926B01B9
:10D4D0007C01405847953327222740685FE3B60117
:10D4E000C70149015A010E94A3689401A5010E9445
:10D4F00061684FEF5FEF53D19B01AC018216930639
:10D50000A406B50661F78F909F90AF90BF90CF9023
:10D51000DF90EF90FF905F91DFDE950FA8CE772729
:10D520006627B3D0C82FD92F7F936F939D2E8C2E53
:10D5300009910032E9F30930D9F30637C9F30C3009
:10D54000B9F30A30A9F30D3099F353D070D0EEF14E
:10D550005BDE17FB97F9C92ED82EE72EF62E88270B
:10D560000062053651F4099144D04BD0992319F04B
:10D5700017FD3DC036C017FD8195ECE8F0E0182F8F
:10D580009C2D8D2D7E2D6F2D9F7798178707760701
:10D590006105D9F01A0D3AF411957896912F9B19DF
:10D5A00097322CF504C0912F9B0D9732D4F49C2D0B
:10D5B000112359F0159538F4B2D0EF93FF93E0DEC4
:10D5C000FF91EF91F5CF3496F3CFEF91FF91E030DB
:10D5D000EF0711F081929082ECE0CDB7DEB70C94AA
:10D5E000C56C9C2D9F678FE77FEF6FEFEECF83DEDB
:10D5F000ECCF11270B3219F00D3211F4106809919C
:10D6000008958827992700338CF011F415FF0AC07C
:10D610000A3364F41062992329F40E9414660F708F
:10D62000800F911D9D2E8C2E0991EDCF0895689449
:10D6300062DEBB24BA94AA240E3229F416FD24C05B
:10D64000106406F11DC00033FCF019F4E89415FFD6
:10D6500012C00A33CCF410629F3084F4B394E8947F
:10D660005527442733272AE00E94146C0F70600F5F
:10D67000711D811D911D16FDAA9402C016FFA39471
:10D680009D2E8C2E0991D8CF0895AA27BB27FF91F4
:10D69000EF910C94A96C092E99234AF052E441EBC6
:10D6A00032E7683173078407950758F0F8CD9F7704
:10D6B00052E44EEA3CEA603573078407950708F0A8
:10D6C0001ACE0F925FE348EB3AEA2BE359DEFF9262
:10D6D000EF92DF92CF9250E04CE022DEECEBF0E0F4
:10D6E0002BD05F2D4E2D3D2D2C2DCF90DF90EF9028
:10D6F000FF90FEE94595441F551FF51B55274068CF
:10D7000004C04695379527955795FA95D2F7452F3A
:10D71000550F550B44D00F9007FC06C00895559146
:10D7200045913591259108959B01AC019FE380E8D7
:10D73000772766270C94A368FF92EF92DF92CF922F
:10D74000BF926B017C01B59016D0B590BB2069F0FB
:10D750009F938F937F936F93B601C7010CD02F9146
:10D760003F914F915F910E94A368BF90CF90DF904F
:10D77000EF90FF900895D3DF02C09601A701EF93C9
:10D78000FF930E94C069FF91EF91C9DFEF93FF9370
:10D790000E946168FF91EF91BA9479F708959CDD3A
:10D7A000992359F0AA27940FA51F43F032F04FEFA9
:10D7B00050E09417A50714F45ACD9DCD0EF02FC05C
:10D7C00029C097FD6CCD88DD992309F468CDFF92BF
:10D7D000EF92DF92CF92C92E9FE38F77EAEDF0E0D0
:10D7E000ABDF0C2CC92ED82EE72EF62E602D6E57EF
:10D7F000770B872F972F0ADD5FE341E332E728E1BC
:10D80000BFDD5C2D4D2D3E2D2F2DCF90DF90EF9065
:10D81000FF9057CC9FEF80E870E060E008959FE7AD
:10D8200080E870E060E00895629FD001739FF0018E
:10D83000829FE00DF11D649FE00DF11D929FF00DA0
:10D84000839FF00D749FF00D659FF00D9927729FD7
:10D85000B00DE11DF91F639FB00DE11DF91FBD0162
:10D86000CF0111240895991B79E004C0991F9617E0
:10D8700008F0961B881F7A95C9F780950895AA1B12
:10D88000BB1B51E107C0AA1FBB1FA617B70710F0AB
:10D89000A61BB70B881F991F5A95A9F780959095DD
:10D8A000BC01CD01089597FB092E07260AD077FD0C
:10D8B00004D0E5DF06D000201AF4709561957F4F03
:10D8C0000895F6F7909581959F4F0895A1E21A2E3D
:10D8D000AA1BBB1BFD010DC0AA1FBB1FEE1FFF1F14
:10D8E000A217B307E407F50720F0A21BB30BE40B64
:10D8F000F50B661F771F881F991F1A9469F76095AB
:10D900007095809590959B01AC01BD01CF01089564
:10D9100097FB092E05260ED057FD04D0D7DF0AD07D
:10D92000001C38F450954095309521953F4F4F4F4E
:10D930005F4F0895F6F790958095709561957F4FAC
:10D940008F4F9F4F08952F923F924F925F926F9209
:10D950007F928F929F92AF92BF92CF92DF92EF927F
:10D96000FF920F931F93CF93DF93CDB7DEB7CA1B00
:10D97000DB0B0FB6F894DEBF0FBECDBF09942A882B
:10D98000398848885F846E847D848C849B84AA84D3
:10D99000B984C884DF80EE80FD800C811B81AA8160
:10D9A000B981CE0FD11D0FB6F894DEBF0FBECDBF2B
:10D9B000ED010895911125C0803251F08A3041F077
:10D9C0008C3031F08D3021F0893011F08B3099F7A7
:10D9D00008958F931BD08F9109F080620895E1998B
:10D9E000FECFBFBBAEBBE09A11960DB20895F7DF34
:10D9F00001921A94E1F70895019010D01A94E1F77A
:10DA0000089599278827089585FDFBCF806291119D
:10DA1000F8CF8136ECF38B37DCF70895E199FECF30
:10DA2000BFBBAEBB0DBA11960FB6F894E29AE19A5D
:04DA30000FBE089588
:10DA3400C42A2D4752D4423E00001F003B005A0026
:10DA440078009700B500D400F300110130014E01B5
:10DA540001010000DC4300007A4400002545000079
:10DA6400A040000025450000404000007244000032
:10DA7400004000001A440000803F0000F243000010
:10DA840000000000DC43CDCCCCBD0000DC43000032
:10DA940000C000005C430000FAC400005C4353690A
:10DAA4006E6B746F6E00000000000000005374651C
:10DAB4006967746F6E000000000000005A656974A5
:10DAC4006F66667365740000000000547261636BD6
:10DAD400696E74657276616C6C004C6175747374F4
:10DAE4006165726B6500000000426C7565746F6F50
:10DAF4007468000000000000534D5320203D0000D6
:10DB0400000000000000004D6F646500000000008C
:10DB14000000000000002563256325632563256359
:10DB240025632563256325632563256325632563B1
:10DB340000504D4C522C32362C30312C30312C309C
:10DB440033333900504D4C522C32342C30322C307B
:10DB54003130302C3033393800504D4C522C323463
:10DB64002C30322C303130312C3033393900446F81
:10DB740000467200536100536F004D6F004469000A
:10DB84004D6900000000466C75672053746172741F
:10DB9400203D20256C750D0A00466C756720456E86
:10DBA400646520203D20256C750D0A00466C756760
:10DBB4007A65697420203D20253032642068202550
:10DBC400303264206D696E2E0D0A0065A203245064
:10DBD4004E4D52583131312C5741524D2A34440D57
:10DBE4000A0024504E4D52583130382C4747412CAE
:10DBF4004753412C524D432C5654472A36440D0A60
:10DC04000024504E4D52583130332C4747412C316B
:10DC14002C4753412C312C524D432C312C56544714
:10DC24002C312A36360D0A0001050A14274E00004D
:10DC3400004E4F00004F000000534F0000530000FF
:10DC44000053570000570000004E5700000000002A
:10DC54000024504E4D52583131312C434F4C442AFC
:10DC640034300D0A004A414E00464542004D4152AF
:10DC740000415052004D4149004A554E004A554C0E
:10DC84000041554700534550004F4B54004E4F56EA
:10DC94000044455A000000000025302E316600245F
:10DCA40050424235302C302C002C302E302C302C6D
:10DCB400302C312E30302C302C003030002A2532DC
:10DCC4002E3078004750474741004750565447008C
:10DCD4004750475341004750524D43000000005203
:10DCE400040000005401000000560100000053002D
:10DCF400000000550000000060000000006100000A
:10DD04000000840000000087000000008300000081
:10DD14000086000000008800000000890000000068
:10DD24008200000000850000000058000000005937
:10DD340000000000570000000050001F1D1F1E1FA0
:10DD44001E1F1F1E1F1E1F30313233343536373825
:0CDD54003945652E000000550D20000030
:00000001FF
